:020000040800F2
:1000000000000220EDF40008919800089398000881
:10001000959800089798000899980008000000003B
:100020000000000000000000000000009B98000895
:100030009D980008000000009F980008A198000803
:1000400031F5000831F5000831F5000831F50008F8
:1000500031F5000831F5000831F5000831F50008E8
:1000600031F5000831F5000831F500082D6400086D
:1000700031F5000831F5000831F5000831F50008C8
:1000800031F5000831F5000831F5000831F50008B8
:1000900031F5000831F5000831F50008ED9A000847
:1000A00031F5000831F5000831F5000831F5000898
:1000B000999A000831F5000831F5000831F500087B
:1000C00031F5000831F5000831F5000831F5000878
:1000D00031F5000831F50008019C000831F50008F1
:1000E00031F5000831F50008A598000831F5000841
:1000F00031F5000831F5000831F5000831F5000848
:1001000031F5000831F5000831F5000831F5000837
:1001100031F5000831F5000831F5000831F5000827
:1001200031F5000831F5000831F5000831F5000817
:1001300031F5000831F5000831F5000831F5000807
:1001400031F5000831F5000831F50008D5980008B0
:1001500031F5000831F5000831F5000831F50008E7
:1001600031F5000831F5000831F5000831F50008D7
:1001700031F5000831F5000831F5000831F50008C7
:0801800031F5000831F500081B
:100188003CA0050800000020A40B0020A80B0020BC
:1001980038CF0020064B07481A68074B1A60074BF0
:1001A80000221A70064B01221A7001F02ABC00BF07
:1001B800143C0020300E002020420020FC3B002090
:1001C800B43B002008B5034801F01BFC024B002299
:1001D8001A7008BDC0100020B43B002008B5054BBC
:1001E800012200201A7004F053FC0348BDE80840BF
:1001F80001F007BC38420020641100202DE9F041CD
:10020800144C204602F089FF00201349134A02F0DB
:100218003BFD1349134A0746002002F035FD1249F9
:10022800124A0646002002F02FFDD22105463A4622
:1002380023460A2002F040FED22132462346FA2005
:1002480002F03AFE5A20D2212A462346BDE8F04160
:1002580002F032BE780F0020D68F0508CD010008C5
:10026800DF8F0508E5010008E78F05089D010008F4
:1002780008B5054B012200201A7004F009FC034858
:10028800BDE8084001F0BDBB3842002064110020E1
:10029800044B054800221A70044B02221A7001F020
:1002A800B0BB00BFFC3B0020780F0020B43B00200F
:1002B80008B5034801F0A5FB024B00221A7008BDDF
:1002C800C0100020B43B00202DE9F041144C20461A
:1002D80002F023FF00201349134A02F0D5FC13490A
:1002E800134A0746002002F0CFFC1249124A06467C
:1002F800002002F0C9FCD22105463A4623460A20CE
:1003080002F0DAFDD221324623465A2002F0D4FD0B
:10031800AA20D2212A462346BDE8F04102F0CCBDEE
:10032800300E0020D68F0508B9020008F08F0508A6
:1003380099020008F98F050879020008002008B51D
:1003480004F0A6FB064B00221A70064B1B78022B02
:100358000CBF05480548BDE8084001F052BB00BF86
:1003680038420020B43B0020780F0020300E0020D7
:1003780010B5084C204602F0D0FE00200649074A76
:1003880002F082FCD22102462346E620BDE8104056
:1003980002F092BDAC120020029005084503000847
:1003A80010B5074C4FF6E071206801F0C1FF2068D6
:1003B800044901F06BFFBDE8104003F0E7B800BF47
:1003C800A80B00200B90050810B5074C4FF6E071FC
:1003D800206801F0ADFF2068044901F057FFBDE82F
:1003E800104003F0D3B800BFA80B002020900508E8
:1003F80010B5074C4FF6E071206801F099FF2068AE
:10040800044901F043FFBDE8104003F0BFB800BF46
:10041800A80B00203590050810B5074C4FF6E07181
:10042800206801F085FF2068044901F02FFFBDE82E
:10043800104003F0ABB800BFA80B00204A90050895
:100448002DE9F04F724C85B0FFF7AAFF002004F0A9
:100458001FFB23790BB9FFF7CBFF63790BB9FFF7C4
:10046800DBFFA3790BB9FFF7AFFF694B5A79002A75
:1004780000F0C2801A79002A00F0BE809979002223
:100488001A715A7101B19A71624BDFF8B8A1DFF89D
:10049800B8811A70604EDAF80010604CDFF8ACB121
:1004A800DFF8AC915E4F5F4D4FF4967006F02FF871
:1004B800D8F800104FF4987006F029F831684FF416
:1004C8009A7006F024F821684FF49C7006F01FF823
:1004D800554A4FF49E701168019206F018F8DBF83F
:1004E80000104FF4A07006F012F8D9F800104FF47D
:1004F800A27006F00CF839684FF4A47006F007F8FB
:1005080029684FF4A67006F002F8484B4FF4A8701B
:100518001968029305F0FBFFDFF838C14FF4AA70A1
:10052800DCF80010CDF80CC005F0F1FFDFF804E1AD
:100538004FF4AC70DEF8001005F0E9FF019AD4ED35
:10054800001A92ED002A9AED000AD8ED000A96EDFD
:10055800001A07F01DFD029B9BED000A93ED002A8F
:10056800D9ED000A97ED001AD5ED001A07F01EFD27
:100578009BED007ADAED007A2D49DDF80CC0029B7C
:10058800019A77EE677A99ED007AC1ED0A7AD8ED8B
:10059800007A77EE677A97ED007AC1ED0B7AD6ED9F
:1005A800007A77EE677A95ED007AC1ED0C7AD4ED92
:1005B800007A77EE677A93ED007AC1ED0D7ADCF870
:1005C8000030134CCB63D2ED007A1A4A20681368C6
:1005D80077EE677A0B64C1ED0E7A4FF6E07101F0A1
:1005E800A7FE2068144901F051FE07F02CFD02F027
:1005F800CDFF124803F00EF8FFF7D2FE002007F0F7
:10060800E3FC0F4805B0BDE8F04F01F0FAB900BFB0
:10061800A80B0020B43B0020240E00200C0E002064
:10062800200E0020F00D00201C0E0020F40D0020EC
:100638007CC50020FC0D00205F900508809698007E
:10064800C0100020080E0020100E0020180E0020F8
:10065800280E00202C0E002008B5002007F0B4FC5E
:100668000248BDE8084001F0CCB900BFC010002026
:100678002DE9F04F494D4A4E85B000244FF6FF78DA
:10068800284602F04AFD4146224623464548009442
:10069800019401F011FE0427B060224623464FF66C
:1006A800E07141480097019401F006FE234630604E
:1006B800414622463D480097019401F0FDFD3C4922
:1006C800F0603C4A204602F0DFFA3B493B4A0746C5
:1006D800204602F0D9FA3A493A4A8046204602F0C2
:1006E800D3FA3949394A8146204602F0CDFA3849C9
:1006F800384A8246204602F0C7FA3749374A8346C5
:10070800204602F0C1FA36490390364A204602F0E4
:10071800BBFA21468446B268CDF808C02B4620466D
:1007280002F0CAFB214632682B467D2002F0C4FB4A
:100738002321F2682B46B42002F0BEFB37213A464B
:100748002B46FA2002F0B8FB692142462B46FA20D4
:1007580002F0B2FB9B214A462B46FA2002F0ACFB82
:10076800C82152462B46322002F0A6FB5A462B4699
:10077800C8216E2002F0A0FBDDF808C0C82162463F
:100788002B46AA2002F098FB039AF020C8212B469A
:1007980005B0BDE8F04F02F08FBB00BF1C10002071
:1007A800A80B0020739005084A9005087B9005085F
:1007B80083900508C90900088B9005087509000889
:1007C80093900508251000089B9005085D0D00080A
:1007D800A2900508210D0008A990050861060008E7
:1007E800B09005084904000818B9044B93ED000AB5
:1007F8007047034B93ED000A704700BF080E0020B6
:10080800180E002018B9044B93ED000A7047034BEB
:1008180093ED000A704700BF100E0020280E00203C
:1008280018B9044B93ED000A7047034B93ED000A87
:10083800704700BF240E0020200E002018B9044B7A
:1008480093ED000A7047034B93ED000A704700BF11
:100858000C0E0020F00D002018B9044B93ED000A8F
:100868007047034B93ED000A704700BF1C0E002031
:10087800F40D002070B52DED028B9FED108A044613
:100888000E460A25F0EE488A07F02AF878EE808AA4
:1008980007F02CF80A4838EE008A02F0BBFE013D4A
:1008A800F2D1F2EE047AC8EEA78A88EE278AC4ED60
:1008B800008A86ED008ABDEC028B70BD0000000046
:1008C800A086010010B50E4C0E4802F0A3FE04F1FC
:1008D800140104F11000FFF7CDFF4FF6E07004F0AB
:1008E800ABF8FFF771FD5E220023DF206E2104F0D4
:1008F800B3F901232371044B1A68044B1A6010BD25
:10090800A80B0020A0860100143C002020420020F3
:1009180010B5002007F074FB0F4B104C18601048FE
:1009280002F078FE04F11C0104F11800FFF7A2FFA1
:100938004FF6E07004F080F8FFF75AFD5E220023BE
:10094800DF203C2104F088F901236371054B1A6804
:10095800054B1A6010BD00BFFC0D0020A80B00203D
:10096800A0860100143C002020420020104908B550
:1009780001F120002431FFF77DFF4FF6E07004F00D
:100988005BF8FFF721FDB7206E215E22002304F0FB
:1009980063F9084B1A68084B1A60084B02224FF09B
:1009A800804001211A70BDE808400CF0D2BF00BF9A
:1009B800A80B0020043C002020420020E00C00206E
:1009C80008B5002007F010FB114B1860114802F021
:1009D80021FE114901F128002C31FFF74BFF4FF69A
:1009E800E07004F029F8FFF703FDB7203C215E22F0
:1009F800002304F031F9094B1A68094B1A60094BB6
:100A080001214FF080401970BDE808400CF0A1BFEB
:100A18002C0E0020A0860100A80B0020043C00201A
:100A280020420020E00C00202DE9F84380462DEDFF
:100A3800068B10EE100A11EE905A11EE109A10EE75
:100A4800904A0DF0D7FE064648460F460DF0D2FEF6
:100A580041EC100B41EC180B0FF08EFE304653ECB6
:100A6800102B39460DF01AFF0EF0FAF9B0EE480ACD
:100A7800F0EE680A454B186009EE900A0FF07CFF0B
:100A8800304653EC102B39460DF008FF0EF0E8F90C
:100A98003F4B09EE100A186020460DF0ABFE0646E3
:100AA80028460F460DF0A6FE41EC100B41EC1A0B40
:100AB8000FF062FE304653EC102B39460DF0EEFE77
:100AC8000EF0CEF9B0EE4A0AF0EE6A0A314B186021
:100AD80008EE100A0FF050FF304653EC102B394641
:100AE8000DF0DCFE0EF0BCF908EE900A79EE688A8B
:100AF80039EEC88A9FED287A68EEA87A48EE087A17
:100B080028EE078A9FED257A68EE878A88EE278A7D
:100B1800234B1860C8EEA78A68EE897A17EE900A08
:100B28000DF068FE00221F4B0DF006FD68EE297AD5
:100B3800044617EE900A0D460DF05CFE02460B4681
:100B4800204629460DF0F6FC68EEA99A0EF088F9C1
:100B580058EE499AB8F1000F09D1134B83ED008A7A
:100B6800124BC3ED008A124B1860124B08E0124B6F
:100B780083ED008A114BC3ED008A114B1860114BAD
:100B8800C3ED009ABDEC068BBDE8F883140E002077
:100B9800000E0020F80D002000004842000048C266
:100BA800040E002000004940080E0020100E00200E
:100BB800240E00200C0E0020180E0020280E002005
:100BC800200E0020F00D00202DE9F74F044610EE0E
:100BD800109A10EE907A11EE105A11EE906A12EEF9
:100BE800108A002842D14FF6E07003F025FF4846EE
:100BF8000DF000FE824638468B460DF0FBFD52464E
:100C0800CDE900015B464049404812F0EBFA3F4A03
:100C180023460520372104F03DF828460DF0EAFD6B
:100C2800824630468B460DF0E5FD5246CDE900017F
:100C38005B463749354812F0D5FA344A2346052031
:100C4800692104F027F840460DF0D4FD2CA3D3E920
:100C580000230DF023FE02460B462C482D4912F0C6
:100C6800C1FA05209B21294A234641E04FF4FC6044
:100C780003F0E2FE48460DF0BDFD824638468B463D
:100C88000DF0B8FD5246CDE900015B461E491F48EC
:100C980012F0A8FA1D4A00230520502103F0FAFF9C
:100CA80028460DF0A7FD044630460D460DF0A2FD7E
:100CB8002246CDE900012B461549144812F092FA54
:100CC800124A00230520822103F0E4FF40460DF07C
:100CD80091FD0BA3D3E900230DF0E0FD02460B467E
:100CE8000A480C4912F07EFA084A0520B42100236C
:100CF80003B0BDE8F04F03F0CDBF00BFAFF30080F5
:100D0800000000A2941A6D42B7900508D80B002085
:100D1800C8900508D99005080C4A0D4B92ED092A90
:100D280092ED050AD2ED060A92ED071AD2ED081ADD
:100D3800126C012083ED132A83ED140AC3ED150A02
:100D480083ED161AC3ED171A1A663DE77CC5002015
:100D5800A80B00200C4A0D4B92ED042A92ED000AD4
:100D6800D2ED010A92ED021AD2ED031AD26B0020DD
:100D780083ED132A83ED140AC3ED150A83ED161AC1
:100D8800C3ED171A1A661FE77CC50020A80B0020C0
:100D9800F0B52DED088B044683B06B4B002851D17C
:100DA80093ED0B1AD3ED091A93ED0A0AD3ED080A4D
:100DB800FFF73AFE654BD3ED009A654B93ED008A39
:100DC800644BD3ED008A644B684601A993ED00AAF1
:100DD800FFF750FD00980DF00DFD064601980F46EF
:100DE8000DF008FD41EC100B41EC1B0B0FF0C4FC9F
:100DF800304653EC102B39460DF050FD0EF030F80C
:100E0800B0EE4B0AF0EE6B0A09EE100A0FF0B4FDD3
:100E1800304653EC102B39460DF040FD0EF020F80B
:100E280007EE100A68EE077A28EE098A59EE897AE1
:100E380009EE878A204677EEA88A38EE0A8A07F0F4
:100E4800D3F851E093ED071AD3ED051A93ED060A8E
:100E5800D3ED040A0120FFF7E7FD404BD3ED009ADC
:100E68003F4B93ED008A3F4BD3ED008A3E4B6846DB
:100E780001A993ED00AAFFF7FDFC00980DF0BAFC5C
:100E8800044601980D460DF0B5FC41EC100B41EC01
:100E98001B0B0FF071FC204653EC102B29460DF06C
:100EA800FDFC0DF0DDFFB0EE4B0AF0EE6B0A09EE2B
:100EB800100A0FF061FD204653EC102B29460DF067
:100EC800EDFC0DF0CDFF07EE100A68EE077A28EE6C
:100ED800098A59EE897A09EE878A002077EEA88A6E
:100EE80038EE0A8A07F08CF8F1EE487A28EE088A7C
:100EF80008EEA88A064687EE888A18EE100A0DF0D2
:100F080079FC07EE106AF8EEC77A044617EE900AE5
:100F18000D460DF06FFC0AA3D3E900230DF0BEFCCB
:100F280002460B46204629460DF0E2FD0DF098FFDB
:100F380000EE100A03B0BDEC088BF0BDAFF30080E3
:100F48001F85EB51B81E1940A80B0020080E002081
:100F5800100E0020240E00200C0E0020180E002079
:100F6800280E0020200E0020F00D002038B50120AA
:100F7800FFF70EFF1C4C4FF6E07084ED000A03F0FB
:100F88005BFD5E22A021DF20002303F065FE174BE6
:100F980001259D71164B93ED000A164BD3ED000AFF
:100FA800154B93ED001A154BD3ED001A144B002086
:100FB80093ED002AFFF708FE124B93ED000A124B3F
:100FC800D3ED000A114B93ED001A114B2846D3EDCF
:100FD800001A94ED002AFFF7F7FDFFF7E1F90D4B32
:100FE8001A680D4B1A6038BDF40D0020A80B0020BC
:100FF800080E0020100E0020240E00200C0E0020E9
:101008001C0E0020180E0020280E0020200E0020A4
:10101800F00D0020143C00202042002008B50020DC
:10102800FFF7B6FE0E4B4FF6E07083ED000A03F0B3
:1010380003FDB720A0215E22002303F00DFEFFF779
:10104800EBF9084B1A68084B1A60084B03224FF05B
:10105800804001211A70BDE808400CF07ABC00BF3E
:101068001C0E0020043C002020420020E00C002040
:101078002A4B2B48062210B51A704FF6E07400F080
:10108800C0FC0020214607F0B1FA3120214607F0C4
:10109800ADFA6320214607F0A9FA9520214607F00A
:1010A800A5FAC7204FF4FC6107F0A0FA4EF29C7035
:1010B80003F0C2FC0520012100231A4A03F0EAFDCF
:1010C800052020210023184A03F0E4FD05205221C1
:1010D8000023164A03F0DEFD842100230520144A6C
:1010E80003F0D8FD4FF4F06003F0A6FCB621114AD6
:1010F8000023052003F0CEFD4FF6FF7003F09CFCA3
:101108000D4A00238720DC2103F0C4FD0B4B00228D
:101118001A600B4B01221A7010BD00BF3842002024
:10112800F4130020E79005081E910508169105089C
:10113800EB90050838960508ED9005081C3C002042
:10114800FC3B002038B53B4B3B483C4D07221A700E
:101158004FF6E07400F055FC0020214607F046FAEF
:101168003120214607F042FA6320214607F03EFA73
:101178009520214607F03AFA2146C72007F036FAAB
:101188004EF29C7003F058FC0520012100232C4AE4
:1011980003F080FD0520202100232A4A03F07AFD70
:1011A800052052210023284A03F074FD05208421DC
:1011B8000023264A03F06EFD0520B6212A460023A7
:1011C80003F068FD40F213144FF4F06003F034FCB0
:1011D800204601211E4A002303F05CFD2046202101
:1011E8001C4A002303F056FD204652212A460023BC
:1011F80003F050FD20468421174A002303F04AFDDE
:10120800B621164A0023204603F044FD4FF6FF702E
:1012180003F012FC124A00237D20DC2103F03AFD82
:10122800104B00221A60104A012313700F4A1370E2
:1012380038BD00BF38420020F4130020219505086E
:10124800F2900508F6900508FA900508FD90050843
:101258000691050802910508019105080591050800
:101268000A9105081C3C0020FC3B0020A4430020F8
:1012780038B52D4B2D4805241C704FF6E07500F04D
:10128800C0FB0020294607F0B1F92720294607F0BE
:10129800ADF94F20294607F0A9F97720294607F02C
:1012A800A5F99F20294607F0A1F9C720294607F08C
:1012B8009DF94EF29C7003F0BFFB012100232046EC
:1012C8001B4A03F0E7FC162100232046194A03F0C5
:1012D800E1FC3E2100232046174A03F0DBFC66218F
:1012E80000232046154A03F0D5FC8E210023204612
:1012F800134A03F0CFFCB621124A0023204603F01C
:10130800C9FC4FF6FF7003F097FB0F4A00237D20BE
:10131800DC2103F0BFFC0D4B00221A600C4A0123AC
:1013280013700C4A137038BD38420020F4130020A3
:101338002195050815910508199105081D910508BD
:101348002191050825910508299105081C3C0020D4
:10135800FC3B0020A44300203B4B3C48042270B5D2
:101368001A704FF6E07400F04CFB0020214607F09D
:101378003DF93120214607F039F96320214607F06D
:1013880035F99520214607F031F9314E314D214686
:10139800C72007F02BF94EF29C7003F04DFB052097
:1013A80001210023324603F075FC0520202100238B
:1013B800294A03F06FFC052052210023274A03F035
:1013C80069FC052084210023254A03F063FC0520DD
:1013D800B6212A46002303F05DFC40F213144FF4B3
:1013E800F06003F029FB204601213246002303F078
:1013F80051FC204620211B4A002303F04BFC2046C9
:1014080052212A46002303F045FC20468421164A2F
:10141800002303F03FFCB621144A0023204603F0C2
:1014280039FC4FF6FF7003F007FB114A00237D20BB
:10143800DC2103F02FFC0F4B00221A600E4A012317
:1014480013700E4A137070BD38420020F413002048
:101458004A91050821950508359105084591050823
:101468003A9105083F9105084491050849910508F6
:101478004D9105081C3C0020FC3B0020A4430020A3
:10148800F8B5334B3348344F344E03221A704FF6B5
:10149800E07400F0B6FA0020214607F0A7F86320B0
:1014A800214607F0A3F8B3204FF4F06107F09EF847
:1014B8002146C72007F09AF84FF6FF7003F0BCFAF0
:1014C8004EF29C75DC2100237D20254A03F0E2FBC7
:1014D800284603F0B1FA0520012100233A4603F01B
:1014E800D9FB0520522100231E4A03F0D3FBB62165
:1014F80000230520324603F0CDFB40F213144FF4CD
:10150800F06003F099FA012120463A46002303F0DF
:10151800C1FB522120460023324603F0BBFBB62113
:10152800114A0023204603F0B5FB284603F084FA4D
:101538000E4A00230520A22103F0ACFB0C4B00222D
:101548001A600C4A012313700B4A1370F8BD00BFD0
:1015580038420020F41300206791050821950508FA
:1015680058910508629105086691050826910508B5
:101578001C3C0020FC3B0020A443002008B5074B7E
:10158800074802221A7000F03CFA06F029FF054BC2
:1015980000221A60044B01221A7008BD384200204C
:1015A800F41300201C3C0020FC3B0020002008B560
:1015B80003F06EFA064B00221A70064B1B78022BBA
:1015C8000CBF05480548BDE8084000F01ABA00BF3E
:1015D80038420020B43B0020780F0020300E002055
:1015E8002DE9F14F2D4C204601F097FD00202C49A4
:1015F8002C4A01F049FB2C492C4A8146002001F075
:1016080043FB2B492B4A0746002001F03DFB2A49A2
:101618002A4A0646002001F037FB2949294A05468F
:10162800002001F031FB2849284A8046002001F0BB
:101638002BFB2749274A8246002001F025FBD221AF
:1016480083464A462346E62001F036FC28203A46DF
:101658002346014601F030FC462132462346282025
:1016680001F02AFC64212A462346282001F024FCA4
:10167800822142462346282001F01EFC524623467A
:101688002820A02101F018FC28205A46BE21234614
:1016980001B0BDE8F04F01F00FBC00BF641100209D
:1016A80002900508B51500086B9105088515000816
:1016B80058910508891400084D9105086113000820
:1016C8007691050879120008819105084D110008E6
:1016D800ED90050879100008034B01224FF4FC60D7
:1016E8001A7003F0A9B900BFD80C00200B4B10B535
:1016F800002420461C7003F0CBF906F009FC06F024
:1017080085F9074B1C70074B01221A7006F0CCFFB5
:101718000548BDE8104000F074B900BFD80C00209F
:1017280038420020B43B0020300E00200A4B10B590
:10173800002420461C7003F0ABF906F0E9FB074BC8
:101748001C70074B02221A7006F0AEFF0548BDE870
:10175800104000F056B900BFD80C002038420020D5
:10176800B43B0020780F002008B5064B0020187005
:1017780003F08EF9044B054803221A70BDE80840AF
:1017880000F03FB9D80C0020B43B00201C1000200A
:101798000C4B10B500220C4C1A7006F0B9FB04F083
:1017A80003F906F056FC06F07FFF20684FF6E0715B
:1017B80000F0BEFD2068054900F068FDBDE8104056
:1017C80001F0E4BED80C00200C0C00208B91050819
:1017D8000E4B002210B51A700088C83880B2042851
:1017E80005D90B480B4A0C4B872102F0F7F80B4C34
:1017F800C0B204F063F920684FF6E07100F098FD7C
:1018080020680749BDE8104000F040BDD80C002012
:101818009F910508B4D00308BF9105080C0C00205F
:10182800F09105082DE9F04F5848594D87B000242C
:1018380001F073FC4FF6FF71224623465548009489
:10184800019400F039FD042607464FF6E071224660
:10185800234651480096019400F02EFD4FF6E071A2
:101868008046224623464D480096019400F024FD08
:101878004FF6FF7181462246234649480096019457
:1018880000F01AFD234628604FF6FF7122464548AE
:101898000096019400F010FD43496860434A2046D1
:1018A80001F0F2F94249434A8246204601F0ECF938
:1018B8004149424A8346204601F0E6F940490390EF
:1018C800404A204601F0E0F93F4904903F4A20464B
:1018D80001F0DAF93A46059021462C4B204601F0F2
:1018E800EBFA21464246294BC82001F0E5FA0A21C5
:1018F8004A46264BC82001F0DFFA2A68234B6421A8
:10190800782001F0D9FA78206A68204B014601F066
:10191800D3FAC82505262827E0B203F0FFFF2C4A92
:101928000146284601F0B0F994FBF6F106FB114197
:1019380079431E31024689B20020144B0134013527
:1019480001F0BAFA042CADB2E6D1D22152460520F4
:101958000E4B01F0B1FAD2215A464C200B4B01F044
:10196800ABFAD221039A094B9C2001F0A5FAD221A7
:10197800049A064BEC2001F09FFA059A034BEC20E1
:10198800B42107B0BDE8F04F01F096BAC0100020AE
:101998000C0C0020009205080A9205081792050809
:1019A800229205080C900508369205089917000838
:1019B8003E92050871170008479205083517000878
:1019C80050920508F516000859920508E116000816
:1019D800D917000808B500F03FFAFEF70FFCFEF72C
:1019E80047FEFEF771FCFFF7FBFDFFF71BFFFEF755
:1019F800BFFC00F0D7FA00F0D9F8BDE8084000F0C5
:101A0800A1B910B5044628B90F48104A104B452112
:101A180001F0E4FF0F4B1868844213D010B1C3697A
:101A280000219847002003F033F8002003F01AF84B
:101A38004FF6FF7003F000F8E3692046012198474C
:101A4800044B1C6010BD00BF62920508C3D0030898
:101A58007E920508140C00200048D2E7C010002030
:101A68004FF6FF7070474FF6FF70704713B50029A7
:101A780044D04FF2DE7003F00BF8002003F0D2F8E8
:101A88000F2002F0D9FF1E4C1E4A412101230A20D3
:101A980003F000F9042003F0C5F8236828209621F4
:101AA800042B21DC0123184A03F0F4F801A90DF1F5
:101AB8000602206803F074FB0F2002F0BDFFBDF89A
:101AC8000400BDF8061014382822002380B202F062
:101AD800E3FFBDF80610BDF80400143989B22822C6
:101AE800012302F0D9FF09E0084A012303F0D2F8E4
:101AF8001E20A521064A012303F0CCF81CBD00BF17
:101B0800180C00208E920508A1920508BD920508C0
:101B1800D392050837B51E4C2368042B05462BDCE9
:101B280001A80DF1060103F039FBBDF80630BDF838
:101B380004201849042009F011FF2368002B04DA57
:101B48001548164A164B592105E0042B05DD1248A5
:101B5800124A144B5A2101F041FF04EB8302BDF8ED
:101B6800041001339180BDF806102360052BD18045
:101B780008D1201D03F094FB00230B482360FFF7D6
:101B880040FF03E028460121FFF770FF3EBD00BF7C
:101B9800180C0020EA9205082F930508D5D00308F1
:101BA80051930508689305080812002037B50B4CB7
:101BB800204601F0B2FA0A4B0A4900930025012099
:101BC800094A0A4B019501F050F929460246234675
:101BD800284603B0BDE8304001F06EB9D40E0020AD
:101BE800751A0008691A00086F1A00081D1B0008FA
:101BF8004FF6FF7070474FF6FF7070471FB54FF6EE
:101C0800E07002F045FF002003F00CF80F2002F00E
:101C180013FF0021294A2A4C01230A2003F03AF82D
:101C2800002002F009FF042002F0FCFF0A2019211D
:101C3800244A012303F02EF82521234A01230A20F0
:101C480003F028F81F2002F0F7FE01230A203721AD
:101C58001E4A03F01FF8237873B301231E20962130
:101C68001B4A03F017F862881A49684611F0BAFA55
:101C780001231E20A2216A4603F00CF8A288164907
:101C8800684611F0AFFAAE216A4601231E2003F020
:101C980001F80F2002F0D0FE6088A188143880B2C5
:101CA8002822002302F0F8FEA1886088143989B23E
:101CB8002822012302F0F0FE1FBD00BF96930508FD
:101CC800300C0020A8930508C8930508E893050878
:101CD8000B9405081D9405082A94050801B18DE7A1
:101CE800704713B50DF1060101A803F00BFA144B68
:101CF80001221A705988BDF80420891A0E311C294E
:101D080019460AD89C88BDF80600201A0E301C28EF
:101D180003D899680131996001E000238B60084B72
:101D28009968012905DD00229A601A70FFF794FE70
:101D380005E05A80BDF806209A80FFF75FFF1CBDBA
:101D4800300C002037B50B4C204601F0E6F90A4B61
:101D58000A49009300250120094A0A4B019501F020
:101D680084F8294602462346284603B0BDE8304099
:101D780001F0A2B808120020E51C0008F91B0008B1
:101D8800FF1B0008EB1C000808B5154B00221A6061
:101D9800144B1A68144B1A6007F0EAFC134B1B78B3
:101DA800023B052B15D8DFE803F00306090F120CD8
:101DB800FFF7E4FB0DE0FFF763FB0AE0FFF7CCFA5F
:101DC80007E0FFF7BFF904E0FFF752FA01E0FFF779
:101DD8004FF907F0C5FC064B01221A7008BD00BF79
:101DE8001C3C0020143C00202042002038420020E7
:101DF800A443002038B50F4B0F4D00241C700F4B27
:101E08001C700F4B4FF0FF321A600E4B1A680E4BC6
:101E180020461A6002F03CFE0C4B1B78022B0CBFCC
:101E28000B480C48FFF7EDFD2C70BDE8384007F073
:101E380097BC00BF38420020A4430020FC3B002090
:101E48001C3C0020143C002020420020B43B002011
:101E5800780F0020300E002070B5124C204601F09B
:101E68005CF900200146224600F086FA00200E495F
:101E78000E4A00F009FF0E490E4A0646002000F0FF
:101E880003FFD2210546324623464FF4827001F003
:101E980013F8DC20D2212A462346BDE8704001F021
:101EA8000BB800BFF4130020A9900508FD1D000819
:101EB80037940508911D000810B5064C4FF6FF71C0
:101EC800206800F035FA044B20681968BDE8104016
:101ED80000F0DCB93C0C00209801002008B5002077
:101EE80002F0D6FD054B1868054B196800F0CEF9CD
:101EF8000448BDE80840FFF784BD00BF3C0C002043
:101F080094010020C010002008B5FFF7D5FF00207D
:101F1800014605F0F1FEBDE8084001F037BB008836
:101F2800A0F5C87080B2092808B505D90748084A3D
:101F3800084B8F2101F052FD074B1880074BFF21FA
:101F4800197005F0D9FEBDE80840B5E73B940508CF
:101F5800E7D003085E940508981400209A1400201E
:101F68000088A0F5967080B2092808B505D90848F8
:101F7800084A094B832101F031FD084B1880084BB2
:101F88000121197005F0B8FEBDE8084094E700BFCC
:101F98003B940508FCD003085E94050898140020BB
:101FA8009A1400202DE9F34100243A483A4D01F0F3
:101FB800B4F8224623464FF6FF713848009401943E
:101FC80000F07AF904262246234607464FF6FF71A9
:101FD80033480096019400F06FF9234628602246A2
:101FE8004FF6FF712E480096019400F065F92D49CF
:101FF80068602D4A204600F047FE2C492C4A0646C8
:10200800204600F041FE214680463A462046214BB4
:1020180000F052FF2A681F4B2046282100F04CFF91
:102028003246D2211B4B5A2000F046FFAA20D2216B
:102038004246184B00F040FF0F254FF4967440F2CB
:10204800351620461B491C4A00F01EFE0134024684
:10205800782128460F4BA4B2233500F02DFFB44257
:10206800ADB2EED10F254FF4C87440F29916204650
:102078001249134A00F008FE013402469B21284603
:10208800044BA4B2233500F017FFB442ADB2EED131
:10209800BDE8FC81501300203C0C00208F940508FB
:1020A8001D9005089B940508111F0008A4940508B5
:1020B800E51E0008AD940508691F0008AF940508DF
:1020C800271F000808B508B143682BB90348044A1C
:1020D800044B9B2101F082FC586908BDB1940508A6
:1020E80010D10308D394050808B5FFF7EBFF806803
:1020F800123080B208BD08B5FFF7E4FF406806302B
:1021080080B208BD2DE9F84F04468846FFF7DAFF8C
:102118006689E589074606F1030905F10F0AB8F152
:10212800000F1FD01F2002F087FC2046FFF7DCFFBE
:1021380083462046FFF7DFFF294603465FFA8BF206
:10214800F0B202F0ADFC042002F06CFD0B364FF645
:10215800FF70033502F070FCB0B2A9B23A680123EF
:1021680002F098FD3D69204641464A465346A84735
:10217800BDE8F88F13B504460DF1060101A802F079
:10218800C1FF2046FFF79EFF6389BDF80410BDF824
:102198000620C91AE389D21A0339C3680F3A2046C0
:1021A80098471CBDF7B5044614200D4616461F4631
:1021B80010F0A6FC089BC7600361064B0649074A56
:1021C80080E8700000930190054B002000F04DFE60
:1021D800FEBD00BF0D210008FF200008F120000807
:1021E8007D210008704708B508B143682BB9044839
:1021F800044A054BAD2101F0F1FB586908BD00BF49
:10220800F294050828D10308D3940508F8B50546C3
:102218000E46FFF7E8FF836B04461BB1284631469C
:10222800984700E018466F8994F83C30ED890EB95C
:10223800034310D0208E02F0FFFB608E02F012FCE8
:1022480094F8350002F0EEFC94F83430384629460C
:10225800224602F01FFD002384F83C30F8BD08B583
:10226800FFF7C1FF90F83500BDE8084002F0EFBC69
:1022780038B5FFF7B8FF044611F03AF8054694F868
:10228800350002F0DFFC684380B238BD38B50D4632
:10229800FFF7A9FF29462E22044611F059F850B13C
:1022A800204629462E2211F0A5F8002384F82E3066
:1022B800012384F83C3038BD2DE9F7430746402018
:1022C8000E461546984610F01BFC044628B91148DE
:1022D800114A124B4E2101F081FB114B114A124950
:1022E8008DE818000020114B00F0BFFD39468146EB
:1022F800FFF7CCFF9DF82830268684F835300B9BF5
:102308006586A363002384F8348084F83C3048460B
:10231800BDE8FE83F294050840D10308109505082E
:10232800152200086722000879220008ED2100081C
:1023380010B50C46FFF757FF0123048680F83C30A0
:1023480010BD00BF4FF4A0707047C8207047704799
:10235800074B1B78022B07B508D1064B1B78022BBD
:1023680004D001A80DF1060102F0CCFE0EBD00BF9D
:10237800A44300203842002073B50A4B06460D4698
:102388001446009300200849084A094B019000F0C0
:102398006CFD294602462346304602B0BDE870402F
:1023A80000F08ABD572300084D2300085323000876
:1023B8005923000813B502AB03E90600436843B18B
:1023C800027C0124082A9C7004D11B692146984785
:1023D80000E01C4620461CBD30B500282BD0058BDC
:1023E800002425E0036A1A7C012A05D15B681A8853
:1023F8008A421BD1187F30BD052A06D15B681A882E
:102408008A4213D193F82C0030BD032A06D15B68A9
:102418001A888A420AD193F8250030BD062A05D1C8
:102428005B681A888A4201D1D87A30BD01340430F9
:10243800AC42D7D3002030BD08B181750120704768
:10244800F8B504460D46D0B1E175D0F898309847F4
:10245800012D0DD12746002606E0F86900F1080293
:10246800436906CA98470136238B04379E42F4D342
:10247800D4F898302046294698470120F8BDF8BD81
:10248800F8B50546084617460E4610F031FF013FDD
:10249800B84234BF04463C463CB128463146224641
:1024A80010F0A8FF00232B55F8BD2C70F8BDF7B528
:1024B800044600200090019000296CD00E8B68E043
:1024C80000F1080351F823301D7C042D04D15D6808
:1024D8002D88954247D0013000F1080351F8233088
:1024E8001D7C012D04D15D682D8895423BD00130BB
:1024F80000F1080351F823301D7C052D04D15D68D7
:102508002D8895422FD0013000F1080351F823306F
:102518001D7C032D04D15D682D88954223D00130A0
:1025280000F1080351F823301D7C022D04D15D68A9
:102538002D88954217D0013000F1080351F8233057
:102548001D7C072D04D15D682D8A95420BD0013082
:1025580000F1080351F823301D7C062D08D15D6871
:102568002D88954203D103F10801204615E001307A
:1025780000F1080351F823502B7C082B09D16F6810
:102588003F88974204D105F1080120461A4605E024
:102598000130B04294D320466946082210F060FD0D
:1025A8002046FEBDF8B505460F461646002830D031
:1025B8004388032B2FD0202010F0A2FA04460028CD
:1025C8002BD040F80C5B39460C22FFF759FF182036
:1025D800E66110F095FA0646B8B1022303740123A8
:1025E80063760F4B446063600E4BA3600023237631
:1025F8006B8805EB830201339BB2012B50606B8023
:102608000CD16A685268137608E0204610F080FA08
:1026180004E0064602E0002600E006463046F8BD23
:102628008C5004082A4D040837B5456802AB03E905
:1026380006003DB3037C0124042B85F8314022D1E8
:10264800688E02F0F9F995F8300002F0EBFA95F887
:10265800343043B9BDF80200BDF80610AA1C234661
:1026680002F018FB0FE0012B03D1084840F2395162
:1026780004E0022B07D1054840F24151044A054BBA
:1026880001F0ACF92C4620463EBD00BF2395050855
:10269800001C040821950508F8B504460F4616469F
:1026A80010B3838A0A2B20D0202010F029FA05467F
:1026B800E8B14460102200F108003946FFF7E0FE57
:1026C8004FF6FF73A08A2B801F236B8000232B7685
:1026D800831D013080B20128EE6144F82350A082A6
:1026E80007D1A3691876F8BDF8BD0020F8BD012010
:1026F800F8BD0120F8BD2DE9F0411D464B1C98425C
:1027080080460C4617460CDD95420ADC013208F17A
:1027180001035B1A521BC8B2D2B29BB2294602F01F
:10272800BDF9A8F10208BDF81800C4EB080802F0CA
:1027380083F901261FFA88F808E0A919601C80B2FD
:1027480089B24246002302F0A7F901367B1B9E425C
:10275800F3D3BDE8F081F8B5C7B2144638461E4633
:102768000D4602F09FF9621E92B23846294602F0E1
:1027780099F9304602F060F9022606E0A21B92B2EF
:102788003846294602F08EF90136A642F6D3F8BD3E
:1027980070B5044600F11E003C22002380B20D46AD
:1027A80002F07AF91E3DA9B220463C220123BDE879
:1027B800704002F071B970B5044601380322002355
:1027C80080B20D4602F068F9013DA9B22046032205
:1027D8000123BDE8704002F05FB9F7B5089D2E7B74
:1027E800EF7A1C463604AB7A06EB0726F618431A2E
:1027F800687B06EB00602D1800200190121B08462C
:102808002146009501F098FEFEBD30B5456885B0BB
:1028180004AB03E906007DB101242C736D68BDF893
:102828000800BDF80A109DF80C209DF80E300095A0
:10283800FFF7D3FF204600E0284605B030BD2DE95C
:10284800F04385B004AB03E906004468BDF80860AE
:10285800BDF80C70002C41D0012384F8263094F880
:1028680025300BB9A26800E06268FFB2BDF80A1013
:102878009DF80E30009230463A46FFF7AEFF04F15D
:102888000C08022002F0CEF9404610F031FD054652
:1028980000B1451E0F3F0024153E1FFA87F90DE0D1
:1028A80002F0CAF902F0CEF904FB106189B2484679
:1028B8002022002302F008FA0134E4B2AC42EFD33C
:1028C800002002F0B9F8B8B2B1B24246012302F0D2
:1028D800FBF9002002F0A6F9012000E0204605B02F
:1028E800BDE8F0832DE9F04385B004AB03E90600A9
:1028F8004568BDF80860BDF80C70002D3CD0012378
:102908006B762B7EBDF80A10012B0CBF6A68AA688B
:102918009DF80E300092FFB23A463046FFF75DFF51
:102928000C35022002F07EF9284610F0E1FC0E3F3B
:1029380081460024163E1FFA87F80DE002F07CF964
:1029480002F080F904FB106189B24046202200237E
:1029580002F0BAF90134E4B24C45EFD9002002F094
:102968006BF8B8B2B1B22A46012302F0ADF90020E3
:1029780002F058F9012000E0284605B0BDE8F083D0
:102988002DE9F04F85B00546DDF8409002914846A4
:102998009046039310F0ACFCDDF838A0DDF83CB0AD
:1029A8000646294600242F4611E024B1B4420CBF44
:1029B8005B46534600E0039B01F10805ADB2009366
:1029C8002846029A4346FFF708FF01342946B442D5
:1029D800EBDD002002F030F8022002F023F97D1D23
:1029E80008F10508A8B21FFA88F14A46012305B084
:1029F800BDE8F04F02F04EB970B5406886B006AB3E
:102A080003E9060000282ED0012380F82D308668BF
:102A1800164BF21A534243EB020390F82C205AB19A
:102A2800002B134D134B144A08BF1D46134B00F1DE
:102A38001C0418BF13460AE0002B0D4D0D4B0E4A1F
:102A480018BF1D460D4B00F10C0408BF1346BDF816
:102A58001200BDF81410BDF81620009601950294D6
:102A6800FFF78EFF012006B070BD00BF7025040877
:102A7800AC210408522704088E23040834290408CA
:102A880070B5446886B006AB03E9060004B30123B9
:102A98006377A668104B227FF11A4B4243EB010380
:102AA8000AB10BB904E01BB966680C4D0C4B01E088
:102AB8000C4D0D4BBDF81200BDF81410BDF81620D2
:102AC80000960C3401950294FFF75AFF012000E0AC
:102AD800204606B070BD00BFBC300408F82C0408BE
:102AE800DA2E040892320408683404082DE9F04309
:102AF80085B004AB03E906004468BDF80860BDF87A
:102B08000A90BDF80C50BDF80E80002C00F08C80A7
:102B18000123A3740220676802F084F84FF6FF705F
:102B280001F0A0FF002001F087FFEDB25FFA88F8FE
:102B3800A6F1160189B230462A4643460097FFF7A8
:102B48004CFE277A002F2ED1A28A234600E00137B7
:102B5800974204D29969097E04330029F7D002F01C
:102B68006BF802F06FF8A9F116091FFA89F90E211E
:102B780001FB10914FF6FF7208F101085FFA88F324
:102B880089B2009248462A46FFF7B5FD022002F0B6
:102B980049F81F2001F050FFA38A002B38D0103DC0
:102BA800E8B2303E2CE0E3685C68A28A2346013A2A
:102BB800002700E00137974204D29969097E04335F
:102BC8000029F7D002F038F802F03CF80E2101FB9A
:102BD80010914FF6FF7208F101085FFA88F389B285
:102BE800009248462A46FFF786FD022002F01AF8AE
:102BF8001F2001F021FFA38A53B1103DE8B21A3E0D
:102C08000637B1B254F827200123083202F05CF8E5
:102C1800002002F007F84FF6FF7001F023FF1F2095
:102C280001F00AFF012000E0204605B0BDE8F0836E
:102C38002DE9F04105463620884614461F460FF018
:102C48005FFF0646E0B120F8025B41462E22FFF7FF
:102C580017FCBDF8183086F8344073861820012315
:102C680086F8307086F831300FF04AFF044618B104
:102C780004234660037404E030460FF049FF00E087
:102C880004462046BDE8F081F8B5064624200F46E4
:102C980015460FF035FF0446D8B10F4B0680836008
:102CA8000E4B39464360102200F10C00FFF7E8FB99
:102CB8000126002318202562237766770FF020FF6E
:102CC800054610B14460067404E020460FF020FF6A
:102CD80000E005462846F8BDBC300408162B040859
:102CE800F8B506462C200F4615460FF009FF044696
:102CF800E8B120F80C6B39461922FFF7C1FB0D4BE0
:102D0800A562A3600C4B6360002384F8253018206B
:102D1800012384F826300FF0F3FE054618B103238B
:102D28004460037404E020460FF0F2FE00E005461C
:102D38002846F8BDC84904086646040810B5044684
:102D480014200FF0DDFE20B100234380014B0480E6
:102D5800036110BDAD25000838B5054644200FF0C5
:102D6800CFFE0446C0B10E4B058243600D4B036095
:102D7800012383740023037283820B4B036418209E
:102D88000FF0BEFE054618B107234460037404E043
:102D980020460FF0BDFE00E00546284638BD00BFBE
:102DA8005C420408523E0408A12600082DE9F041BF
:102DB80005463420884614461F460FF0A1FE0646F5
:102DC80020B3144B05808360134B414643601022A7
:102DD80000F10C00FFF754FB214606F11C001022FD
:102DE800FFF74EFB002386F82C30182001233763A9
:102DF80086F82D300FF084FE044618B1052346608E
:102E0800037404E030460FF083FE00E004462046D9
:102E1800BDE8F08170250408CA1F04082DE9F041B7
:102E2800044614200D46164698460FF069FE0746DC
:102E3800B8B1069B048003610023C3720123456077
:102E4800068180F80A80037318200FF059FE0446A3
:102E580018B106234760037404E038460FF058FEA3
:102E680000E004462046BDE8F0812DE9F041044623
:102E780018200D46164698460FF042FE0746B8B190
:102E880001238370069B04800361079B456086606D
:102E9800C0F80C80436118200FF032FE044618B1C8
:102EA80008234760037404E038460FF031FE00E061
:102EB80004462046BDE8F0812DE9F34198461B8B76
:102EC8001D2B05460C4617464FF0000000F2B48053
:102ED800B5F5A07F0090019000F2AE80F02900F2D5
:102EE800AB80127CADF80610511EADF802500729D0
:102EF80000F28A80DFE801F045595E04456A1476DD
:102F08007B684E4A7A611A8893F834303A80013BDC
:102F1800DBB2012B7FD8ADF80240ADF806507AE05D
:102F280005F11602ADF8002004F11602ADF80420F0
:102F380002AE434A16E903007A6107F1080282E803
:102F4800030003F10802013348F82270A8F818308A
:102F58007B681A8A187A3A8000286CD1FFF7FCFE41
:102F68003849436859603849DF600126163D1960C1
:102F780002461E72A8B2E1B24346FFF79DFF3046F3
:102F88005AE0012A0CBF314B314B78687B6130F82D
:102F98000C3B3B8010F0ACF9431CDB001A34ED18F5
:102FA800ADF80440ADF8005035E07B68294A1B684D
:102FB8007A6102E0284A7B687A611B8814353B8075
:102FC800ADF800501434ADF8044024E07B68234A7F
:102FD8007A611A883A801A899B7AAD18ADF8005040
:102FE800E418F0E77E681E4B7B61338838463B80E7
:102FF80073689847013D4519ADF80050B3683846E5
:103008009847013C0419DEE71648174A174B40F267
:103018001A3100F0E3FC02AA12E9030007F10803E1
:1030280083E80300B8F8183003F10802013348F8C0
:103038002270A8F818300120BDE8FC81312600086C
:10304800F52A0008483A04083E360408892A000888
:10305800012A0008ED28000847280008132800085E
:10306800BD23000823950508101C040821950508B0
:10307800F8B51646002834D01378002B2ED0028BD2
:10308800002327E0046A257C042D21D165682F8858
:103098008F421DD195F8313053B16F8E01F0F2FC9B
:1030A80004F1080268866369204606CA98476F8655
:1030B800A81C31462E22FFF7E3F995F831307BB191
:1030C80004F108026369204606CA98470120F8BD42
:1030D800013304309342D5D30020F8BD1846F8BD1B
:1030E8000120F8BD70B5B8B1068B0446002310E086
:1030F800256A287C04280AD16D682888884206D168
:103108001046A91C2E22FFF7BBF9012070BD013320
:103118000434B342ECD3002070BD38B5044620B364
:10312800134BC361134BC0F89830134BC0F89C3055
:10313800124B00257822C0F8A0308575C575058327
:10314800294600F120000FF0CDFFD4F89830204632
:10315800294698470A4A1388312B07D8094941F864
:10316800234001331380012038BD38BD284638BDBF
:103178004924000841240008E1230008B724000876
:10318800440C00209C1400202DE9F041044600283E
:1031980000F0B380078B02460025A8E0136A1E7C66
:1031A800042E00F08780012E23D1586803888B42B3
:1031B80040F09B8005F108070FF0AAFC54F827009F
:1031C8004FF00008C0F804800FF0A2FC228B531EB9
:1031D8009D4208D00732238354F8221044F8271060
:1031E80044F8228002E044F8278025833046BDE871
:1031F800F081052E5ED0032E5CD0022E13D15B68C1
:10320800186803888B4270D14388013B9BB2438086
:103218000BB90FF07DFC05F1080654F82630586804
:103228000FF076FC4EE0072E21D15E68338A8B4280
:103238005BD1002706E0BB1D013756F823000FF0CD
:1032480067FCFFB2B38ABB42F5D80027B78205F105
:10325800080654F8263058680FF05AFC54F826002F
:1032680033E044F8267025830120BDE8F081062E5E
:103278001ED1586803888B4237D105F108060FF034
:1032880047FC54F82600002747600FF041FC228BCA
:10329800531E9D4209D00833013A54F82310228363
:1032A80044F8261044F82370DEE744F826701AE044
:1032B800082E1AD1586803888B4216D10FF028FCC3
:1032C80005F1080654F82600002747600FF020FC97
:1032D800228B531E9D42C4D0073254F8221044F862
:1032E800261044F822702383BEE701350432BD421C
:1032F800FFF454AF0020BDE8F081BDE8F08170B55F
:10330800044600282AD0068B751E083600EB860670
:103318001EE056F8043D1A7C042A13D0012A11D065
:10332800052A0FD0032A0DD0022A02D15B681B6838
:1033380009E0072A02D15B68198A05E0062A01D04C
:10334800082A04D15B6819882046FFF71DFF013D54
:10335800681CDED100232383012070BD70BDF0B549
:1033680028B30023068B1A461EE0046A257C072D25
:1033780018D16468258A8D4214D1A78A002504EBE8
:1033880083040DE004EB050C0435DCF818C09CF848
:1033980018C0BCF1010F03F1010301D1D8B2F0BD8F
:1033A800BB42EFD301320430B242DED30020F0BD7D
:1033B80070B508B3048B00231BE0026A157C072D47
:1033C80015D15268158A8D4211D10023958A11466C
:1033D8001C46012007E013B99669307601E08E6932
:1033E800347601330431AB42F5D3012070BD01338B
:1033F8000430A342E1D3002070BD2DE9F04128B389
:103408000023078B1A461EE0046A257C072D18D175
:103418006468258A8D4214D1B4F814C0002504EBE1
:1034280083040CE066190435B66996F81880B8F17B
:10343800010F03D106F10800BDE8F08101336345AF
:10344800F0D301320430BA42DED30020BDE8F08167
:103458002DE9F04700282FD00023B0F818C01D46EA
:1034680027E0046A267C072E21D16468268A8E42CA
:103478001DD1B4F81480002604EB830915E009EB8C
:103488000604A7693C7E012C0DD192F800A0BAF180
:10349800000F08D007F1080011461022FEF7F0FFD0
:1034A8002046BDE8F087013304364345E7D30135AC
:1034B80004306545D5D30020BDE8F087F0B5B0B13C
:1034C800068B002510E0046A277C062F0AD1646861
:1034D80027888F4206D123819DF814306260A37239
:1034E8000120F0BD01350430B542ECD30020F0BD19
:1034F80010B500210446FEF7A3FF20460121BDE8D0
:103508001040FEF79DBF38B598B1048B02460023E2
:103518000CE0106A058804328D4206D100F10802D9
:10352800436906CA9847012038BD0133A342F0D346
:10353800002038BD10B50C460021FEF781FF20465B
:103548000121BDE81040FEF77BBF13B502AC04E9CA
:103558000C00BDF80230834206D8BDF80030834223
:1035680034BF0020012000E00020BDF806308B4267
:1035780006D8BDF804308B4234BF0021012100E099
:103588000021002818BF0846C0B21CBD38B5114B31
:10359800114A1988002319E052F8045FA87D012810
:1035A80012D100240CE004F1080355F82300037C31
:1035B800082B03D1436800211B6998470134A4B242
:1035C8002B8BA342EFD838BD01339BB28B42E3D19A
:1035D80038BD00BF440C002098140020704770B517
:1035E800094CA5787DB9094B1E78012E0BD163686B
:1035F800013363606268064B9A4204D9284601F099
:10360800D3FAA670656070BD440C0020300000201D
:1036180040420F00054A9060134602E0996801395C
:10362800996091680029F9D1704700BF440C0020C7
:10363800F0B585B001F064FD002800F0498100254F
:1036480002A80DF10A01ADF80850ADF80A5001F0D2
:1036580059FD03A80DF10E01ADF80C50ADF80E5050
:1036680001F09CFDBDF80C10BDF808200091BDF8D4
:103678000E10BDF80A3001912C46964D9649082047
:1036880008F06CF9A878012803D101F08DFAAC7024
:1036980019E1924B5B78012B40F01581AB78002B38
:1036A80040F011816B6029888D4A09E152F8046F56
:1036B800B07D012840F002810025FAE005F10803F9
:1036C800BDF8080056F82340BDF80A1004F10803B5
:1036D8000CCBFFF73AFF002800F0E980237C013B80
:1036E800062B00F29F80DFE803F00429159D1F9D3B
:1036F8004C006668012304F10805337795E8060055
:10370800636920469847002333772046636995E824
:10371800060086E0636893F8252012F1FF3218BF8F
:10372800012283F8252077E0636893F82C2012F1B2
:10373800FF3218BF012283F82C206DE06268137EE7
:103748001568002B6ED16E882F462946184606E06C
:1037580051F804EFDEF804E001338EF81800B342A4
:10376800F6D301231376002607E057F8040F00F17B
:103778000802436906CA984701366B889E42F4D30B
:1037880050E0656820892E68A37B227B0096A0F113
:10379800160189B2FFF721F81420FFF73BFF2B7AB7
:1037A800C3B9AF8A29461A461E4609E0886990F8C7
:1037B80018E00676BEF1010F08BF13460431013246
:1037C800BA42F3D301220BB9AB6924E0053355F8AB
:1037D800233020E06368DB685A680023908A154626
:1037E80019461F4609E0AE6996F818E03776BEF12B
:1037F800010F08BF0B46043501318142F3D3411E46
:103808008B4203D1053052F8203003E004D207334D
:1038180052F8233001221A7604F1080206CA6369B5
:1038280020469847237C013B072B4CD8DFE803F060
:103838000410074B0A0D123A63681B6A34E0636888
:103848009B6A2DE063681B6B2AE063681B6927E0AD
:10385800636824E063681A7A7AB9988A1946013845
:1038680000E00132824204D28C69247E0431002CAB
:10387800F7D0063253F8223011E0DB685A68908A94
:1038880011460138002300E00133834204D28C69D9
:10389800247E0431002CF7D0063352F82330DB693C
:1038A800984710E06368DB68204698470BE00135CD
:1038B800ADB2338BAB423FF601AF04E001339BB2AC
:1038C8008B427FF4F3AE01F061FC0F20FFF7A2FEFC
:1038D80005B0F0BD440C00204995050830000020D3
:1038E80098140020034B9A6812B19A68013A9A60BA
:1038F800704700BF440C00202DE9F3470120DFF892
:10390800D080DFF8D090014609F0C2FB00250124E1
:1039180003234FF480760227404669468DF8053028
:1039280000968DF804708DF806508DF8074009F060
:1039380007F840460821224609F082F8234BDFF8B1
:1039480098801A6844F2A243B2FBF3FA0AF1FF3AEC
:10395800204621461FFA8AFA09F0CAFBC8F804A0D3
:1039680048464146A8F80050A8F80250A8F8085060
:1039780088F80A5009F058FF7023A8F80C3004237F
:10398800A8F810300AF1FF3A6323642203FB0AF314
:10399800B3FBF2F39BB2C8F8143008F10C014846A7
:1039A800A8F80E40A8F81870A8F81A50A8F81C60D3
:1039B800A8F81E500AF056F84846214609F0C9FFF3
:1039C800484621460AF0CFFABDE8FC879C01002052
:1039D8000000024000000140540C002083B50E4650
:1039E8000746154910201C46154607F0B7FF10205A
:1039F800124907F0B3FF1020114907F0AFFF10205C
:103A08000E4907F0ABFF002310200E49019307F081
:103A1800A5FF334610200C493A4607F09FFF1020B7
:103A28000A492A4607F09AFF10200949224607F05A
:103A380095FF019B0133E7E78395050888950508FD
:103A4800A8950508B8950508C8950508DD950508E1
:103A5800EE95050808B5164B1A6A01321A621A6AF9
:103A6800012A1A4603D013484FF4A0710FE0586298
:103A7800194602E04B6A013B4B62506A0C4B002826
:103A8800F8D11A6A012A06D00A4840F24B110A4AAC
:103A98000A4BFFF7A3FF1A6A013A1A621B6A2BB195
:103AA8000448054A064B40F24D11F2E708BD00BF35
:103AB800540C0020FF950508EE53040829960508C4
:103AC8003A9605080C4B0D491A6844F2A24364283B
:103AD800B2FBF3F3D4BF20EAE0706420013B9BB251
:103AE8004B60013B58436422B0FBF2F080B248615E
:103AF80003480C3109F039BF9C010020540C002008
:103B08000000014010B5134B93F828202AB1124841
:103B1800124A134B4FF40A710EE0012283F8282051
:103B280066234FF0C042013BDBB2108033B90A482C
:103B38000A4A0C4B40F23221FFF750FF1488A4B216
:103B48008442F0D1084B1980024B002283F82820C8
:103B580010BD00BF540C0020FF950508F853040859
:103B68004B960508219505080000026010B5FFF77F
:103B7800C3FE6420FFF7A6FFE5204FF40041FFF7DE
:103B8800C1FF00200121FFF7BDFF01204FF4807124
:103B9800FFF7B8FF02204FF4E061FFF7B3FF0320FF
:103BA80041F23001FFF7AEFF04200021FFF7AAFF22
:103BB800082040F20221FFF7A5FF09200021FFF7A6
:103BC800A1FF0A200021FFF79DFF0C200021FFF72D
:103BD80099FF0D200021FFF795FF0F200021FFF727
:103BE80091FF10200021FFF78DFF11200021FFF722
:103BF80089FF12200021FFF785FF13200021FFF71E
:103C080081FF102041F2B071FFF77CFF37211120AE
:103C1800FFF778FF3220FFF71DFF122040F23B111B
:103C2800FFF770FF3220FFF715FF13204FF4C05144
:103C3800FFF768FF0F212920FFF764FF3220FFF705
:103C480009FF20200021FFF75DFF21200021FFF759
:103C580059FF30200021FFF755FF31200721FFF7DA
:103C680051FF322040F20311FFF74CFF352040F29C
:103C78000741FFF747FF40F20444362040F60F1192
:103C8800FFF740FF37202146FFF73CFF38204FF46D
:103C98008061FFF737FF39202146FFF733FF3C20CB
:103CA8000021FFF72FFF3D204FF48061FFF72AFF27
:103CB80050200021FFF726FFEF215120FFF722FFB8
:103CC80052200021FFF71EFF532040F23F11FFF75B
:103CD80019FF60204FF41C51FFF714FF61200121E8
:103CE800FFF710FF6A200021FFF70CFF802000215A
:103CF800FFF708FF81200021FFF704FF8220002141
:103D0800FFF700FF83200021FFF7FCFE842000213D
:103D1800FFF7F8FE85200021FFF7F4FE9020102120
:103D2800FFF7F0FE92200021FFF7ECFE932003211D
:103D3800FFF7E8FE95204FF48871FFF7E3FE972020
:103D48000021FFF7DFFE98200021FFF7DBFE0720A8
:103D580040F27311BDE81040D4E610B5FFF7CCFD72
:103D68006420FFF7AFFE21210720FFF7CBFE3220AA
:103D7800FFF770FE01210020FFF7C4FE3220FFF795
:103D880069FE23210720FFF7BDFE3220FFF762FE00
:103D980000211020FFF7B6FE41F28830FFF75AFEE7
:103DA80033210720FFF7AEFE3220FFF753FE112024
:103DB80046F63001FFF7A6FE3220FFF74BFE4FF420
:103DC800C0610220FFF79EFE3220FFF743FE12205B
:103DD80046F6EB41FFF796FE3220FFF73BFE032045
:103DE8004AF6A401FFF78EFE3220FFF733FE0021CA
:103DF8000C20FFF787FE3220FFF72CFE0D2040F63F
:103E08000C01FFF77FFE3220FFF724FE0E204FF44F
:103E18002C51FFF777FE3220FFF71CFEB0211E2041
:103E2800FFF770FE3220FFF715FE012042F63F3102
:103E3800FFF768FE3220FFF70DFE05200021FFF78F
:103E480061FE3220FFF706FE00210620FFF75AFE2A
:103E58003220FFF7FFFD16204EF61C71FFF752FEC9
:103E68003220FFF7F7FD172040F20311FFF74AFE53
:103E78003220FFF7EFFD00210B20FFF743FE322031
:103E8800FFF7E8FD00210F20FFF73CFE3220FFF787
:103E9800E1FD41200021FFF735FE3220FFF7DAFD72
:103EA80042200021FFF72EFE3220FFF7D3FD00212C
:103EB8004820FFF727FE40F23F143220FFF7CAFDE3
:103EC80021464920FFF71EFE3220FFF7C3FD0021DF
:103ED8004A20FFF717FE3220FFF7BCFD00214B20D8
:103EE800FFF710FE3220FFF7B5FD44204FF46F4175
:103EF800FFF708FE3220FFF7ADFD00214520FFF750
:103F080001FE3220FFF7A6FD21464620FFF7FAFD05
:103F18003220FFF79FFD302040F20771FFF7F2FDD6
:103F28003220FFF797FD31204FF40171FFF7EAFDCA
:103F38003220FFF78FFD32204FF40171FFF7E2FDC9
:103F480040F202543220FFF785FD21463320FFF767
:103F5800D9FD3220FFF77EFD342040F20751FFF7EC
:103F6800D1FD3220FFF776FD35204FF40171FFF7C0
:103F7800C9FD3220FFF76EFD36204FF40171FFF7BF
:103F8800C1FD3220FFF766FD21463720FFF7BAFD55
:103F9800A4F500743220FFF75DFD21463A20FFF7B3
:103FA800B1FD3220FFF756FD2F2041F2BE21FFF769
:103FB800A9FD3220FFF74EFD21463B20FFF7A2FD69
:103FC8003220FFF747FD00212320FFF79BFD322019
:103FD800FFF740FD00212420FFF794FD3220FFF772
:103FE80039FD25204FF40041FFF78CFD3220FFF703
:103FF80031FD00214F20FFF785FD3220FFF72AFD14
:104008004E200021FFF77EFD3220BDE8104021E55B
:1040180008B5124B93F829202AB11148114A124BBE
:1040280040F242210FE0012283F829202221662351
:104038004FF0C042013BDBB2118033B90848094A4E
:104048000A4B40F25B21FFF7C9FC108880B2222896
:10405800F0D1024B002283F8292008BD540C00201F
:10406800FF950508055404084B9605082195050891
:1040780010B5224B49F22032032823D8DFE800F09C
:10408800021A0B111C8846F6280041F228019442B6
:1040980018BF01461AE01C8841F2080046F60801DC
:1040A80004E01C8841F2300046F63001944208BF13
:1040B80001460BE0188846F62001904208BF4FF4ED
:1040C800815103E00E4840F2792113E01B8848F63D
:1040D8008912934205D049F22032934207D1032036
:1040E80000E01120FFF70EFDBDE8104090E70448FE
:1040F80040F28521034A044BFFF770FC3200002090
:10410800FF9505081A54040821950508014B1880E5
:104118000A209FE4000002604FF0C043188003F5B6
:1041280000331A881A88188880B270472DE9F04140
:10413800022098B00121002408F0AAFF01250226D8
:104148008C48169616A98DF85C508DF85D608DF830
:104158005E408DF85F4008F0F3FB1820294608F010
:1041680097FF2846294608F0ABFF21460C228248D3
:1041780008F066FC29460C227F4808F061FC0421FF
:104188000C227D4808F05CFC05210C227A4808F0D6
:1041980057FC07210C22784808F052FC08210C2211
:1041A800754808F04DFC09210C22734808F048FCBA
:1041B8000A2171480C2208F043FC0B216E480C229E
:1041C80008F03EFC0E210C226B4808F039FC0F2148
:1041D8000C22694808F034FC07210C22674808F0D3
:1041E8002FFC08210C22654808F02AFC09210C2222
:1041F800624808F025FC0A210C22604808F020FCDF
:104208000B210C225D4808F01BFC0C210A465B4878
:1042180008F016FC0D210C22584808F011FC0E215C
:104228000C22564808F00CFC0C2254480F2108F0C8
:1042380007FC03274CF6B3734F48169316A98DF85D
:104248005C608DF85E408DF85F408DF85D7008F019
:1042580077FB4FF6807316A9484816938DF85C6073
:104268008DF85E408DF85F408DF85D7008F068FB52
:1042780040F6B830FFF7EEFB314622463D4808F0DD
:10428800D4FB44F6FF70FFF7E5FB2A463146394870
:1042980008F0CBFB40F6B830FFF7DCFB4FF4805357
:1042A8000F961196099310264FF400230DF13C0840
:1042B80068460C93109412941395149415940094D2
:1042C8000194029404940694079408940A9405941B
:1042D8000B940396CDF8348008F0ABF86846109438
:1042E80012941395149415940F971197CDF838805C
:1042F80008F09FF82946204608F01BF940F6B83028
:10430800FFF7A8FB2046FFF707FF04461C491D4D91
:104318003046224607F022FB48F689139C421AD001
:1043280049F220339C420DD041F289239C4212D09D
:104338003046154907F012FB1448154A154BA621BB
:10434800FFF74CFB30461449224607F007FB2C8048
:10435800FFF70CFC0AE0FFF700FD48F689122A80F7
:1043680010200E4941F2892307F0F8FA18B0BDE889
:10437800F08100BF00040240000C0240001002401F
:10438800609605083200002077960508FF95050815
:104398003254040821950508AE960508E3960508E9
:1043A8004FF0C04322221A8003F5003382B01A88E6
:1043B80092B2ADF806201B889BB2ADF80630BDF866
:1043C800060080B202B07047134B1B8848F689126A
:1043D800934210B504460BD049F22032934213D1D0
:1043E800C1F1EF01202089B2FFF78CFB212006E004
:1043F800C1F1EF014E2089B2FFF784FB4F2021461F
:10440800BDE81040FFF77EBB0448054A054B40F263
:10441800F321FFF7E3FA00BF32000020FF950508FB
:104428003B540408219505082DE9F0410D46C5F1D6
:10443800F008411E5E18C2EB0802C5F1EF039BB2FB
:1044480092B2B6B29A422CBF904698469A4234BF6E
:1044580011461946864234BF3746074640F23F1395
:10446800864238BF06469E4228BF1E461B4B1B8805
:1044780048F68912B8F1EF0F28BF4FF0EF089342C2
:10448800044610D049F2203293421FD15020FFF742
:1044980039FB51204146FFF735FB52203946FFF7DB
:1044A80031FB53200AE041EA082189B24420FFF792
:1044B80029FB45203946FFF725FB46203146FFF703
:1044C80021FB20462946BDE8F0417DE70448054A1E
:1044D800054B40F2DD21FFF781FA00BF32000020D2
:1044E800FF95050849540408219505080020014650
:1044F800F0224FF4A07397E7072040F27311FFF7FB
:1045080001BB07200021FFF7FDBA10B51446FFF7DD
:104518005BFFFFF77DFD2046BDE81040F6E508B5D6
:10452800FFF752FF4FF0C04322221A8003F50033F1
:104538001A88188880B208BDF8B580B202FB03F566
:1045480089B292B29BB2069C9DF81C60FFF76CFF83
:104558000020FFF78DFD002709E034F8020B1EB19B
:10456800030A43EA002080B2FFF7D0FD0137AF42CB
:10457800F3DBBDE8F840B9E72DE9F74F16469DF89B
:1045880034200C9F01920546B2B280B20C46984680
:1045980089B29BB2FFF748FF4FF0000B0020FFF7EE
:1045A80067FDDA463DE0002D30DB09EB050340F2FC
:1045B8003F1293422ADC002C28DB0BEB0403EF2B81
:1045C80024DC19F00F0F04D1B9F1000FC8BF0AF1AC
:1045D800010A174B09EA0303002B03DA013B63F0D6
:1045E8000F030133019A0AB1C3F10F03012202FA42
:1045F80003F337F81A2013401BB213B10D4B588D33
:1046080001E00D4A508880B2FFF780FD09F10109E9
:1046180001E04FF00009C145C5DB0AF1010A0BF1C1
:10462800010BB345F5DB03B0BDE8F04F5EE700BF13
:104638000F000080540C0020320000202DE9F04FBC
:1046480085B004469DF83C00029200278A460390F4
:1046580088463E4640F23F1C9B463AE0002C2FDB42
:10466800E1452DDCBAF1000F2ADBB8F1EF0F27DCAA
:104678002A0702D1002DC8BF01361B49294000294D
:1046880003DA013961F00F010131039A0AB1C1F16E
:104698000F010E9830F8162003FA01F10A4012B201
:1046A80072B112494A8D019392B21FFA89F01FFA2A
:1046B80088F1CDF800C0FFF728FFDDF800C0019BA6
:1046C800013509F101095D45C8DB0136013708F1FB
:1046D8000108029A974203DAA14600250123F2E76E
:1046E80005B0BDE8F08F00BF0F000080540C00201B
:1046F80082B0044BADF80600BDF8062092B25A8588
:1047080002B07047540C002082B0044BADF806008C
:10471800BDF8062092B25A8002B0704732000020DD
:1047280070B50646FFF7E2FE0020FFF7A1FCF02473
:1047380009E0013D3046ADB2FFF7E8FC002DF8D1A5
:10474800013CA4B214B14FF4A075F2E770BD70B586
:104758001D461446FFF738FE2846FFF789FC00255A
:10476800054E05E0708D80B2FFF7D0FC0135ADB283
:10477800A542F7D170BD00BF540C00202DE9F041CF
:104788000C4616461F461A4600230546FFF7DFFF6C
:10479800611E711828463A46002389B2FFF7D7FFF1
:1047A8002846214632460123FFF7D1FF013D7F19F4
:1047B800B8B2214632460123BDE8F041C7E770B5DB
:1047C80080B202FB03F489B292B29BB2FFF72CFECF
:1047D8000020FFF74DFC0025054E04E0708D80B2E7
:1047E800FFF794FC0135A542F8DBBDE870407DE693
:1047F800540C0020F8B5561A0C46013189B21F46F0
:104808000546FFF7E1FD0120FFF732FC4FF0C043FA
:1048180022221A800E4A0F491388B6B2002304E0F8
:104828001088013321F8020B9BB2B342F8D121461C
:104838002846FFF7C9FD0120FFF71AFC002404E011
:104848003846FFF763FC0134A4B2B442F8D1F8BD8E
:1048580000000260A643002070B5194B194AD98D93
:1048680092F9004064180025A4B2AC4208BF0124A4
:10487800C62C28BFC6240F2615704FF6FF7288B0C5
:104888009E85DC855A8519200A222B462146FFF78A
:104898005EFF21463046FFF742FE224603460A499C
:1048A80068460EF09FFC6A4604A808490EF09AFC78
:1048B8003220D22104AA2B4600F0ECF908B070BDD2
:1048C800540C0020502B0020229705082A97050831
:1048D8002DE9F0431F2093B0FFF722FF4FF47840F3
:1048E800FFF71EFF4FF6E0754FF4FC60FFF718FF67
:1048F8002846FFF715FF0020494CFFF711FF00205D
:104908000146642203464FF6FF79A4F82A90FFF780
:104918001EFF00200A2164220346FFF718FF00202B
:104928000146642201234FF478476585FFF70FFF9E
:104938007720EF21C82200234FF4FC666785FFF734
:1049480006FFBD213222012340F23F106685FFF7A2
:10495800FEFEA0203222002378216785FFF7F7FEAC
:10496800A0207821322201234FF01F086685FFF727
:10497800EEFEA020782132220223A4F82A80FFF735
:10498800E6FEA0207821322203236585FFF7DFFEAB
:10499800244B2549A3F8028002AD3C2228460EF09C
:1049A8005FFBEB20C3210522302300950025A4F8E6
:1049B8002A900195FFF7E0FD32210A2096220B4646
:1049C8006785FFF7DBFE32213C2096220B46668581
:1049D800FFF7D4FE32210B4696226E20A4F82A80D7
:1049E800FFF7CCFEFFF78DFDFFF786FD3220FFF7BE
:1049F80069F82846FFF766F86420FFF763F80B4B61
:104A080003F110028DE8240028465A681B682946DD
:104A1800FFF792FD1195119B01331193FBE700BF3E
:104A2800540C0020320000205E540408A0780108CD
:104A3800004870476815002082B0064BADF80600A4
:104A4800BDF8062092B21A80188880B202B0FFF72B
:104A58004FBE00BF64150020014B188880B2704714
:104A68006415002082B0064BADF80600BDF806209C
:104A780092B21A80188880B202B0FFF745BE00BF14
:104A880066150020014B188880B270476615002013
:104A9800FFF746BEFFF7C8BCFFF759BEFFF76EBE6B
:104AA800FFF78DBE2DE9F04F4FEA420800253D4C37
:104AB80085B082468B46C8F1030817462E461FFA72
:104AC80087F909EB0B0C228805EB0A031FFA8CFC0B
:104AD8009BB26146184692B2CDF804C00293FFF724
:104AE80014FDC9EB0B0292B20392029B2288039930
:104AF800184692B2FFF709FDDDF804C02288C5EB1D
:104B08000A039BB26146184692B20293FFF7FDFC76
:104B1800029B22880399184692B2FFF7F6FC05EB30
:104B28000B0292B2039209EB0A03228803999BB203
:104B3800184692B20293FFF7E8FC029B2288C5EB65
:104B48000B0C1FFA8CFC1846614692B2CDF804C0D3
:104B5800C9EB0A09FFF7D9FC228803991FFA89F9DA
:104B680092B24846FFF7D1FC2288DDF804C092B221
:104B780048466146FFF7C9FCB8F1000F04DA08EBB4
:104B8800860808F1060805E0F31B08F10A0808EB97
:104B98008308013F01360135BE42ADB28FD905B059
:104BA800BDE8F08F6415002008B9FFF7AABC0128FA
:104BB80001D1FFF7A1BC7047704700200146F022E1
:104BC8004FF4A073FFF730BC704708B505280CD820
:104BD800DFE800F0121403050709094808BD094871
:104BE80008BD094808BD094808BD0948094A0A4BD3
:104BF80040F24111FEF7F2FE084808BD084808BD1A
:104C080020000020100000200800002000000020E4
:104C18002F9705089A5404082195050828000020B4
:104C28001800002010B50446FFF7CFFF014B1860AD
:104C38001C7110BD38000020014B1879704700BF67
:104C48003800002008B5FFF7C0FF808808BD08B508
:104C5800FFF7BBFFC08808BDF7B51F460B4B0C4ECE
:104C68001D681446EA882B68203C5443A4B2AE1B46
:104C780003EB440418BF0126AB888DE8500017B138
:104C8800FFF7DCFC01E0FFF777FCFEBD38000020F1
:104C9800280000202DE9F0410F46984615460446A5
:104CA800084E08E0204643463946FFF7D5FF3368EB
:104CB8009B88E418A4B215F8012B002AF2D1BDE8AC
:104CC800F08100BF3800002010B504460846214690
:104CD800BDE81040DEE7094B70B5044618790E466A
:104CE8001546FFF7B4FFC6F1F001091A89B220464C
:104CF8002A460023BDE87040CCE700BF38000020FA
:104D0800704700BF044B1A680AB9044A1A601A6847
:104D18001018186010467047840C002038CF002007
:104D28004FF0FF30704708B50248034A034B37215C
:104D3800FEF754FE4E970508B0540408219505085F
:104D48000120704710B504460A48022108F026FCE5
:104D58000028F9D00748214608F0E9FB0548012159
:104D680008F01CFC0028F9D00248BDE8104008F003
:104D7800DBBB00BF0038004010B51948022108F01D
:104D88000DFC0028F9D01648002108F0D0FB144883
:104D9800012108F003FC0028F9D0114808F0C4FBF1
:104DA8000402A4B2002301E001339BB2002BFBD024
:104DB8000B48022108F0F2FB0028F9D0084800212E
:104DC80008F0B5FB0648012108F0E8FB0028F9D0F7
:104DD800034808F0A9FB2043C0F3CB0010BD00BF77
:104DE800003800402DE9F0478AB00AAF0A200121B7
:104DF80008F04EF94FF4604347F8143D474EDFF88A
:104E080024A1012400254FF00208304639468DF8C8
:104E18001A508DF818808DF819808DF81B4007F00E
:104E28008FFD30460D21052207F00AFE30460E217F
:104E3800052207F005FE052230460F2107F000FE87
:104E480021464FF4804008F047F9504608F022FA0E
:104E58004FF48273ADF802304FF40073ADF80A30A6
:104E68003823ADF80C30504607236946ADF81030AA
:104E7800ADF80050ADF80450ADF80650ADF8085044
:104E8800ADF80E5008F038FA5046214608F0CFFA2F
:104E9800A9468DF81A5030464FF480553946059585
:104EA8008DF818408DF819808DF81B4007F048FDE3
:104EB8003046294607F0B5FD4025394618488DF893
:104EC80018908DF819808DF81A908DF81B4005956B
:104ED80007F036FD21464FF4804008F009F9062115
:104EE800032008F093FB0C2307A88DF821300795C1
:104EF8008DF820908DF8224007F016FA17238DF8C8
:104F0800243009A80F238DF825308DF826308DF828
:104F1800274002F041FB0AB0BDE8F08700040240D8
:104F2800000C024000380040014B1878704700BF61
:104F3800880C0020024B5A889B8802800B8070479F
:104F4800880C0020014B00221A707047880C002042
:104F5800F0B593B06846002148220EF0C3F86D46BC
:104F6800002464484FF4805107F05DFD002301E000
:104F780001339BB2002BFBD09020FFF7E3FE002308
:104F880001E001339BB2002BFBD0FFF7F5FE4FF495
:104F980080510746574807F044FD002301E00133DC
:104FA8009BB2002BFBD053484FF4805107F03BFDD8
:104FB800002301E001339BB2002BFBD0D020FFF788
:104FC800C1FE002301E001339BB2002BFBD0FFF7A9
:104FD800D3FE4FF480510646464807F022FD45F8B7
:104FE800047B01342E6244484021E4B207F007FDF7
:104FF80010B9092CB5D101E0092C78D19DE80C0035
:10500800D218029B03980699D218049BC018059BD6
:10501800C018079BCB180899032490FBF4F092FB67
:10502800F4F25B1893FBF4F3151AC11A9C1A002DBD
:10503800B8BF6D420029B8BF4942002CB8BF6442CE
:10504800502D03DD502909DD502C50DC8D4205DA46
:10505800AC424FF0020405DB111806E08C424FF019
:10506800020401DAD11800E0C1180A9B099A0C98C9
:105078000F9DD2180B9BD2180D9BC0180E9BC01801
:10508800109BEB18119D91FBF4F1032492FBF4F2B1
:1050980090FBF4F05B1993FBF4F3161AC41A9D1AEB
:1050A800002EB8BF7642002CB8BF6442002DB8BFAE
:1050B8006D42502E89B203DD502C09DD502D16DCCF
:1050C800A64205DAB5424FF0020405DB131806E0E4
:1050D800A5424FF0020401DAD31800E0C318074ACA
:1050E80093FBF4F39BB2938001235180137013B0A8
:1050F800F0BD00BF00040240000C0240880C0020F4
:10510800FFF712BFF7B505460C4601A80DF10601D9
:10511800FFF710FF1B4BBDF80660BDF8040093E8CD
:105128000600724301FB002299685218164992FB47
:10513800F1F207EE102AF8EEC77A40F23F17FCEEBC
:10514800E77A17EE902A92B2B2F5207F28BF3A4646
:105158002A801D69DA685B696E4302FB0060C0182B
:1051680090FBF1F107EE101AF8EEC77AFCEEE77A39
:1051780017EE903A9BB2B3F5F07F28BFEF23238058
:10518800FEBD00BF900C002040420F00FFF7DABEC2
:10519800014B187E704700BF900C0020FFF7CABE75
:1051A800042808B505D90748074A084B7D21FEF7AA
:1051B80015FC054B03EB8000038B0B80438B13809E
:1051C80008BD00BF6F970508B65404088D970508F9
:1051D80008B5082001F08CF942F69643C31A5842E4
:1051E80040EB030008BD10B50A2001F0A9F90C4CEA
:1051F80020600E2001F0A4F96060122001F0A0F9EF
:10520800A060162001F09CF9E0601A2001F098F9DE
:1052180020611E2001F094F901236061237610BDFE
:10522800900C002010B5FFF7DDFD01F02BFA0446C5
:1052380001F034FA074903462246202006F08EFB87
:10524800FFF7C6FF28B101F037FA10B9BDE81040E2
:10525800C9E710BDC997050810B5104C0A20216888
:1052680001F055F961680E2001F051F9A16812208A
:1052780001F04DF9E168162001F049F921691A2079
:1052880001F045F961691E2001F041F9082042F654
:105298009641BDE8104001F01DB900BF900C0020F8
:1052A8002DE9F04F0346A7B0B0F800C01C898688E6
:1052B800DF885D89CDF810C0B249B0F802C0B3F8F4
:1052C8000C90B3F80E80CDF824C00FFA84FB30B2EE
:1052D80001220FFA87FE0BEB000C0A7629B20FFAAF
:1052E80089FACDF888C001EB0E0C0FFA88F2CDF8D8
:1052F80090C00AEB0B0CCDF830C002EB010CCDF8D6
:1053080058C0B3F810C05B8ACDF800C00FFA8CFC07
:1053180006910CEB00010A9102930CEB0A011BB2F7
:10532800239103EB0E010E9199182591049900FA27
:1053380081F0584450446044DDF824C006990EFAC0
:105348008CFEDDF810C01FFA80FB1CFB0CF08E44AD
:1053580016FB0600964414FB0400009A19FB09008A
:105368009E4412FB02001FFA8EFA09F021FADDF8BA
:1053780024C0029ACDE912011CFB0CF017FB0700B0
:1053880015FB050018FB080012FB020009F010FAD3
:10539800DDF824C0029ACDE9140104991CFB01F33D
:1053A80017FB063615FB0466009B18FB096612FB03
:1053B800036009F0FDF9DDE91423CDE90001DDE919
:1053C800120109F06BFA04460D46DDE900010246B8
:1053D8000B4609F063FA02460B462046294609F0B7
:1053E800A9F8CDE91801584609F0F2F9CDE91001FC
:1053F800DDE91023DDE9000109F050FACDE90601E5
:10540800504609F0E5F9804689464246DDE9120131
:105418004B4609F043FADDE91023CDE91C01DDE92B
:10542800140109F03BFA002206460F46564BDDE907
:10543800180109F033FA424604460D464B46DDE9A9
:10544800060109F02BFA02460B4609F075F80246E8
:105458000B462046294609F06FF8424604460D4699
:105468004B46DDE91C0109F019FA02460B462046B5
:10547800294609F05FF8DDE9102304460D46304659
:10548800394609F00BFA02460B462046294609F030
:1054980051F8DDF828C0CDE902014FEA8C10DDF89B
:1054A80030C000EB0C20DDF810C0A0241CFB040069
:1054B80009F07EF9DDF838C0CDE90A014FEA8C1011
:1054C800DDF858C000EB0C20DDF824C01CFB0400FC
:1054D80009F06EF9CDE90C01504609F069F9DDE9EA
:1054E8001023CDE91601DDE90C0109F0D7F9424690
:1054F800CDE91E014B46DDE90A0109F0CFF9424624
:10550800CDE920014B46DDE9000109F0C7F9324633
:105518003B4609F00FF8CDE90E01584609F048F965
:10552800DDE91C23CDE91A01DDE9060109F002F8DD
:10553800DDF88CC0C024CDE9060104FB0CF0DDF8D1
:1055480088C0302505FB0C00DDF810C078261CFB50
:10555800060009F02DF9DDF894C0824604FB0CF032
:10556800DDF890C005FB0C00DDF824C01CFB06002C
:105578008B4609F01DF9DDE9102306460F4609F0B0
:105588008DF903E0900C0020000014404246CDE95C
:1055980004014B465046594609F080F9DDE91423C9
:1055A80080468946DDE90A0109F078F9DDE900233A
:1055B80004460D46DDE90C0109F070F902460B4678
:1055C8002046294608F0B6FF0022A14B09F066F9EB
:1055D800DDE9202304460D46DDE91E0108F0AAFF97
:1055E80002460B46DDE9160109F058F902460B465A
:1055F8002046294608F0A0FF002204460D46954B98
:10560800DDE90E0109F04AF902460B462046294613
:1056180008F092FFDDE9022309F06AFA88A3D3E9CA
:10562800002309F03BF909F0D3FB8B490860DDE959
:105638001223DDE90C0109F031F9DDE90023044604
:105648000D46DDE90A0109F029F902460B46204614
:10565800294608F06FFF00227D4B09F01FF9DDE9AC
:105668001E2304460D46DDE9200108F063FF0246CB
:105678000B46DDE91A0109F011F902460B462046EE
:10568800294608F059FF002204460D46714BDDE912
:10569800060109F003F902460B462046294608F0A0
:1056A8004BFFDDE9022309F023FA65A3D3E90023C0
:1056B80009F0F4F809F08CFB674A5060DDE90E2325
:1056C800DDE90A0109F0EAF8DDE9062304460D469A
:1056D800DDE90C0109F0E2F802460B4620462946AE
:1056E80008F02AFF002204460D465A4BDDE918014E
:1056F80009F0D4F802460B462046294608F01CFF5C
:10570800DDE9022309F0F4F94DA3D3E9002309F0F8
:10571800C5F809F05DFB504B59469860DDE9142344
:10572800504609F0BBF8DDE9002304460D46304633
:10573800394609F0B3F802460B462046294608F0D8
:10574800F9FE0022424B09F0A9F8424604460D46EC
:105758004B46DDE9040108F0EDFE02460B46DDE9A3
:10576800160109F09BF802460B462046294608F028
:10577800E3FE35A3D3E9002304460D46DDE90E0117
:1057880009F08CF802460B462046294608F0D4FE5C
:10579800DDE9022309F0ACF929A3D3E9002309F0D4
:1057A8007DF809F015FBDFF8B0C0DDE91223CCF86D
:1057B8000C003946304609F071F8DDE9002304464B
:1057C8000D465046594609F069F802460B462046F0
:1057D800294608F0AFFE00221D4B09F05FF8DDE90D
:1057E800042304460D464046494608F0A3FE0246F7
:1057F8000B46DDE91A0109F051F802460B4620462E
:10580800294608F099FE10A3D3E9002304460D4663
:10581800DDE9060109F042F802460B462046294612
:1058280008F08AFEDDE9022309F062F904A3D3E94E
:10583800002309F033F809F0CBFA074908610DE0B5
:105848000000000080842E410000000000C082405B
:105858000000144000008940900C0020DDE90E2370
:105868005046594609F01AF8DDE9062304460D4664
:105878003046394609F012F802460B4620462946BA
:1058880008F05AFE11A3D3E9002304460D46DDE9CA
:10589800180109F003F802460B462046294608F08D
:1058A8004BFEDDE9022309F023F90AA3D3E900231B
:1058B80008F0F4FF09F08CFA034A506127B0BDE8FC
:1058C800F04FC9E4AFF30080900C00200000000006
:1058D80000C082400000000080842E41AFF30080A9
:1058E800064B074A596811601969064A1160D96957
:1058F800054A11609A6A054B1A60704740000020FB
:10590800243C00204442002018420020CC3B0020C8
:10591800014B1878704700BFAC0C0020032808B56D
:1059280005D90548054A064B7121FEF757F80C239F
:105938005843044B185808BD04980508E254040855
:105948001E98050840000020032808B505D9064818
:10595800064A074B7621FEF741F8064B0C2202FB5C
:105968000030406808BD00BF04980508F2540408D8
:105978001E98050840000020034B044A1B780C21A0
:1059880001FB032398687047AC0C002040000020FE
:10599800034B044A1B780C2000FB032399607047D3
:1059A800AC0C002040000020144B1B78012B10B5D4
:1059B800134B144C0ED11968C82000F0A8FD2168BB
:1059C800CC2000F0A4FD104BD020196800F09FFDFA
:1059D800D4200DE01968D82000F099FD2168DC205A
:1059E80000F095FD084BE020196800F090FDE420D8
:1059F800064B1968BDE8104000F089BDEC0D002089
:105A0800243C00204442002018420020CC3B0020C7
:105A1800144B1B78012B10B5134C0FD1C82000F084
:105A28008FFD2060CC2000F08BFD104B1860D0203B
:105A380000F086FD0E4B1860D4200EE0D82000F050
:105A48007FFD2060DC2000F07BFD084B1860E02023
:105A580000F076FD064B1860E42000F071FD054B60
:105A6800186010BDEC0D0020243C002044420020AA
:105A780018420020CC3B002008B502F0D9FA10B13A
:105A8800BDE80840C4E7BDE8084029E70148FBF73E
:105A9800B8BF00BF501300200148FBF7B2BF00BFDA
:105AA800501300200148FBF7ACBF00BF5013002083
:105AB8000148FBF7A6BF00BF50130020032808B514
:105AC80005D91448144A154B4E21FDF787FF144B8E
:105AD8001870144B02281870134B0FD0032813D0DA
:105AE800012805D0114A12681A60BDE80840CDE7C0
:105AF8000F4A12681A60BDE80840CDE70D4A1268DF
:105B08001A60BDE80840CDE70B4A12681A60BDE884
:105B18000840CDE704980508035504084898050887
:105B2800AC0C0020123C00209801002090010020BD
:105B38008C0100208801002084010020064B0749C1
:105B48005960C021002219721E211A70D9601A7476
:105B58005A611A76DA6170479415002040787D0101
:105B680010B50321FF22C02001F072F81F4C10214C
:105B780020608022C02001F06BF811212060802273
:105B8800C02001F065F8122120608022C02001F0B9
:105B98005FF8132120608022C02001F059F81421F9
:105BA80020608022C02001F053F815212060802257
:105BB800C02001F04DF8802220601621C02001F09D
:105BC80047F82060C0201721802201F041F82060AA
:105BD800074CC020227AB72101F03AF80023237439
:105BE80063612376E3610123237010BDF03B00203D
:105BF8009415002038B5C0200321FF2201F028F8B1
:105C08000B4D00242B19615D5A78C020023401F035
:105C18001FF8C82CF6D1B121AC22C02001F018F829
:105C2800C0200321002201F013F8002038BD00BF76
:105C3800175504082DE9F34706460F4692461D46B8
:105C48001AB90C1FE401914635E005EE902A06EEDC
:105C5800903AB8EE657AF8EE667AFC01C7EE277AD4
:105C6800A4F500749FED5C7A67EE877A17EE900AC8
:105C780008F0C0FD41EC100B0AF0D6FD59EC108B72
:105C88004946404609F0CCF824184FEACA1008F0F3
:105C98008FFDCDE90001284608F08AFD4B464246B3
:105CA80008F0FCFD02460B46DDE9000108F042FC65
:105CB80009F0B6F88146002E14BF4FF022084FF0C5
:105CC8001A08C5F307224146C02000F0C1FF08F1B9
:105CD8000101EAB2C02000F0BBFFC4F3014208F1A1
:105CE8000201C02000F0B4FFC4F3072208F1030149
:105CF800C02000F0ADFFE2B208F10401C02000F0BE
:105D0800A7FFC9F3034305F4702243EA123208F1EE
:105D18000501C02000F09CFF08F10601C9F3072225
:105D2800C02000F095FF08F107015FFA89F2C02052
:105D380000F08EFFC020B121A02200F089FF07EEFD
:105D4800107A264CF8EEC77A0EBBD4ED015A06EE4F
:105D580090AAB8EE657A05EE905AB8EE666AF8EE43
:105D6800656A0123C6EE266A237477EEA67A67EE83
:105D7800277A17EE900A08F03DFD41EC100B0AF067
:105D880053FD51EC100B09F04BF8606120E005EE73
:105D980090AAD4ED016AB8EE656A05EE905AB8EE9D
:105DA800667AF8EE656A0123C6EE266A237677EEF0
:105DB800A67A67EE277A17EE900A08F01BFD41ECE9
:105DC800100B0AF031FD51EC100B09F029F8E061D5
:105DD8000020BDE8FC8700BF0000004394150020A8
:105DE8000022012326E7012838B50D4604D00228F1
:105DF8000CBF3C242C2400E034242146C02000F0B1
:105E0800A1FF05F0070200F00F0040EA0212214648
:105E1800C020BDE8384000F01BBF2DE9F3470A9CBD
:105E28001D4607468A461646524B01E06D0864082F
:105E38009C42FBD82DB906F10076043EF601A9462E
:105E480034E006EE905AB8EE667A06EE904AF8EE1E
:105E5800667AF601C7EE277AA6F500769FED467AB0
:105E680067EE877A17EE900A08F0C4FC41EC100B35
:105E78000AF0DAFC59EC108B4946404608F0D0FF8E
:105E88003618E80108F094FCCDE90001204608F036
:105E98008FFC4B46424608F001FD02460B46DDE901
:105EA800000108F047FB08F0BBFF8146022F9BBFAB
:105EB800324BDB194FF0000893F8C880C4F307226F
:105EC8004146C02000F0C4FE08F10101E2B2C9B2A7
:105ED800C02000F0BDFE08F10201C9B2C6F30142BC
:105EE800C02000F0B5FE08F10301C9B2C6F30722CD
:105EF800C02000F0ADFE08F10401C9B2F2B2C02022
:105F080000F0A6FE04F47024C9F3034308F1050168
:105F180043EA1432C9B2C02000F09AFE08F1060123
:105F2800C9B2C9F30722C02008F1070800F090FEA3
:105F38005FFA89F25FFA88F1C02000F089FEBAF1B1
:105F4800010F0CBF2F220F220DB942F04002012F82
:105F580006D002D3022F0AD105E0C020102104E0A8
:105F6800C020112101E0C020122100F071FE0020A4
:105F7800BDE8FC87FFFF0F00000000431755040829
:105F880007B5012300930023FFF747FF0EBD002844
:105F98000CBFFF22002208B5C020032100F058FEE4
:105FA800002008BD08B5C020B121AC2200F050FE89
:105FB800002008BD08B50420012107F069F84FF456
:105FC80080700121BDE8084007F092B807B50223A8
:105FD800009303238DF804300348002369468DF8A5
:105FE800073006F0ADFC0EBD0008024030B5124D7A
:105FF8008BB0002406A8069407940894099405F029
:106008006DFE00948DF804408DF8054002940394C9
:1060180004942846012469468DF8144005F02FFEA3
:1060280028460B212246062305F0A4FE28462146D1
:1060380005F06EFE0BB030BD0020014010B5002108
:1060480004460122302000F003FEC0B9012001F00F
:106058001FF8002CB8BF4034E4B21021224630208B
:1060680000F0F6FD012001F013F83020112122463E
:1060780000F0EEFD0120BDE8104001F009B810BDA8
:1060880010B5002104460122302000F0E1FDC0B91E
:10609800012000F0FDFF002CB8BF4034E4B212210B
:1060A8002246302000F0D4FD012000F0F1FF30201E
:1060B8001321224600F0CCFD0120BDE8104000F07D
:1060C800E7BF10BD38B5012205460C463020002137
:1060D80000F0BEFDF0B9012000F0DAFF25EAE57214
:1060E8005F2AA8BF5F223B21D2B2302000F0B0FD6A
:1060F800012000F0CDFF24EAE4725F2AA8BF5F22E6
:10610800D2B230203C2100F0A3FD0120BDE8384088
:1061180000F0BEBF38BD302810B504460ADC10F1C7
:106128007F0F02DB002802DB05E06FF07E0404F538
:10613800807400E03024002130200A4600F088FDF9
:10614800A8B90120E4B200F0A3FF41212246302083
:1061580000F07EFD012000F09BFF30204221224606
:1061680000F076FD0120BDE8104000F091BF10BDA1
:10617800282810B5044609DC10F1180F02DB0028A6
:1061880002DB04E06FF017047F3400E028240021CC
:1061980030200A4600F05CFDA8B90120E4B200F006
:1061A80077FF53212246302000F052FD012000F0F5
:1061B8006FFF30205421224600F04AFD0120BDE83F
:1061C800104000F065BF10BD08B530200021012245
:1061D80000F03EFD60B9012000F05AFF3020332165
:1061E800402200F035FD0120BDE8084000F050BF16
:1061F80008BD10B530200021012200F029FD044619
:1062080060B9012000F044FF30203321224600F01D
:106218001FFD0120BDE8104000F03ABF10BD10B5C9
:1062280030200021012200F013FD0446A0B901200E
:1062380000F02EFF34212246302000F009FD012015
:1062480000F026FF30203721224600F001FD012012
:10625800BDE8104000F01CBF10BD4020EEE6402015
:106268000EE708B500210122302000F0F1FC0120E2
:1062780000F00EFF30203421024600F0E9FC012036
:1062880000F006FF30203721024600F0E1FC012033
:10629800BDE8084000F0FCBE08B50021012230200E
:1062A80000F0D6FC012000F0F3FE302034210C224F
:1062B80000F0CEFC0120BDE8084000F0E9BE000077
:1062C800184B1949D3ED006A93ED017A00231A4659
:1062D8009FED166A03E0F0EE476AB0EE677A505E0B
:1062E80005EE900AF8EEE57A0133C7EE867A9BB29E
:1062F80018B204327F2877EEE67AECDD27EE077ACB
:1063080007EEA77A0A49074A0B80BDEEC77A002331
:1063180013605360C2ED027A17EE102A054B920003
:106328001A607047B00C0020502700200000FA4582
:10633800803B00201C1800202DE9F84F2E4B2F4AD7
:1063480019682F4B19B92F4911602F4A02E02F49BC
:1063580011602F4A1A602F4BDFF8BCA0DFF8BC9001
:10636800DFF8BCB000221A80244A9846176830E04B
:1063780007EB84036500B3F9023007EE103AF8EE34
:10638800C77A013617EE900A08F034FA18A3D3E951
:10639800002308F083FA08F01BFD29F815002AF8F5
:1063A800140037F9243007EE103AF8EEC77A0135B1
:1063B80017EE900A08F01EFA0DA3D3E9002308F09F
:1063C8006DFA08F005FD2BF8140029F81500A8F857
:1063D8000060B8F8006034B2FF2CC9DD00F05EF848
:1063E80000F06AF801F07CF9BDE8F84F68E700BFF3
:1063F8009A9999999999E93F101800200418002052
:106408003C160020522F0020522B0020523700202B
:1064180052330020803B00205023002050270020CA
:106428005025002010B50B4C204605F0D6FE0A4B2F
:1064380018600A4805F0D1FE094B1860FFF77CFF89
:10644800084B0949012220469A81BDE8104005F011
:1064580045BF00BF1060024010180020886002404D
:106468002C180020B00C002020800010014B186868
:10647800704700BF1C18002008B5054B054819884F
:106488000022012309F0C2F9034B187008BD00BFB0
:106498007000002038230020541E002003480449BF
:1064A800044A4FF4807309F029BA00BF7400002031
:1064B800502300203621002003480449044A4FF4A1
:1064C800807309F01BBA00BF80000020502500200F
:1064D8007019002038B505460C460135C1F307216F
:1064E80000F0E4FDA8B2E1B200F0E0FD00B238BD72
:1064F80038B5044600F0EEFC01340546A0B200F0C1
:10650800E9FCEDB2C0B240EA052000B238BD37B5AB
:106518000B0E8DF804300B0C8DF805300B0A8DF836
:1065280006308DF80710002400E0284601AB451C12
:10653800E15C013400F0BAFD042CADB2F5D13EBDEA
:1065480037B5002400E02846451C00F0C3FC01AB29
:10655800ADB2E0540134042CF5D19DF805009DF846
:106568000430000440EA03609DF8073018439DF8A2
:10657800063040EA03203EBD38B50446642000F0EA
:1065880087FD25786068AD00EDB2257006F03DFA0C
:10659800237A40FA03F000F003000543104B2570FE
:1065A80005F00F055A5D6378D218D2B2D3B2013222
:1065B800D2B2022A637001D80022A2705BB2012B0A
:1065C80003DD0123A3700023637094F901300133C4
:1065D80003DAFF23A3700023637094F9020038BD27
:1065E800E2550408F7B504200121234F06F050FDB9
:1065F80002AD01214FF48040012406F079FD002608
:106608004FF4B0733846694645F8083D8DF8046084
:106618008DF8074006F094F91020214606F038FD61
:1066280078236946154800938DF804608DF8074073
:1066380006F086F90420214606F02AFD21464FF48B
:10664800804006F055FD1C233846694600938DF8B6
:1066580004608DF8074006F073F90220214606F021
:1066680017FDB02306488DF8046069468DF8074089
:10667800009306F065F9FEBD0008024000100240D4
:1066880000040240802108B5034806F0B8F9D0F1AB
:10669800010038BF002008BD0004024008B54FF4CF
:1066A8008071044806F0ABF9D0F1010038BF002032
:1066B80008BD00BF0008024008B5FFF7E3FF08B1B6
:1066C800FFF7ECFFC0B208BD10B5642000F0E0FC95
:1066D8000F48FFF751FF044610B90E4B187009E038
:1066E800FFF7DCFF30B9002C0A4B01DD012200E086
:1066F800FF221A700848FFF73FFF0028074B01D117
:10670800187010BD01DD012200E0FF221A7010BDD3
:10671800C00000201C420020CC000020502B00208C
:1067280007B50220012106F0B3FC012300938DF880
:10673800043002238DF805300448002369468DF89B
:1067480006308DF8073006F0FBF80EBD0004024055
:1067580010B5084C01210022204606F066F940F2E7
:10676800FF4000F095FC012120460A46BDE8104094
:1067780006F05BB90004024008B5FFF7E9FF002105
:106788000A46302000F064FA012000F081FC012163
:106798000A46302000F05CFA012000F079FC002164
:1067A8000122302000F054FA012000F071FC012190
:1067B8000822302000F04CFA012000F069FC022188
:1067C8000122302000F044FA012000F061FC002191
:1067D8000A46302000F03CFA012000F059FC1B2149
:1067E800CD22302000F034FA012000F051FC0421C1
:1067F8000322302000F02CFA012000F049FC062189
:106808000822302000F024FA012000F041FC072182
:106818000A46302000F01CFA012000F039FC08215B
:106828008022302000F014FA012000F031FC1E21F3
:10683800B022302000F00CFA012000F029FC0521DC
:106848009122302000F004FA012000F021FC0D21F3
:106858000322302000F0FCF9012000F019FC0E2181
:106868000022302000F0F4F9012000F011FC14217E
:106878008022302000F0ECF9012000F009FC0B2107
:106888008822302000F0E4F9012000F001FC3020DB
:106898000C21822200F0DCF9012000F0F9FB122122
:1068A8008822302000F0D4F9012000F0F1FB1321F8
:1068B8008C22302000F0CCF9012000F0E9FB002107
:1068C8000122302000F0C4F9012000F0E1FB0C2186
:1068D8000822302000F0BCF9012000F0D9FB0D217E
:1068E8000822302000F0B4F9012000F0D1FB0E217D
:1068F8000822302000F0ACF9012000F0C9FB0F217C
:106908000822302000F0A4F9012000F0C1FB00218A
:106918000A46302000F09CF9012000F0B9FB402124
:106928000222302000F094F9012000F0B1FB00228F
:106938004121302000F08CF9012000F0A9FB302023
:106948003F21D42200F084F9012000F0A1FB0021AE
:106958000122302000F07CF9012000F099FB102181
:106968000F22302000F074F9012000F091FB112172
:106978000F22302000F06CF9012000F089FB122171
:106988000022302000F064F9012000F081FB13217F
:106998000022302000F05CF9012000F079FB092189
:1069A8003C22302000F054F9012000F071FB002156
:1069B8000122302000F04CF9012000F069FB302062
:1069C8003421024600F044F9012000F061FB302038
:1069D8003721024600F03CF9012000F059FB36212E
:1069E8000322302000F034F9012000F051FB392156
:1069F8000322302000F02CF9012000F049FB3B2154
:106A08003C22302000F024F9012000F041FB3C2119
:106A18000A46302000F01CF9012000F039FB002163
:106A28000A46302000F014F9012000F031FB512112
:106A3800C022302000F00CF9012000F029FB3020A2
:106A48005221002200F004F90120BDE8084000F0BE
:106A58001FBB00BF2DE9F04F454E464D93B00121B5
:106A68004FF4001006F014FB304605F0B7FA4FF06B
:106A7800C0630293404B0393404B002404934FF4AC
:106A880000794FF400334FF480684FF400674FF4F7
:106A9800005A4FF4807B304602A90C930193099762
:106AA800CDF8189005940794CDF82080CDF828A04B
:106AB800CDF82CB00D9405F01DFB22463046304928
:106AC80005F073FB3046012105F079FB01210A46E8
:106AD8004FF0402006F04AFD284605F07FFA294A83
:106AE800019B0392284A0C9304922846402202A94B
:106AF800059209970294CDF818900794CDF8208054
:106B0800CDF828A0CDF82CB00D9405F0F3FA224664
:106B180028461E4905F049FB2846012105F04FFB90
:106B280042F2107701220221194806F01FFD38466B
:106B380000F0AEFA3046012105F017FB0121284686
:106B480005F013FB384600F0A3FA0B238DF8443008
:106B580011A801238DF845408DF846408DF847303F
:106B680000F01AFD384600F093FA13B0BDE8F08F34
:106B780010600240886002400C40004052370020FC
:106B8800522F00200C3C004052330020522B002092
:106B9800003C004002481021012205F05DBB00BF07
:106BA8001060024013B50220012106F071FA4FF47B
:106BB80010730E4C009302238DF804308DF80530C5
:106BC80001238DF806302046002369468DF80730EA
:106BD80005F0B6FE20460621042205F031FF2046C6
:106BE8000921042205F02CFF1CBD00BF000402404F
:106BF80030B5154D85B001214FF4001006F06CFA40
:106C0800284605F033FF0023ADF804304BF6FF7338
:106C1800ADF806303323ADF808304FF48063ADF893
:106C28000A304FF48043ADF80C3004AC074B2846CB
:106C3800012144F8103D05F0BBFF2846694605F0E0
:106C480043FF05B030BD00BF00540040801A060065
:106C580073B54FF4961306460D461446019304E0A7
:106C6800019B5A1E0192002B57D031484FF4003136
:106C780006F0B6F80028F3D12D48012105F0A4FF4D
:106C88004FF48053019304E0019B5A1E0192002B9C
:106C980045D02748274906F08EF80028F4D0244824
:106CA8003146002205F0A8FF4FF48053019304E019
:106CB800019B5A1E0192002B33D01D481E4906F035
:106CC8007AF80028F4D01A48294606F018F84FF444
:106CD8008053019303E0019B5A1E01921BB3144891
:106CE800164906F068F80028F5D01148214606F044
:106CF80006F84FF49613019303E0019B5A1E019284
:106D08009BB10B480E4906F06BF80028F5D00848EF
:106D1800012105F065FF002008E0012006E00220BF
:106D280004E0032002E0042000E005207CBD00BF51
:106D380000540040010003008200070080000700A3
:106D48000400001037B54FF4961304460D4601931E
:106D580005E0019B5A1E0192002B00F09B805648CB
:106D68004FF4003106F03CF80028F2D152480121D6
:106D780005F02AFF4FF48053019305E0019B5A1E4A
:106D88000192002B00F088804B484C4906F013F81C
:106D98000028F3D048482146002205F02DFF4FF483
:106DA8008053019304E0019B5A1E0192002B75D079
:106DB8004148434905F0FFFF0028F4D03E482946E2
:106DC80005F09DFF4FF48053019304E0019B5A1E88
:106DD8000192002B64D038483A4906F001F800289F
:106DE800F4D03548012105F0EFFE4FF480530193AC
:106DF80004E0019B5A1E0192002B53D02E482F49C4
:106E080005F0D9FF0028F4D02B482146012205F0CF
:106E1800F3FE4FF48053019304E0019B5A1E019244
:106E2800002B41D0244C2849204605F0D9FF0028E2
:106E3800F3D02046002105F0E7FE20460121238BF0
:106E480005F0CEFE4FF48053019304E0019B5A1ED7
:106E58000192002B2AD018481C4905F0C1FF0028D0
:106E6800F4D0154805F04DFF4FF480530193124AB2
:106E780003E0019B591E0191D3B113889B05F8D4F7
:106E8800012104460C4805F0BFFE0B48104905F0E7
:106E9800C1FF0EE001240CE002240AE0032408E00C
:106EA800042406E0052404E0062402E0072400E0A8
:106EB800082420463EBD00BF0054004001000300E6
:106EC80082000700040000100200001040000010BB
:106ED8000004001013B54FF496130446019305E01F
:106EE800019B5A1E0192002B00F0B08061484FF4BC
:106EF800003105F075FF0028F2D15E48012105F048
:106F080063FE4FF48053019305E0019B5A1E0192E2
:106F1800002B00F09D805748574905F04CFF00288A
:106F2800F3D05448A021002205F066FE4FF48053A8
:106F3800019305E0019B5A1E0192002B00F08A8004
:106F48004C484E4905F037FF0028F3D0C4F305211B
:106F5800484805F0D4FE4FF48053019304E0019BA8
:106F68005A1E0192002B77D04248454905F038FF58
:106F78000028F4D0E1B23F4805F0C1FE4FF4805339
:106F8800019304E0019B5A1E0192002B66D03948F8
:106F98003B4905F025FF0028F4D03648012105F0CB
:106FA80013FE4FF48053019304E0019B5A1E019293
:106FB800002B55D02F48304905F0FDFE0028F4D0AD
:106FC8002C48A121012205F017FE4FF480530193AC
:106FD80004E0019B5A1E0192002B43D0254C2949FD
:106FE800204605F0FDFE0028F3D02046002105F0DC
:106FF8000BFE20460121238B05F0F2FD4FF4805350
:10700800019304E0019B5A1E0192002B2CD01948D1
:107018001D4905F0E5FE0028F4D0164805F071FE7C
:107028004FF480530193134A03E0019B591E0191C9
:10703800E3B113889905F8D4012104460D4805F0F9
:10704800E3FD0C48114905F0E5FE10E001240EE0CF
:1070580002240CE003240AE0042408E0052406E0E6
:10706800062404E0072402E0082400E0092420465E
:107078001CBD00BF0054004001000300820007004F
:10708800040000100200001040000010000400106E
:1070980082B0002304E0019B01330193009B01337C
:1070A8000093009B8342F6D302B0704737B54FF484
:1070B800805304460D46019304E0019B5A1E019239
:1070C800002B6ED03D484FF4003105F089FE0028B2
:1070D800F3D13A48012105F077FD4FF4805301932D
:1070E80004E0019B5A1E0192002B5CD033483449BE
:1070F80005F061FE0028F4D03048A021002205F0F8
:107108007BFD4FF48053019304E0019B5A1E0192CA
:10711800002B4AD029482B4905F04DFE0028F4D011
:10712800C4F30521254805F0EAFD4FF48053019387
:1071380004E0019B5A1E0192002B38D01F482249B7
:1071480005F039FE0028F4D0E1B21C4805F0D7FD5F
:107158004FF48053019303E0019B5A1E019243B3FD
:107168001648194905F027FE0028F5D01348294686
:1071780005F0C5FD4FF49613019303E0019B5A1ED9
:107188000192C3B10D48114905F02AFE0028F5D037
:107198000A48012105F024FD0D48FFF779FF00207A
:1071A8000AE0012008E0022006E0032004E00420B1
:1071B80002E0052000E006203EBD00BF005400406C
:1071C800010003008200070080000700040000108F
:1071D800A0860100F7B54FF4805304460D461646C5
:1071E800019304E0019B5A1E0192002B75D041487F
:1071F8004FF4003105F0F4FD0028F3D13D4801219A
:1072080005F0E2FC4FF48053019304E0019B5A1E01
:107218000192002B63D03748374905F0CCFD002890
:10722800F4D03448A021002205F0E6FC4FF4805346
:10723800019304E0019B5A1E0192002B51D02D4866
:107248002E4905F0B8FD0028F4D0C4F305212948DB
:1072580005F055FD4FF48053019304E0019B5A1E3D
:107268000192002B3FD02348254905F0A4FD0028B2
:10727800F4D0E1B21F4805F042FD4FF4805301936A
:1072880004E0019B5A1E0192002B2ED019481C497C
:1072980005F091FD0028F4D000244FF4961710E073
:1072A800295D144805F02BFD019703E0019B5A1E48
:1072B8000192E3B10F48134905F092FD0028F5D07B
:1072C8000134E3B2B342EBD30A48012105F088FC4C
:1072D8000D48FFF7DDFE00200AE0012008E002204B
:1072E80006E0032004E0042002E0052000E0062078
:1072F800FEBD00BF005400400100030082000700EB
:107308008000070004000010A086010013B50520C6
:10731800012105F0BDFE184C4FF4E0530093022301
:107328008DF804308DF805302046002369468DF825
:1073380006308DF8073005F003FB20460A210622A7
:1073480005F07EFB20460C21062205F079FB06227B
:1073580020460B21A4F5006405F072FB4FF40043AE
:1073680020466946009305F0EBFA20460F210622D5
:1073780005F066FB1CBD00BF000802401FB50446AF
:10738800FFF7CEF9FFF734FCFFF7F6F9FFF7BEFF7A
:1073980001214FF4004005F09FFE02940F4C10238A
:1073A800ADF80230204600236946ADF80430ADF848
:1073B8000C30ADF80030ADF8063005F0BCFF69467A
:1073C8004FF0402006F08BF82046012106F03BF8EC
:1073D8004FF04020012106F036F81FBD003C004068
:1073E800014B1860704700BFCC0C0020704710B5E7
:1073F8000A4A1379262B04D80949C8540133137152
:1074080010BD074A0123591ED45C0133272B54545D
:10741800F9D1034B83F8260010BD00BFCC0C002027
:10742800543B0020704710B504462078FFF7DFFF73
:1074380014F8013F002BF8D110BD38B504460D46AD
:10744800013D14F8010BEDB2FFF7D1FF002DF7D184
:1074580038BD00BF014B1878704700BFD40C00201E
:10746800014B5878704700BFD40C0020024B1878A5
:1074780080F00100704700BFD40C0020024B0022AE
:107488001A705A70704700BFD40C0020014B0122BB
:107498001A707047D40C0020014B01225A707047B3
:1074A800D40C002082B0002304E0019B0133019337
:1074B800009B01330093009B8342F6D302B07047D0
:1074C80007B50420012105F0E3FD01214FF48040B8
:1074D80005F00EFE4FF40073009300238DF804307E
:1074E8000348012369468DF8073005F029FA0EBDD7
:1074F800000802400D4B07B51A680D484FF47A731F
:10750800B2FBF3F20B4B013A5A600B4AF02182F8B6
:10751800231000229A6007221A60084B084A009339
:107528000121084B03F03AFF0EBD00BF9C0100206B
:10753800283C002010E000E000ED00E0B802002048
:107548009C02002004020020054B1A6812B11A6838
:10755800013A1A60034B1A6801321A60704700BF7B
:10756800DC3B0020F43B002082B0044B0190019AE0
:107578001A601A68002AFCD102B07047DC3B002070
:10758800704700BF40F0BE60024B40F42020D86036
:10759800704700BF00ED00E0C37810B503B3164B89
:1075A8004278DB688478DB43C3F30223C3F1040128
:1075B800C9B202FA01F10F2242FA03F2C9B222401B
:1075C8000A430E4B01781201CB18D2B283F800237C
:1075D80003780122590903F01F0302FA03F307E0B5
:1075E80003780122590903F01F0302FA03F320313B
:1075F800024A42F8213010BD00ED00E000E100E051
:1076080021F0604121F07F01014B084398607047E9
:1076180000ED00E0044B1A6909B1104301E022EAC9
:1076280000001861704700BF00ED00E0044B1A68C5
:1076380004280CBF42F0040222F004021A607047CA
:1076480010E000E000000000034A044B1A60044AFE
:10765800044B1A60704700BF0000FA452418002048
:10766800DB0FC93F20180020034B00221A60034A91
:10767800034B1A60E8E700BF504200200000FA45BB
:107688001C17002007EE100A024BF8EEC77AC3ED6C
:10769800007A70471C17002038B510EE100A07F062
:1076A800A9F80DA3D3E9002307F0F8F8084B04461E
:1076B80018680D4607F09EF80B46024629462046F4
:1076C80007F016FA07F0CCFB024B186038BD00BF74
:1076D8002418002020180020182D4454FB2119409C
:1076E8002DE9F04F2DED068B6F4CDFF8F0A189B036
:1076F8000027A34637F80A506C4B2580FE5A6C4B7E
:107708006680186807F076F865A3D3E9002307F0C8
:10771800C5F807F05DFB6368664AC018011101F5FA
:1077280080610905090D6060C0F30B100DF1200C94
:1077380032F8203032F82120616A238115FB02F0EB
:10774800628115FB03F516FB02F216FB03F60CEB40
:107758004103E0602561C0F3CF30C5F3CF356261E6
:10776800A661C2F3CF32C6F3CF3623F8200C23F834
:10777800105C23F8182C23F8086C4F4BA0830131B8
:107788000B40002BE5832284668403DA013B63F017
:1077980003030133CBF82430002B76D14748484AFD
:1077A8006946042308F06AFB4648474A04A90423AB
:1077B80008F064FB4548464A02A9042308F05EFB2A
:1077C800444A454806A9042308F058FBB4F9283070
:1077D80007EE903AB4F92A30B8EEE79A07EE903AF5
:1077E800B4F92C30B8EEE78A07EE903AB4F92E30A7
:1077F800F8EEE79A07EE903AF8EEE78A68EE087A2C
:1078080049EE097A17EE900A06F0F4FF41EC100BE6
:1078180009F096F951EC100B07F022FB68EEA87AF4
:1078280049EEA97A0AEE100A206317EE900A06F0CC
:10783800E1FF41EC100B09F083F951EC100B07F054
:107848000FFB68EE897A58EE297A28EE288A0AEE24
:10785800900A606309EE298A17EE900A06F0CAFFBB
:10786800804618EE100A894606F0C4FF49EC108BD2
:1078780041EC110B09F0DCF88AEE2AAA51EC100B46
:1078880007F0EEFA84ED0FAAA0630237B7F5007F80
:107898007FF430AF09B0BDEC068BBDE8F08F00BFB8
:1078A80039D6C56D305FC440E40C00207019002043
:1078B80020180020FC55040803000080B4000020B4
:1078C8000C0D0020A80000200E0D00209C000020B8
:1078D800100D0020120D00209000002036210020FD
:1078E800014B93ED0F0A7047E40C0020014B93ED18
:1078F8000E0A7047E40C0020014B93ED0C0A704708
:10790800E40C0020014B93ED0D0A7047E40C0020B5
:1079180010B5FEF725F90020012324210246FEF7C1
:1079280089F9114B1C780020012C05D10146FEF77E
:107938005AFA2046002104E00721FEF754FA0120F4
:107948000721FEF750FA63221221C020FFF780F9C1
:1079580002200121FEF747FAFEF724FB0120BDE8CB
:107968001040FEF714BB00BFEC0D00200D4B1B7838
:10797800012B05D10C4B0D4A196812688A181A6038
:107988000B4B1B78012B084B196805D1094A91420A
:1079980007DD01321A607047074A914201DD013262
:1079A8001A607047B43B002020420020B03B002002
:1079B800EC0D00207FD1F008FF1FA1070E4B1B78AC
:1079C800012B05D10D4B0E4A196812688A1A1A60E4
:1079D8000C4B1B78012B094B05D10B4A19689142B6
:1079E80008DC1A6070471A68B2F57A2FDCBF4FF4CA
:1079F8007A221A60704700BFB43B00202042002062
:107A0800B03B0020EC0D002040420F00024B1A68EA
:107A1800024B1A60704700BF143C0020204200202F
:107A28002DE9F04F824658488BB0B0FBF1F00C4678
:107A380006F0BEFE41EC100B08F0F6FE51EC100B00
:107A480007F0EEF9C307074648BF471E04FB07F0D7
:107A580006F0AEFE46A3D3E9002307F049F8044632
:107A68000D4645EC104B08F0DFFE59EC108B204614
:107A780042464B46294606F05DFDCDE904014946DC
:107A8800404607F0CDF93CA3D3E900230990DDE98E
:107A9800040107F07FF900283DD1002401234FF0AD
:107AA8001509224698462046DFF8E4B003E023464D
:107AB80042462C46B04600FB04355D452ED800FBF7
:107AC8000826DDE904012EA3D3E9002307F062F9B3
:107AD80030BBDDE9042300202C4907F009F841EC0C
:107AE800100B0390029108F09FFE0398029953EC43
:107AF800102B8DED060B06F01DFD09F1FF39CDE9C0
:107B080004015FFA89F9DDE9060107F089F9B9F19D
:107B1800000FCCD104E00125002601E025464646A9
:107B2800099BD9B2BAF1000F0BD132462B46504609
:107B3800FEF780F801230093504651463A465346D3
:107B480009E032462B460120FEF774F80120009028
:107B580001463A460023FEF760F9FEF723FA0120B2
:107B68000BB0BDE8F04FFEF712BA00BFAFF30080CC
:107B78000000000084D77741956479E17FFDA53D39
:107B8800BBBDD7D9DF7CDB3D00E9A4350000F03F61
:107B9800FFFF0F001F4B1B78022B10B539D01E4B6F
:107BA8001E4A19681E4B1F4C1B68CB189342236052
:107BB80018DC0020FFF734FF01202168FFF730FFB1
:107BC800194B1C780020012C05D10146FEF70BF952
:107BD8002046002104E00721FEF705F901200721CE
:107BE800FEF701F9114B1B78022B12D10A4C104BEE
:107BF80022681B689A420CDA0E4B1B78012B08D1BD
:107C08000D4B186800F070F80C4B22681B68D318ED
:107C1800236010BDA44300202042002080D1F0083A
:107C28003C42002040420020EC0D0020B43B0020E4
:107C3800043C0020FC3B0020CC3B0020B03B002053
:107C480008B5FEF71FFD094B5A78187002435A70A1
:107C58001AB19A7801329A7030B99B78034A012B8D
:107C680002D900235370937008BD00BF240D002073
:107C780007B50420012105F00BFA4FF46043009387
:107C880001238DF8043002238DF8053004480023C1
:107C980069468DF806308DF8073004F051FE0EBDA8
:107CA80000080240084B1A684FF47A73B2FBF3F2EB
:107CB800064B013A5A60064AF02182F82310002246
:107CC8009A6007221A6070479C01002010E000E0CB
:107CD80000ED00E0034B5A6812B15A68013A5A6045
:107CE800704700BF240D0020024B58605A68002AD4
:107CF800FCD17047240D002030B585B004460D46F0
:107D080001A85C490A220BF0ABF95B4B1B78032BEB
:107D180010D8DFE803F00205080B01A8574907E06F
:107D280001A8574904E001A8564901E0564901A8AD
:107D38000BF080FA04AA131913F80C3C5D19EDB284
:107D48002F2D01D80A3502E0392D01D90A3DEDB2AF
:107D580004AB1C194FF6FF7004F80C5CFCF76CFEC2
:107D68000020FCF75FFF0DF103050F2420462334A4
:107D78005A21002315F8012FA4B2FCF76DFFB4F5C2
:107D8800A57FF3D164205A212C220023FCF764FF3D
:107D98000023CD205A212C22FCF75EFF0020FCF79F
:107DA8004BFE354B1B78032B62D8DFE803F0022823
:107DB8004B5601A931480BF03DFA0A2200212F4801
:107DC8000BF0DCFB314A324B12781860012A06D1DD
:107DD800304A904201DC01321A602F4A06E0B0F5C1
:107DE800FA5FBCBF4FF4FA521A602C4A1B689342E0
:107DF800C4BF274B1A602A4B1A682A4B20E001A9F6
:107E08001F480BF017FA0A2200211D480BF0B6FB99
:107E18001E4A254B12781860012A06D11D4A904245
:107E280001DC01321A601C4A06E0B0F5FA5FBCBFFB
:107E38004FF4FA521A60194A1B68934218DD1A4B1C
:107E48001A6015E001A90F480BF0F4F90D4800215C
:107E58000A220BF093FB154B09E001A90A480BF025
:107E6800E9F9094800210A220BF088FB104B186039
:107E780005B030BD47990508123C0020E03B0020C2
:107E8800083C002025420020D03B0020EC0D0020BB
:107E9800243C00203F420F0080D1F00840420F00F0
:107EA800143C0020204200204442002018420020B8
:107EB800CC3B002010B50D4B0D4C1A680D482146DF
:107EC8000BF090F90C4B0D481A6821460BF08AF913
:107ED8000B4B0C481A6821460BF084F90A4B0B48E7
:107EE8001A682146BDE810400BF07CB9243C0020FC
:107EF80051990508E03B002044420020083C00203E
:107F08001842002025420020CC3B0020D03B002016
:107F180008B500210A220D480BF030FB0C4B00215C
:107F280018600A220B480BF029FB0B4B0021186044
:107F38000A220A480BF022FB094B002118600A228A
:107F480008480BF01BFB084B186008BDE03B0020FD
:107F5800243C0020083C0020444200202542002008
:107F680018420020D03B0020CC3B00209FED010AA6
:107F7800704700BF000000009FED010A704700BF76
:107F880000000000014B93ED020A7047240D002009
:107F9800054B83ED000AC3ED010A83ED021AC3ED18
:107FA800031A83ED042A70477CC50020054B83ED36
:107FB800050AC3ED060A83ED071AC3ED081A83ED17
:107FC800092A70477CC50020044B18B1012801D14B
:107FD800034A00E0034A12681A60704720420020F2
:107FE800043C0020143C002010B9034B186870476B
:107FF800024B1868704700BF243C0020143C002046
:1080080010B9034B18687047024B1868704700BFD7
:1080180044420020043C002008B54FF49570FEF758
:1080280067FA40F26523C31A584240EB030008BDC3
:1080380008B5C620FEF75CFA40F28D13C21A50420A
:1080480040EB020008BD4FF4957040F26521FEF741
:1080580041BAC62040F28D11FEF73CBA08B500209F
:10806800F8F7C2FBBCEEC00A4FF4967010EE101A77
:10807800FEF74DFA0020F8F7C5FBBCEEC00A4FF436
:10808800987010EE101AFEF742FA0020F8F7C8FBB5
:10809800BCEEC00A4FF49A7010EE101AFEF737FAC9
:1080A8000020F8F7CBFBBCEEC00A4FF49C7010EE32
:1080B800101AFEF72CFA0020F8F7CEFBBCEEC00A27
:1080C8004FF49E7010EE101AFEF721FA0120F8F70F
:1080D8008BFBBCEEC00A4FF4A07010EE101AFEF72E
:1080E80016FA0120F8F78EFBBCEEC00A4FF4A27016
:1080F80010EE101AFEF70BFA0120F8F791FBBCEE10
:10810800C00A4FF4A47010EE101AFEF700FA01200E
:10811800F8F794FBBCEEC00A4FF4A67010EE101AE4
:10812800FEF7F5F90120F8F797FBBCEEC00A4FF40B
:10813800A87010EE101ABDE80840FEF7E8B92DE95E
:10814800F04F85B0FFF768FF002875D04FF49670A0
:10815800FEF7F6F9604ADFF8B4B110604FF4987092
:108168000192FEF7EDF95D4BDFF8A4A118604FF41A
:108178009A700293FEF7E4F9CBF800004FF49C7074
:10818800FEF7DEF9CAF800004FF49E70FEF7D8F942
:10819800DFF88091DFF88081C9F800004FF4A07003
:1081A800FEF7CEF9C8F800004FF4A270FEF7C8F940
:1081B8004B4F4C4E38604FF4A470FEF7C1F9306055
:1081C8004FF4A670FEF7BCF9474D484C28604FF4B1
:1081D800A870FEF7B5F920604FF4AA70FEF7B0F961
:1081E800434908604FF4AC700391FEF7A9F984463F
:1081F8004048C0F800C0029B3F481B68019A0361D1
:10820800DBF8003003994361DAF8003012688361C3
:10821800D9F80030C260C361D8F80030C0F838C05F
:1082280003623B684362336883622B68C3622368D6
:1082380003630B6843630EE02F4B304C30483149E1
:10824800DC6000221A6158619A61D9611C625A6225
:108258009862DA621963284A2B4BD2ED033AD2EDC1
:10826800044AD2ED055AD2ED066AD2ED077A92EDAC
:10827800083A92ED094A92ED0A5A92ED0B6A92ED8C
:108288000C7AC3ED003AC3ED014AC3ED025AC3EDBF
:10829800036AC3ED047A73EE633A74EE644A75EECA
:1082A800655A76EE666A77EE677A83ED053A83ED6E
:1082B800064A83ED075A83ED086A83ED097AC3ED10
:1082C8000A3AC3ED0B4AC3ED0C5AC3ED0D6AC3ED70
:1082D8000E7A05B0BDE8F08F080E0020100E0020C1
:1082E800280E0020200E0020F00D0020F40D0020A4
:1082F8002C0E0020FC0D0020240D00200000F04270
:1083080000008CC2CCBC8C2C7CC50020240E002024
:108318000C0E00201C0E0020180E002060EEA00A93
:10832800B7EE007AF0EE606A70EE077A40EE006A07
:1083380047EEA70A36EEC77A08B5C7EE200A10EE50
:10834800900A06F057FA0022084B06F0A7FA002216
:10835800074B06F0F1F806F083FD07EE900AFDEEF4
:10836800E77A17EE900A9F3008BD00BF0000594019
:108378000000E03F38B52DED028BF7EE008AB0EE35
:10838800608A70EE288A10EE900A28EE088A06F0B5
:1083980031FA08EEA88A00220F4B06F07FFA04464D
:1083A80018EE100A0D4606F025FA02460B4620463E
:1083B800294606F09DFB0022084B06F0BDF806F0A2
:1083C8004FFD07EE900AFDEEE77A17EE900A773038
:1083D800BDEC028B38BD00BF000069400000E03FE3
:1083E800F0B5694D2DED068B95E80F008DB008AE00
:1083F800103586E80F000FCD01AC0FC495E80700D3
:108408004FF6FF7384E807009F2077216422FAF76C
:10841800A2F9A020772164224FF6FF73FAF79BF99F
:108428009E20772164224FF6FF73FAF794F99F2074
:10843800762164224FF6FF73FAF78DF94FF6FF7332
:10844800782164229F20FAF786F90020FCF750F97A
:108458009F2077216522FCF725FB9F207721642246
:10846800FCF720FB07AD0C36F7EE009A0435F7EE63
:10847800008A95ED009A4FF49674B0EE68AA18EE4B
:10848800900A06F0B7F93EA3D3E9002306F006FAEE
:1084980006F0E6FC08EE900A38EEE98AB0EE490AE2
:1084A800F0EE480AFFF73AFFB0EE490AF0EE480A44
:1084B8000746FFF75FFFBFB281B20F223846FCF7CD
:1084C80024F8013CDBD14FF49674F7EE008A18EEDD
:1084D800900A06F08FF92AA3D3E9002306F0DEF903
:1084E80006F0BEFC08EE900A39EEE88AB0EE490ABA
:1084F800F0EE480AFFF712FFB0EE490AF0EE480A1C
:108508000746FFF737FFBFB281B20F223846FBF7A5
:10851800FCFF013CDBD1B542A8D16C4607AE043460
:1085280094ED009A4FF4C875F7EE008A18EE900A99
:1085380006F060F912A3D3E9002306F0AFF906F0BC
:108548008FFC08EE900A38EECA8AF0EE490AB0EEBF
:10855800480AFFF7E3FEB0EE480AF0EE490A07467C
:10856800FFF708FFBFB281B200223846FBF7CDFF04
:10857800013DDBD1B442D2D10DB0BDEC068BF0BDCC
:10858800295C8FC2F528F03FFC950408121A06EE04
:10859800902A081AB8EEE67A06EE900AF8EEE67A1D
:1085A800C7EE277A9FED047A67EE877AFDEEE77AC1
:1085B80017EE900A704700BF0000A0438A1A06EE23
:1085C800902A081AB8EEE67A06EE900AF8EEE67AED
:1085D800C7EE277A9FED047A67EE877AFDEEE77A91
:1085E80017EE900A704700BF0000484370B5064672
:1085F8000D460024610704D5A0B231462A46FBF790
:1086080084FF0134B4F5A07FF4D170BD70B506467F
:108618000D460024600704D5A1B230462A46FBF770
:1086280074FF0134C82CF5D170BD114B11481B786B
:108638001149124A0068012B114B09D112680860D0
:108648001A60104B1A68104B1A60104B1A680CE02D
:108658001268D2011A600B4B1A680B4BD2011A60D0
:108668000A4B1A68C0010860D201094B1A607047AA
:10867800EC0D0020243C0020143C00204442002043
:10868800043C002018420020B03B0020EC3B0020B6
:108698003C420020024B1A68024B1A60704700BF28
:1086A800143C00202042002008B5FFF7BEFFBDE8BB
:1086B8000840EFE70022F0B51346202603254FF0C7
:1086C8002C0C00E02646303EF6B217460132092E41
:1086D80010F8014B0AD897FBF5F605FB16772FB96A
:1086E800CE1801F803C07470023301E0CC54013392
:1086F800092AE7D12022CA54CB1848225A707A2274
:108708009A700022DA70F0BD70B58CB005460C4640
:1087180008A80E491E460AF065FD08A86946FFF735
:10872800C9FF6A460A4904A80AF05CFDBDF8400082
:10873800FCF782F93046FCF795F92846214604AA49
:108748000023FCF7A7FA0CB070BD00BF57990508C5
:108758002A9705082DE9F04F084B2DED0A8B1B7859
:10876800022BD5B000F02985054B1A78054B5AB96C
:108778001A68802392FBF3F808E000BFA4430020A6
:10878800EC0D002020420020D3F80080D44CD54DB9
:10879800216CE36BC3EB0802CB1A92FBF3F307EEF1
:1087A800903AB8EEE78AFFF79BF885ED0F0AFFF7D6
:1087B8009DF8D4ED0A7A94ED009AD4ED018A08EE7A
:1087C800279AD4ED0B7A94ED04AA48EE278AD4EDC3
:1087D8000E7A85ED100AE86B08EE27AA10EE109ABB
:1087E80006F008F8064648460F4606F003F841EC3E
:1087F800100B41EC1B0B07F0BFFF304653EC102B5E
:10880800394606F04BF806F02BFBB0EE4B0AF0EEBB
:108818006B0A0AEE900A08F0AFF8304653EC102BBA
:10882800394606F03BF806F01BFB07EE100AD4EDBC
:108838000C6AD4ED027A68EE879A48EE267A59EEE9
:108848002A9A68EEAA8A79EEA79A49EE078AD4EDA1
:10885800037A94ED0D7A48EE077A9FEDA3BA78EE85
:10886800A78ADFEDA2BA68EEA87A49EEA97AF1EEF6
:10887800688AC9EEA79AC8EEA77A29EEA98AC5ED33
:10888800027A17EE900A05F0B5FFCDE904014046DB
:1088980005F09EFF8AA3D3E9002305F0FFFF0446F5
:1088A8001AEE100A0D4605F0A5FF02460B462046B3
:1088B800294605F0F3FF02460B46DDE9040105F001
:1088C80039FE06F0CDFA0AEE100A6AEE0ACAB1EECF
:1088D8004A9A78EE2C7A864B89EE279AC9EEA7AA8F
:1088E800B4EE4B9AF1EE10FAC8BFB0EE4B9AB4EE64
:1088F8006B9AF1EE10FA48BFB0EE6B9AC3ED00AA7E
:1089080083ED019A1AEE900A05F074FF0022794B64
:10891800CDE9020105F00EFE69EE097A044617EE6C
:10892800900A0D4605F066FF224606460F462B467E
:108938002046294605F0B2FF32463B4605F0FCFDCD
:1089480041EC100B08F0FCF80022DDE90201694B4C
:108958005BEC10AB05F0F0FD02460B4605F09EFF00
:1089680032463B4605F0E8FD41EC100B08F0E8F80C
:108978005946504655EC104B06F072FA294608EE57
:10898800900A204606F06CFA07EE900AC8EEA78A0D
:10899800594D5A4CB7EE00CA18EE900A05F02AFF56
:1089A80049A3D3E9002306F0EBF9DFED557A002857
:1089B80018BFF0EE678AF4EE4C8ADFED527AF1EEDA
:1089C80010FAC8BFF0EE678ADFED4F7A6AEE277AB1
:1089D800C5ED008A17EE900A05F00CFFDFED4B7A23
:1089E80037EEC88A0F4678EE6CCA0646C4E90267B5
:1089F8001CEE900A05F0FEFE47EC106B41EC110BE3
:108A0800C4E9000108F014F838EE8C8A3CEE68CA14
:108A180051EC100B88EE0C8A06F022FA3C4B1B78BE
:108A280080F00047B4EE4B8AF1EE10FAC8BFB0EE02
:108A38004B8AB4EE6B8AF1EE10FA48BFB0EE6B8A3F
:108A4800022B6F6076D1334D2C68002C72DB18EE48
:108A5800900A05F0CFFE00222F4B05F01FFF06F00D
:108A6800DFF906468146384605F0C4FE18A3D3E967
:108A7800002305F013FF18A3D3E9002305F05CFDDC
:108A880006F0CEF9254BC3F80080254B03F8348057
:108A980003EBC403C8F307225A70C8F307429A705D
:108AA8001E7198714FEA1862C6F30726C0F30720B3
:108AB800DA705E71D8711B4B1B6801349C4233E03D
:108AC8001F85EB51B81E19402D431CEBE2361A3FA7
:108AD800CDCCCCCC0C5FC44000000000C0FFDF4010
:108AE8007CC50020240D0020003C1C46003C1CC610
:108AF8009C43002000004940804200205845002047
:108B080017B7D13872F97F3F0AD7233D17B7D13944
:108B1800B43B00201C3C00200000F040944300209F
:108B28006C450020183C0020C8BF4FF0FF332C6074
:108B3800C8BF2B60FEF7E0FE7C4C84ED110AFEF7FF
:108B4800E1FE84ED120AFDF791FC4246E0647849A3
:108B580044A80AF047FB606C05F04CFE02460B4641
:108B680034A874490AF03EFBA06C05F043FE0246A7
:108B78000B4638A870490AF035FB19EE900A05F043
:108B880039FE82468B4652466C495B463CA80AF041
:108B980029FB6B49DDE9042340A80AF023FBDDE942
:108BA8000223684920A80AF01DFB19EE100A05F0F7
:108BB80021FECDE90801DDE90823634924A80AF06C
:108BC80011FB18EE900A05F015FECDE90601DDE966
:108BD80006235E4928A80AF005FB384605F00AFE78
:108BE80006460F4632463B4659492CA80AF0FAFA7F
:108BF80018EE100A05F0FEFDCDE90A01DDE90A23A9
:108C0800544930A80AF0EEFA1CA85349E26C0AF05D
:108C1800E9FA524B1B78013BDBB2012B00F29A8236
:108C28004F4B1B78072B00F29582DFE813F0080002
:108C38009302A3002A016D01C901630229020220DF
:108C4800FBF7F0FF4FF6FF70FBF70CFF1F20FBF759
:108C5800F3FE19210023434A2D20FCF71BF84FF699
:108C6800FF70FBF7FFFE00200024FBF7E5FE0F2056
:108C7800B42142464FF6FF730094FFF745FD0F20DD
:108C8800772134AA2346FCF705F8A020772138AAD3
:108C98002346FBF7FFFF0F20412128AA2346FBF7B5
:108CA800F9FFA02041212CAA2346FBF7F3FF0F2050
:108CB80065213CAA2346FBF7EDFF40AA2346A020E6
:108CC8006521FBF7E7FF0F20532120AA2346FBF776
:108CD800E1FFA020532124AA2346FBF7DBFF0F2046
:108CE8009B2130AA2346FBF7D5FF104BDB6CB3F56D
:108CF8007A7FCCBF4FF4FC604FF47840FBF7B2FEAC
:108D08001CAAA0209B210023FBF7C4FF164B1B784D
:108D18000221012B0CBF154A154A4FF48C70002311
:108D2800FBF7B8FF1F20FBF79DFE13E2240D002080
:108D38005C99050866990508719905087C990508E4
:108D480086990508909905089B990508A69905082C
:108D5800B1990508BC990508C8990508B43B0020D5
:108D680038420020D5990508EC0D0020F499050833
:108D7800F899050852465B464EA8B3490AF032FAFC
:108D8800DDE9042351A8B1490AF02CFADDE90223F0
:108D980048A8AF490AF026FADDE908234BA8AD49EF
:108DA8000AF020FAE62002214EAA0023FBF772FF00
:108DB800E620162151AA0023FBF76CFF0220C821E8
:108DC80048AA0023FBF766FF4BAA00230220DC21F8
:108DD800FBF760FFDFEDA07A68EEA78A4FF6E07533
:108DE80018EE900A05F006FD47EC106BCDE902017C
:108DF80007F0C2FC5BEC10AB47EC106B07F0BCFD56
:108E0800002057EC106BFBF72DFE0A214246002389
:108E180005200095FFF778FC4FF47840FBF70CFE2F
:108E2800DDE9020152465B4605F038FD78A3D3E937
:108E3800002305F081FB05F0CBFF324684B23B46A8
:108E4800DDE9020105F02AFD02460B4672A1D1E9CF
:108E5800000105F06FFB05F0BBFF81B22046F9F772
:108E6800AAFC9D20772105220023FBF715FE9F20F1
:108E7800752105220123FBF70FFE2846FBF7DCFDD1
:108E880068E1764B1868764B42461968FFF77EFB17
:108E9800B0F59F7F044602DD724B02221A709FEDE7
:108EA800728AF4EEC8AAF1EE10FA14D5F5EEC0AA4B
:108EB800F1EE10FA0FDDFDEEEAAA4FF4FA711AEEA0
:108EC800902A0020FFF77AFBA3B281B24FF6FF7217
:108ED8001846FBF71AFBB4EEC89AF1EE10FA40F107
:108EE8003981DFED627AB4EEE79AF1EE10FA40F3D9
:108EF8003181BDEEC99A5E4819EE102A4FF4FA7115
:108F0800FFF75CFBA4B2F0E0544B1868544B4246A0
:108F18001968FFF73BFBB0F59F7F064602DD514B12
:108F280002221A70F5EEC09AF1EE10FA1DDD5046D5
:108F380059463BA3D3E9002305F022FFA8B13AA381
:108F4800D3E900235046594605F0A8FC02460B46D3
:108F58000020484905F0EEFA05F03AFFB4B281B2B4
:108F68004FF6FF722046FBF7D0FA1AEE100A05F00A
:108F780041FC2FA3D3E9002304460D4605F01EFF4C
:108F8800002800F0E7802046294625A3D3E90023DE
:108F980005F0F6FE002800F0DD8027A3D3E90023C2
:108FA8002046294605F07AFC02460B460020324945
:108FB80005F0C0FA05F00CFFB6B281B2304696E073
:108FC800264B1868264B42461968FFF7DFFAB0F5BA
:108FD8009F7F044602DD234B02221A70DDE9060159
:108FE80017A3D3E9002305F0E9FE68B19DED060B50
:108FF80007F020FD002251EC100B204B05F04EFC31
:1090080005F0E6FE014600E0C821A0B289B29DE065
:109018000000000000E063400000000000C05D4068
:109028009A9999999999B93F0000000000409F408A
:109038009A9999999999B9BF0000000000408F400A
:1090480089B5F81400E3693FFC990508069A0508F4
:10905800109A05081A9A05080000C842243C002006
:1090680044420020A44300200000FA430000FAC351
:109078000CFEFFFF0000694000005940000054C08A
:109088005DA3D3E900233046394605F007FC5CA30D
:10909800D3E9002305F02CFD05F0E2FE4A4B08EE6B
:1090A800100A1868494B42461968FFF76FFAB0F57D
:1090B8009F7F02DD464B02221A70DFED467A48EEAA
:1090C800E77A84B2FDEEE77A204617EE901A4FF65B
:1090D800FF7289B2FBF719FABDEEC88A6FF0B300C8
:1090E80018EE102AB421FFF769FA81B220464FF42E
:1090F800FC622DE0DFED387AB4EEE78AF1EE10FA83
:1091080028D5314B1868314B42461968FFF73EFAAB
:10911800B0F59F7F044602DD2D4B02221A709DEDAB
:109128000A0B07F087FC53EC102B10461946002257
:109138002A4B05F0B3FB02460B460020284905F0F0
:10914800F9F905F045FEA4B281B220464FF6FF7248
:10915800FBF7DBF9234B1B78022B09D043B14FF601
:10916800FF7300930520DC2142460023FFF7CCFA69
:10917800174B1B78022B20D119E0A00180B20023E5
:109188000CA92A18D75CCF5401339BB23F2BF9D9CD
:10919800154A1380154B188000F5806080B2402274
:1091A800FEF718F800B1FEE70134A4B202E0104E51
:1091B800104D002433689C42DFDB55B0BDEC0A8BB0
:1091C800BDE8F08FAFF30080243C0020444200202B
:1091D800A4430020000048430000C8420000594052
:1091E8000000694038420020803B00209043002066
:1091F800304200206C4500200000000000807640CE
:109208001F85EB51B81E19402DE9F04F764B2DED17
:10921800048B93ED008A78EE087A83B017EE900AF3
:1092280005F0E8FA714B064618680F4605F0E2FAB1
:1092380068EE088A82468B46F7EE009A4BEC10AB34
:1092480007F09AFA78EEA97A55EC104B17EE900AC7
:1092580005F0D0FA22462B468046894630463946E4
:1092680005F01CFB02460B464046494605F062F9EC
:1092780005F0F6FD79EEE88A09EE100AC8EE898A4B
:10928800DFED5B7A4BEC10AB68EEA78A07F074FB56
:10929800304653EC102B394605F000FB044619EE16
:1092A800100A0D4605F0A6FA02460B462046294646
:1092B80005F01EFC4F4B002205F0F0FA05F0D0FD3A
:1092C8004D4B1B78033B09EE100A042B78D8DFE8D6
:1092D80003F003122F58460018EE900A05F08AFA98
:1092E800044619EE100A0D4605F084FACDE900018E
:1092F8004248434917E029EE098A08EEA88AB1EEE8
:10930800499AC8EE888A89EE088A18EE900A05F00C
:1093180071FA044618EE100A0D4605F06BFACDE90D
:1093280000013648374922462B4609F05BFF47E0E3
:1093380018EE100A05F05EFA41EC100B07F07AFB04
:109348000022314B51EC100B05F0A8FA05F088FD0E
:1093580005F050FA02460B4628482C492EE018EE34
:10936800100A05F047FA1CA3D3E9002304460D466A
:109378005046594605F092FACDE900011F482449A4
:10938800D1E718EE100A05F035FA15A3D3E9002342
:1093980005F014FDDFED1F7A002818BFB0EE678ACC
:1093A80078EE297A79EEC89AC7EEA99A19EE900A4A
:1093B80005F020FA02460B461048174909F012FF3B
:1093C8000E4A0220CA21002303B0BDEC048BBDE87D
:1093D800F04FFBF75FBC00BFF6285C8FC2A54C407E
:1093E800AE47E17A14AEEF3F884200208C4200205D
:1093F8000000484200004940384200205A420020FC
:10940800249A0508349A0508000034C0449A0508CF
:10941800569A0508A4707D3F729A050873B50546EB
:10942800002800F0AE805A4B18884519ADB22AB210
:10943800002A05DB40F23F139A42C8BF1D4600E0F0
:1094480000250121FAF7C0FF0120FAF711FE514E5D
:109458000024A05B0234FAF759FEB4F5C67FF8D1B0
:10946800A8B2C72201214EF29C73FBF7C3F9484BFF
:109478001D80494B1C68494B2DB21B6806EE905A5B
:109488001B1BB8EEE67A06EE903AF8EEE67A67EE3F
:10949800277A17EE900A05F0ADF90022404B05F047
:1094A80027FB05F095FC4FF6FF7324180093052061
:1094B800DC2122460023FFF727F93A4B3A4A1E6877
:1094C8003A49002003460DE015780D7055784D7027
:1094D80095788D70D578CD700D680832A54203D285
:1094E80028460133B342EFDB304A11684018B4EB29
:1094F800500F0CD2013B2C4911F8330001EBC3018A
:109508001070487850708878C9789070D170264A61
:10951800274C284D02EBC3030022197961F3070297
:10952800597961F30F2292B29979DB7907EE902A83
:10953800002261F3070263F30F2293B2B8EE677A51
:10954800A3F5FE43DFED1C7AFF3B67EE277A06EEB4
:10955800903AC4ED007AF8EEE67A17EE900A05F034
:1095680049F909A3D3E9002305F0C2FA05F078FC0C
:10957800124B28601A782046294602B0BDE8704090
:1095880042E602B070BD00BFCDCCCCCC0C5FC4406D
:1095980058420020A6430020243C002044420020DA
:1095A80000007440183C00206C45002094430020C3
:1095B800884200208C42002000008037384200207A
:1095C80013B5104CB4F85030ADF80630BDF806307D
:1095D8009BB25BB1BDF806004EF29C7380B20121CC
:1095E800C722FBF707F90023A4F85030064B1B7875
:1095F800022B06D1054C94F90000FFF70FFF00235A
:1096080023701CBD240D0020A4430020502B0020F3
:10961800474B1A68474B1B68D31A474A126893FB93
:10962800F2F307EE103AF8EEC77A2DE9F043FCEEB4
:10963800E77A424B17EE908A1B681FFA88F898451C
:109648008DB0C8BF1FFA83F84FF480654FF000094A
:1096580060E02846FDF73EFC60F30704681C80B212
:10966800FDF738FC60F30F24A81C80B2FDF732FC2C
:1096780060F31744E81C80B2FDF72CFC60F31F640C
:10968800281D80B2FDF726FC60F30707681D80B22D
:10969800FDF720FC60F30F27A81D80B2FDF71AFC28
:1096A80060F30706E81D80B2FDF714FC60F30F268F
:1096B800B8B205F08DF80022214B05F0EFF805F05F
:1096C800CFFB05F097F8CDE90001B0B205F080F8BE
:1096D80013A3D3E9002304F02DFF13A3D3E9002338
:1096E80005F006FA05F0BCFB05F084F82246CDE942
:1096F8000201144905A809F075FDC1B205A801F0D9
:10970800F7FC0120FEF7F0FA09F1010908351FFA04
:1097180089F9ADB2C1459CD10DB0BDE8F08300BF59
:1097280000000000C0FFDF40E17A14AE47C1664088
:1097380044420020243C002018420020183C00200D
:109748000000F03E7D9A050808B50021C620FCF708
:10975800C1FE4FF495700021BDE80840FCF7BABE81
:10976800024B4FF6FF721A80704700BF5842002024
:1097780000200146C8224FF4A073FBF720B807B5B4
:109788000DF1070001F0B5FC9DF807000EBD08B506
:10979800FFF7F5FF0028FBD108BD30B5044687B0B8
:1097A80010EE100A0D4605F025F802460B4601A8F2
:1097B800054909F017FD2046294601AA0023FBF7B1
:1097C80069FA07B030BD00BF909A050808B5084887
:1097D80002F018FB0648022102F0E5FB0028F9D048
:1097E800034802F03BFB07EE900AB8EE670A08BD93
:1097F8000020014010B50C4C00232DED028B238076
:109808009FED0A8A06E0FFF7E1FF238838EE008A19
:10981800013323802388182BF5D99FED050A28EEFC
:10982800000ABDEC028B10BD803B00200000000048
:10983800ACC8683910B54FF4C770FCF759FEDB287F
:1098480005D14FF4C870FCF753FE044619E041F205
:10985800E104214644F20100FCF73CFE44F2010019
:10986800FCF746FEA04214BF80244FF4007421B2D6
:109878004FF4C870FCF72EFE4FF4C770DB21FCF7DD
:1098880029FE204610BD00BF7047FEE7FEE7FEE751
:10989800FEE7704770477047FEF71CBA10B5094CD1
:1098A800A37A4BB1084B1A6822F006021A6000F03E
:1098B80013F8204600F04FFE4FF48020BDE810401A
:1098C80002F09ABD283C002010ED00E0014801F0AC
:1098D80011B800BF283C0020364BD3F8882042F44A
:1098E8007002C3F88820344B1A6842F001021A60EB
:1098F80000229A60196821F0847121F4803119607E
:109908002E495960196882B021F480211960DA6003
:10991800009201921A6842F480321A601A6802F4BE
:1099280000320192009A01320092019A1AB9009A03
:10993800B2F5A06FF2D1204B1B6813F4003318BFA7
:1099480001230193019B012B2ED11B4B1A6C42F072
:1099580080521A641A4A116841F4804111609A6869
:109968009A609A6842F400429A609A6842F4A05257
:109978009A60144A5A601A6842F080721A6019682C
:109988000D4A8901FBD5104B40F2056119609368B7
:1099980023F003039360936843F002039360936892
:1099A80003F00C03082BFAD1024B4FF000629A60C7
:1099B80002B0704700ED00E000380240103000248B
:1099C8000070004008544007003C0240184B194AF8
:1099D800996801F00C01042903D0082903D0164B1B
:1099E80019E0164B17E059685A6811F4800F596846
:1099F80014BF124B104B02F03F02B3FBF2F30C4AB8
:109A08005268C2F30142C1F38811013252004B433C
:109A1800B3FBF2F3074A1360054B9A68054BC2F390
:109A280003129A181968127921FA02F21A6070471B
:109A3800003802409C0100200024F40000127A0043
:109A480037B51C230124002501A88DF804308DF8B2
:109A580005508DF806408DF80740FDF79DFD20461E
:109A6800214603F039FB09494CF24F334B6053232D
:109A78000B800D814D804FF0804003F0D5FE4FF0F4
:109A880080402146224604F094FA3EBDC4C5002019
:109A980010B54FF08040012104F0A0FA00281DD035
:109AA80001214FF080400E4C04F0A3FA00214FF042
:109AB800804003F04EFF2378022B07D0032B09D0F8
:109AC800012B0BD1BDE81040F6F722BFBDE81040CE
:109AD800F6F7F8BEF7F74AFA0023237010BD00BF67
:109AE800E00C002008B5402002F078FC30B1FBF70C
:109AF8002FFA4020BDE8084002F07EBC08BD0000F7
:109B0800014608B5044804F033FC0348402104F03A
:109B1800DCFC0028F9D008BD00440040F0B589B04D
:109B28004FF4E1330120019300232B4CADF80830AA
:109B38001E460146ADF80A30ADF80C30ADF81030CD
:109B48000C23ADF80E3003F0A3FA4FF400300121D6
:109B580003F0C2FA20680221072202F071FF0722EF
:109B68006068032102F06CFF0125022704232068A6
:109B7800059305A98DF81A608DF81B508DF818709B
:109B88008DF8197002F0DCFE08236068059305A9BA
:109B98008DF8187002F0D4FEA06801A904F03EFB0D
:109BA8002A4640F225510D4804F076FC262307A8E2
:109BB8008DF81C308DF81D608DF81E608DF81F50D3
:109BC800FDF7EAFCA068294604F0A5FB044A054B0A
:109BD8001A6009B0F0BD00BFB00100200044004089
:109BE800099B000830CF0020024B9868002104F040
:109BF80092BB00BFB001002010B5094C40F22551BE
:109C0800204604F06CFC50B1A288D2B2112A02D1CD
:109C1800044B01211970044B19884A401A8010BD61
:109C280000440040D90C0020780D00207047704790
:109C380073B50120014603F02BFA264C4FF4D85394
:109C48000093022303268DF804302046002369463A
:109C58008DF806308DF807308DF8056002F070FE3B
:109C6800204608210A2202F0EBFE204609210A229A
:109C780002F0E6FE20460B210A2202F0E1FE0A224B
:109C880020460C2102F0DCFE01254FF480632046BB
:109C9800694600938DF806508DF807508DF80560D9
:109CA80002F04EFE0A210A46204602F0C9FE294665
:109CB8004FF4804003F01CFA8020294603F0F4F9A1
:109CC8004FF08050294603F043FA284602F094FBEF
:109CD8007CBD00BF0000024007B54FF4C060FDF72F
:109CE80051FC43238DF804300322012301A88DF889
:109CF80005308DF806208DF80730FDF74DFC0EBDB8
:109D0800782358430723B0FBF3F000230133834241
:109D1800FCD970474FF47A735843F1E737B50023FD
:109D2800104C019305460320FFF7EAFFEB681A6918
:109D3800013C019213D0019A002AF4DA019A42F008
:109D480001020192019A1A61064A1969013A0191C0
:109D580002D00199C907F8D40320FFF7D1FF0020EA
:109D68003EBD00BF410D030010B5C47874B900EBC7
:109D7800820003339B10D0F8D000224603E051F84C
:109D8800044C0132046004319A42F8D1002010BD1D
:109D9800033230B59210D0F8D0400B46002003E0D3
:109DA8002568013043F8045C04339042F8D101EB94
:109DB800800030BD0122F0B50023827040220129C5
:109DC800C37082800CD108230370042343704FF4BE
:109DD800A073C38002230372C1724FF0A04309E04D
:109DE80041B90C230370062343704FF4A063C3806A
:109DF8001F4BC17203F500620261C36046780446D6
:109E080001461A46002508E002F5106C02F530629A
:109E18000A65C1F814C001353A460431B54202F169
:109E28002007F1D303F58062426103F58862C0F828
:109E3800CC20067803F5A0650146002203E0C1F8AE
:109E48008C50013220350431B242F8D31946002231
:109E580002E0C4F8CC1001320434B24201F580515A
:109E6800F7D303F56063C0F80C310020F0BD00BFE4
:109E78000000044038B5037AC2680025012B044667
:109E880025D1936B417A65F3104309B143F48013EC
:109E98009363D36823F4800323F0500343F0100343
:109EA8006FF3C3036FF3C7136FF351436FF3D343D8
:109EB800D3602046FFF732FFE378012B3ED105231C
:109EC80063F34405E36845F020059D6036E0D368F8
:109ED80043F04003D360FFF721FF237A627A032B14
:109EE80014BF4FF434134FF43C130AB143F48013F6
:109EF800E26814209363FFF70DFFE268217AD368C4
:109F0800032908BF43F48033D360237A032B15D188
:109F1800156B012363F39B656FF3D7552D2345F02C
:109F2800805563F316451563C820FFF7F3FEE36811
:109F380045F400051D63C820FFF7ECFEE378012B0C
:109F480007D1E3689D68052262F3440545F02005C2
:109F58009D60002038BDC3689A6842F001029A608B
:109F680000207047C3689A6822F001029A600020B6
:109F7800704707B500230193019B43F02003019329
:109F8800019B61F38A130193019BC2681361064B1D
:109F98001169013B019102D001998806F8D4032088
:109FA800FFF7AEFE00200EBD410D030007B50023EC
:109FB8000193019B43F010030193019BC268136155
:109FC800064B1169013B019102D00199C906F8D4E9
:109FD8000320FFF795FE00200EBD00BF410D0300D2
:109FE80008B5C268D36801296FF35D736FF39E7378
:109FF80002D143F0005302E009B943F08043322014
:10A00800D360FFF787FE002008BDC368586900F0D9
:10A0180001007047C3685B6913F0010F14BF00208B
:10A0280001207047C368586900F001007047C36891
:10A038005A69986910407047C3685868704703693F
:10A048001A6861F301021A607047C26800239361BD
:10A058004FF0FF335361536053610B4B9361C378E7
:10A068009169002B14BF4FF400634FF4016343F46C
:10A07800701343F4405343F0080321EA03010B43F0
:10A0880093610020704700BF00080080F8B5D0F841
:10A098000C3100221A60036915461A6865F3CC2250
:10A0A8001A60C37A012B04461BD10321FFF7C7FFAF
:10A0B800E36880214FF4800261F30F0259629A62CB
:10A0C800C02262F30F0561F31F454FF4A072C3F875
:10A0D800045162F30F056FF31F45C3F80851C3F825
:10A0E8000C5110212046FFF744FF2046FFF75EFF82
:10A0F800226900234FF0FF311361204653611E4649
:10A108009161FF25D361214610E082691768C7F382
:10A11800076707F08007FFB2002F14BF4FF0904782
:10A128000027176001331661043095606278934206
:10A13800EBD300231D46FF2010E04A6D1668C6F3D6
:10A14800076606F08006F6B2002E14BF4FF0904660
:10A1580000261660013315610431906062789342DD
:10A16800EBD323691A6942F480721A61E278012AF2
:10A1780004D1054A402161F359421A632046FFF78A
:10A1880064FF0020F8BD00BF0301010003699B685C
:10A19800C3F34103013B022B9ABF024AD05C032060
:10A1A800704700BF4096040810B5036981699C6830
:10A1B8000A68C4F34100022802D06FF30A0202E0E1
:10A1C800032060F30A020A605A6842F480725A60F7
:10A1D800002010BD30B54D780B780022012D00EB22
:10A1E800830405D105FA03F3A46963F30F0205E0BC
:10A1F800012505FA03F3646D63F31F422368C3F373
:10A20800072505F08005EDB26DB98D6865F30A0381
:10A21800CD78C98865F3934361F3995343F080532C
:10A2280043F4004323600369D9690A43DA610020D3
:10A2380030BD30B54D780B780024012D224600EB57
:10A24800830105D105FA03F3896963F30F0205E079
:10A25800012505FA03F3496D63F31F4203696FF3A0
:10A26800CF340C60D96921EA0202DA61002030BDDE
:10A27800F8B54F780B78012F00EB830349D19E691D
:10A288004C69356833692A4664F3120314B967F3D5
:10A29800DC430BE08F68E419013CB4FBF7F7CC789A
:10A2A80067F3DC43012C08BF64F35E733361C37842
:10A2B800012B06D10B780C6900EB83039B695C6169
:10A2C8000CE0CB78012B09D04B693BB103690C78C2
:10A2D8005E6B012707FA04F434435C63CB78012BE7
:10A2E80007D103699B68DB0554BF45F0005245F070
:10A2F80080520B7800EB830342F004429B691A609A
:10A30800CB78012B38D10A788B8AC968FFF72CFDE6
:10A3180032E05E6D4F6935688C6833692A462FB91B
:10A3280064F31203012464F3DC430AE03F19013F9C
:10A33800B7FBF4F7BF05BF0D67F3DC437C4364F359
:10A3480012033361C378012B05D10B780C6900EB3C
:10A3580083035B6D5C61CB78012B06D14B7913B11C
:10A3680045F0005201E045F080520B7800EB830085
:10A3780042F00442436D1A600020F8BD73B54D7871
:10A38800012D3DD183694A691E681C690094E4B2B5
:10A3980042B962F306048DF800409DF8024065F367
:10A3A800C4040EE08D68AA4286BF4D6165F30604B9
:10A3B80062F306048DF800409DF80240012262F322
:10A3C800C4048DF80240009A1A61C278012A05D1A6
:10A3D8000A780C6900EB82029269546146F00442E3
:10A3E8001A60C378002B34D14B69002B31D0036934
:10A3F8000A78586B012101FA02F202435A6328E0F5
:10A408000B784E698C6800EB83035B6D1A681D69D5
:10A418000095EDB206B14C6164F306059DF8024063
:10A428008DF80050012565F3C4048DF80240009CA6
:10A438001C61C378012B05D10B780C6900EB8303F1
:10A448005B6D5C610B7800EB830042F00442436D66
:10A458001A6000207CBD4B78012B0B7800EB830041
:10A468000AD182691368C3F3076101F08001C9B298
:10A4780021B143F0804301E0426D136843F40013B7
:10A488001360002070474B78012B0B78C97800EBDC
:10A4980083000CBF8269426D02391368C9B26FF339
:10A4A8005553012998BF43F080531360002070472B
:10A4B80003699A69D8691040000C704700EB810164
:10A4C80002694B6D9B685069184070470369986929
:10A4D800DB69184080B2704782B000230093C02324
:10A4E8008DF803300122002362F3C4038DF8023093
:10A4F80018238DF80030009A436D1A61C278012A3A
:10A5080006D100F5B96058611A684FF080221A60C8
:10A5180002B07047D0F8143110B50446D3B10369BE
:10A528009A68D20716D5827A42B1D0F80C21D0F8B1
:10A538000C116FF341026FF300020A605A6842F08F
:10A5480001025A600520FFF7E5FB23695A6822F0EB
:10A5580001025A6010BD837A63B103699B68D90709
:10A5680008D5D0F80C31D0F80C216FF341036FF304
:10A57800000313607047012310B5002280F81231E0
:10A5880004460346FF2104E058698160186D0132D2
:10A598008160607804338242F6D3236900221A610D
:10A5A8005A61DA614FF0FF329A612046FFF7FEFCEC
:10A5B80020461021BDE81040DBE44B78012B0B78D6
:10A5C80000EB83000FD183691868C0F3074000F0DF
:10A5D8002003DBB2CBB900F00200C0B200280CBFE8
:10A5E800302020207047436D1868C0F3074000F002
:10A5F8002003DBB25BB900F00200C0B200280CBF38
:10A608004FF440504FF400507047102070474FF4FB
:10A61800805070474B78012B0B7810B500EB830303
:10A628000AD19C69102A236802D1BDE8104012E7BC
:10A63800202A0CD0302A0FE05C6DB2F5805F2368C9
:10A6480002D143F400131BE0B2F5005F02D143F0DE
:10A65800006315E0B2F5405F0FD1C3F3074202F083
:10A668002002D2B222B100234B71BDE810400AE7A4
:10A6780043F0806343F0802302E00AB962F3CF33EA
:10A68800236010BDF8B50446FFF794FB01220023B0
:10A6980084F8122184F813312827164619464025D4
:10A6A8000CE007FB03F000F58C7022182354D380CC
:10A6B8005670D1709560D1605161013362789342D0
:10A6C800EFD300232826194640250CE006FB03F0AB
:10A6D80000F55C7022182354D3805170D1709560B6
:10A6E800D1605161013362789342EFD32046FFF77E
:10A6F80039FC2046FFF7BEFB00212046FFF770FC1F
:10A708002046FFF7C3FC2046BDE8F840FFF723BC0E
:10A7180070B5CDB20C464FF0280601F07F0106FB5C
:10A72800010115F0800F14BF01F58C7101F55C7102
:10A7380004F07F04ED090C704D708A60CB7005B190
:10A74800CC80022B01D100230B71FFF743FD0020C1
:10A7580070BD10B5CAB201F07F034FF0280404FBA6
:10A76800030312F0800F14BF03F58C7303F55C73B9
:10A7780001F07F01D20919705A701946FFF759FD87
:10A78800002010BD38B501F07F0528246C4304F57E
:10A798005C7401194B6100238B614B70EBB203555C
:10A7A800CA60C478012C08BF0A6113B9FFF7E6FD37
:10A7B80001E0FFF75DFD002038BD70B501F07F04B2
:10A7C8002825654305F58C7541190126E4B2CA6050
:10A7D8000A6100224E7044558A614B6114B9FFF733
:10A7E800CDFD01E0FFF744FD002070BDCAB212F0B4
:10A7F800800F10B54FF0280306D001F07F0403FB4B
:10A80800040303F58C7303E003FB010303F55C7396
:10A81800D209012401F07F0119709C705A70194601
:10A82800FFF719FE002010BDCAB212F0800F10B554
:10A838004FF0280306D001F07F0403FB040303F55F
:10A848008C7303E003FB010303F55C730024D20956
:10A8580001F07F0119709C705A701946FFF713FEBA
:10A86800204610BD08B50B0604D501F07F01FFF79F
:10A8780080FB01E0FFF79AFB002008BD0369002276
:10A8880061F30A1219680A431A60704703695A6823
:10A8980003206FF341025A60FFF73CBA03695A6814
:10A8A800032042F002025A60FFF734BA11F0800F19
:10A8B8004FF0280306D001F07F0103FB010101F5E9
:10A8C8008C7103E003FB010101F55C71FFF775BEB4
:10A8D80011F0800F4FF0280306D001F07F0103FB31
:10A8E800010101F58C7103E003FB010101F55C71C5
:10A8F800FFF790BE2DE9F74F0446FFF78BFB0028C2
:10A9080000F03F822046FFF792FB0546002800F042
:10A918003882C0F3074000F00800C0B2002861D0B8
:10A928002046FFF7C5FDA146824627464FF000089E
:10A93800DFF86CB32E4650E01AF0010F46D05FFAEC
:10A9480088F2114620460092FFF7B8FD10F0010F7B
:10A958000546009A20D07B6D01259D60E178A942CB
:10A9680007D11B69D9F87813C3F31203CB1AC9F8B6
:10A978008833DBF8003020461B6811469847E37897
:10A98800012B09D1B8F1000F06D194F81131052B2C
:10A9980002D12046FFF7A0FD05F00203DBB213B198
:10A9A8007B6D02259D6005F00403DBB213B17B6D5E
:10A9B80004259D6005F00805EDB23DB1DBF80030D7
:10A9C80020469B6898477B6D0820986008F101082D
:10A9D8004FEA5A0A043709F12809BAF1000FABD136
:10A9E80035460120C5F3074303F00403DBB2002B0F
:10A9F80000F0AF802046FFF769FD264683464FF0FA
:10AA0800000801959FE01BF0010F00F09780236973
:10AA18005FFA88F919695D6B04EB890225FA09F573
:10AA28009269ED019268EDB20D431540EA071CD515
:10AA38005A6B012000FA08F122EA01025A63B3694D
:10AA4800974A9860136805465B68204649469847C8
:10AA5800E378AB4209D1B8F1000F06D194F811316F
:10AA6800042B02D12046FFF737FD05F00403DBB2C3
:10AA780013B1B36904259D6005F00803DBB213B177
:10AA8800B36908259D6005F01003DBB213B1B36903
:10AA980010259D6005F02003DBB213B1B3692025B2
:10AAA8009D6005F04003DBB213B1B36940259D609A
:10AAB80005F00203DBB213B1B36902259D6025F0EE
:10AAC8007F0515F0FF0F39D0282505FB084505F54A
:10AAD8008C75C246AB696A69C3EB020CAB689C45CE
:10AAE80028BF9C460CF1030CB3694FEA9C0C9B6988
:10AAF8006746A04614E0AA68E9681C1B944228BF70
:10AB08001446A3B240464A46FFF72EF9EB681B19D4
:10AB1800EB60AB69E71C1C19AC61B3699B69BF08A2
:10AB28009BB2BB4205D9AC696B699C4201D2002B30
:10AB3800E1D1B369802544469D60D04608F10108FB
:10AB48004FEA5B0B0436BBF1000F7FF45CAF019D4D
:10AB5800012005F00203DBB213B1E36802225A6157
:10AB6800C5F3076303F08003DBB2CBB1A37A43B12B
:10AB7800D4F80C31D4F80C216FF341036FF30003C0
:10AB8800136023695A6822F001025A60444B1B681B
:10AB980020469B699847E3684FF000425A610120BC
:10ABA800C5F3072303F00803DBB2F3B13C4B1B6882
:10ABB80020465B6998472369E2689B684FF4006107
:10ABC8005161A27A82B1DB070ED5D4F80C311A682C
:10ABD80042F001021A601A6842F003021A60314B0F
:10ABE8001A6942F006021A61012005F00803DBB277
:10ABF80043B12B4B1B682046DB689847E368082263
:10AC08005A61012005F01003DBB2002B33D0E36852
:10AC18009A6922F010029A611F6A282607F00F032A
:10AC280006FB0346C7F34343022B06F55C7602D0C6
:10AC3800062B1AD10EE047F6F0733B40ABB1C7F3D1
:10AC48000A172046F1683A46FFF7A2F8F368DB19BD
:10AC5800F36007E004F5B96120460822FFF798F889
:10AC6800C7F30A17B369DF19B761E3689A6942F055
:10AC780010029A610120C5F3072303F01003DBB229
:10AC8800002B39D023695A68002622F001025A6045
:10AC980031462046FFF76DF923463246FF2108E08A
:10ACA8004C02002000ED00E058698160186D013207
:10ACB8008160607804338242F6D3236901274FF01C
:10ACC800FF3267F30F069A6167F31F460F22DE61B2
:10ACD8005A612F221A611A686FF30A121A60204605
:10ACE800FFF7FAFBE3684FF480525A61264B1B6862
:10ACF80020461B6998473846C5F3072303F020030D
:10AD0800DBB2EBB12046FFF74FFAE3682046DE6876
:10AD1800FFF73CFA032806D10023A3704FF4007311
:10AD2800A380092304E00123A3704023A380052303
:10AD380063F38D26E3684FF40052DE6001205A6108
:10AD4800C5F3074303F01003DBB24BB10E4B1B688E
:10AD58002046DB699847E3684FF480125A61012066
:10AD6800C5F3074505F02005EDB255B1064B1B6844
:10AD780020461B6A9847E3684FF400125A61012085
:10AD8800FFE7BDE8FE8F00BF4C02002043230B8085
:10AD980000487047BC01002038B51F4B1A68511C89
:10ADA800052A196035D11979002201291A6030D095
:10ADB8009968B1F5006F08BF9A60174B9968DC680D
:10ADC800A1421A4602D100221A7122E086BFC1F5BB
:10ADD80000631361C1EB0404D0F8EC3598BF14612B
:10ADE8001569B3F839300C4C9D428AB204D9591808
:10ADF800ED1AA160256104E06918A1600021ABB2D9
:10AE08002161054901240C7104498A188121FFF741
:10AE1800D4FC002038BD00BF7C0D002063C6002094
:10AE280038B528230A4D03FB01010A4BB1F88813F2
:10AE38001B69044628469847D4F8EC352046B3F8F1
:10AE4800403001212A46FFF79DFC002038BD00BF95
:10AE58001BC600203802002070B50B7813F060057F
:10AE680006460C4625D0202D1FD1CD88B5B113F04C
:10AE7800800F487808D0214B21499B682A4698477B
:10AE8800E2881F49304625E01E4B1D4958641E4B79
:10AE980030465D612A4600F022FB1DE0174B4878DA
:10AEA8009B6829462A46984725E000F077FB02254B
:10AEB80021E04B780A2B11D00B2B14D0062B1AD17A
:10AEC8004B881B0A212B03D1CA883A2A28BF3A2269
:10AED8000E49304600F0EAFA00250CE00C49012240
:10AEE80000F0E4FA07E08B781BB9074A1D46936126
:10AEF80001E000F053FB284670BD00BF3802002077
:10AF08005BC60020BC0100207C0D0020CE01002083
:10AF1800940D002010B581210446FFF71AFC012189
:10AF28002046FFF716FC82212046FFF712FC024B51
:10AF38005B689847002010BD3802002038B5D0F86B
:10AF4800EC350446B3F8392081210223FFF7E0FBF2
:10AF5800D4F8EC350121B3F8402020460223FFF74E
:10AF6800D7FB8221082203232046FFF7D1FB094B98
:10AF7800022200251A715D71074B1B689847D4F8A7
:10AF8800EC35064AB3F8403020460121FFF7FAFBBA
:10AF9800284638BD7C020020380200201BC600204D
:10AFA80010B5074C606CFF2807D0064B064A9B6813
:10AFB800064952699847FF236364002010BD00BF0B
:10AFC800BC010020380200207C0D00205BC6002058
:10AFD80038B510490B79012B19D10C690CB90C71D2
:10AFE80015E0D0F8EC358D68B3F839309C42AAB238
:10AFF80003D95D198D60E41A03E0A3B22C198C60A3
:10B0080000240C61044952188121FFF7D6FB002067
:10B0180038BD00BF7C0D002063C6002000207047AB
:10B02800002070470023F0B5084A094E1D4609E084
:10B038001468C75C375501340133B4F5006F1460E8
:10B0480008BF15608B42F3D10020F0BD880D0020A9
:10B0580063C60020104B114AD3F800C000232DE925
:10B06800F0410F4F16461D460DE0146810F8038096
:10B0780007F804800134802C08BF2C46146034681B
:10B08800644505D001338B42EFD10020BDE8F08143
:10B098000220BDE8F08100BFE4CE0020F8CE0020F9
:10B0A80064CE002021280FD1084B1A680A701A684C
:10B0B800120A4A705A888A70DA78CA701A790A713C
:10B0C8005A794A719B798B710020704730020020B1
:10B0D80007B502AB012103F8010D1846FFF7A2FFDF
:10B0E8000EBD002100E00131435C002BFBD199E744
:10B0F80098E70B4B0B491A68096891420BD00A492B
:10B108008A5C02701A680132802A1A6005D100220E
:10B118001A6001207047002070470120704700BF67
:10B12800E4CE0020F8CE002064CE0020204B1A6820
:10B13800204B1B689A42F0B509D135E00133802BCA
:10B1480008BF00239A4203D11A4B1A602CE01A4C0C
:10B15800E15C0029F2D00A29F0D00D29EED0154C77
:10B168001549134D23600E460023CF182268BA5C98
:10B17800C254226801339F18802F08BF53422F689A
:10B188009A18974210D0B25C1AB10A2A01D00D2A37
:10B19800EBD10022C254074A116859187F2911605F
:10B1A80003D98039116000E000231846F0BD00BFC4
:10B1B800F8CE0020E4CE002064CE0020704700BF07
:10B1C800D0F8E43510B51B6904469847032384F882
:10B1D8001231002010BD08B5042380F81231D0F8D0
:10B1E800E435DB689847002008BD08B5D0F8E0359D
:10B1F800DB6903B19847002008BD08B5D0F8E035F1
:10B208001B6A9847002008BD08B5D0F8E0355B6A8E
:10B218009847002008BD002110B5402204460B467F
:10B22800FFF776FA8021402200232046FFF770FAC4
:10B23800012384F81231D4F8E435A0785B68984784
:10B24800002010BD13B56946044600F085F99DF845
:10B25800001001F01F03012B07D0022B0AD073B98D
:10B268002046694600F026FA0FE02046694600F0BD
:10B2780007FA0AE02046694600F0A2F905E021F045
:10B288007F01C9B22046FFF7B1FA00201CBD38B5CE
:10B29800044600293DD190F81131022B42D1D0F853
:10B2A8003421D0F820319A4211D9C178D21A012913
:10B2B800C0F8342104D1D0F82411CB18C0F82431B7
:10B2C80092B22046D4F8241100F000F92AE0D0F810
:10B2D8003821B2FBF3F503FB152565B99A420AD369
:10B2E800D0F83C319A4206D229462A4600F0EEF8B8
:10B2F800C4F83C5116E0D4F8E035DB682BB194F87B
:10B308001221032A01D120469847204600F00FF960
:10B3180008E0D0F8E0355B6923B190F81221032AE0
:10B3280000D19847002038BD10B5044659BB90F8A5
:10B338001131032B30D1D0F88C23D0F878339A42CE
:10B3480014D9C178D21A0129C0F88C2304D1D0F8B5
:10B358007C13C918C0F87C139A4228BF1A4692B2C7
:10B368002046D4F87C1300F0CAF815E0D0F8E03590
:10B378001B6923B190F81221032A00D1984720466F
:10B3880000F0C6F808E0D0F8E0359B6923B190F8E2
:10B398001221032A00D19847002010BD2DE9F04161
:10B3A800069F0446164698460D46FEF741FC204681
:10B3B8002946C4F8E085C4F8E475C4F8E865FFF7E1
:10B3C80061F9D4F8E4351B6898472046BDE8F04198
:10B3D800FEF782BC00207047D0F8E03510B504466F
:10B3E8001B689847D4F8E4359B689847002010BD3F
:10B3F80008B5D0F8E0355B689847002008BD000024
:10B4080012230B80004870477C02002004230B8025
:10B41800004870478E02002010B5044C04480A46C4
:10B42800214600F075FA204610BD00BFFCCE002072
:10B43800989A05080A4608B50248034900F068FAD0
:10B44800014808BDAB9A0508FCCE00200A4608B59D
:10B458000248034900F05CFA014808BDB99A05089A
:10B46800FCCE002008B50A4608B9044800E00448A4
:10B47800044900F04DFA034808BD00BFC49A050806
:10B48800D19A0508FCCE002008B50A4608B9044838
:10B4980000E00448044900F03BFA034808BD00BF37
:10B4A800DE9A0508FF9A0508FCCE002010B5134661
:10B4B8000C46C0F83821C0F83421022280F8112146
:10B4C80000212246FFF779F9002010BD10B50C467F
:10B4D800134600212246FFF770F9002010BD10B571
:10B4E80013460C46C0F89023C0F88C23032280F83A
:10B4F800112100212246FFF745F9002010BD10B5A3
:10B508000C46134600212246FFF73CF9002010BDE7
:10B518000021042310B50A46044680F811310B4671
:10B52800FFF74BF92046FEF7D7FF002010BD00219A
:10B53800052310B50A46044680F811310B46FFF77B
:10B5480021F92046FEF7C8FF002010BD282303FB81
:10B558000100B0F88803704790F8C8350B7090F870
:10B56800C9354B7090F8CB2590F8CA3503EB022308
:10B578004B8090F8CD2590F8CC3503EB02238B80D7
:10B5880090F8CF2590F8CE3503EB02239BB2CB8001
:10B59800C0F83C31012380F81131704710B591F99A
:10B5A8000030002B044601DBCB880BB9802100E07A
:10B5B8000021FFF71BF92046BDE81040FEF78CBFBD
:10B5C80038B50D4604466B780979012B10D027D37E
:10B5D800032B51D190F81231022B28D0032B47D1DD
:10B5E8006B889BB991B1802910D0FFF7FFF80DE067
:10B5F80090F81231022B1AD0032B39D16B88002B0B
:10B608003AD149B1802907D0FFF70EF9D4F8E035CF
:10B6180020469B68294698472046FFF779FF2BE08C
:10B6280090F81231022B02D0032B21D106E019B376
:10B63800802921D02046FFF7D9F81DE011F0800FAE
:10B648004FF0280306D001F07F0103FB010393F8B4
:10B658001A2103E003FB010191F87223074B02B1A1
:10B6680001221A60204605490222FFF71FFF03E066
:10B6780020462946FFF792FF002038BD980D00208C
:10B6880038B590F81231032B04460D460CD10B79CE
:10B69800012B09D8D0F8E0359B689847EB883BB96F
:10B6A8002046FFF735FF03E020462946FFF776FFDF
:10B6B800002038BD73B54B7804460D46092B00F2BF
:10B6C8001C81DFE813F0D10008011A01E4001A0117
:10B6D80072000A001A01C00092004B881A0A013A47
:10B6E800062A00F20A81DFE812F007001A00270094
:10B6F8000801080108010801D4F8E835A0781B689A
:10B708000DF106019847EB88402B014603D094F8C9
:10B718001231012B3AD10823ADF8063036E0D4F8BF
:10B72800E035A0789B6A0DF1060198470223437023
:10B738000146C4F8EC0529E0DBB2052B00F2DD80F8
:10B74800DFE803F003080D12171CD4F8E835A078D9
:10B758005B6817E0D4F8E835A0789B6812E0D4F865
:10B76800E835A078DB680DE0D4F8E835A0781B69E7
:10B7780008E0D4F8E835A0785B6903E0D4F8E83548
:10B78800A0789B690DF1060198470146BDF806307F
:10B79800002B00F0B680EA88002A00F0B2809A42B6
:10B7A80028BF1A46ADF806205CE08B88002B40F0D5
:10B7B800A480CB88002B40F0A08094F812214B88FD
:10B7C800032A00F09A8003F07F05204684F813517D
:10B7D8002946FFF753F82046FFF79AFE0DB10223DA
:10B7E80000E0012384F812318BE08978464E012964
:10B7F800317100F2828094F81231022B02D0032BAF
:10B808007BD108E0002962D00121032384F81011BC
:10B8180084F8123113E041B9022384F8123184F814
:10B8280010112046FFF7E4FD51E094F810110129AA
:10B8380020464DD0FFF7DCFD317984F81011204601
:10B84800FFF7CAFD43E0CA88012A56D194F812319D
:10B85800022B02D0032B50D102E020462B4913E0E3
:10B8680004F5887120460FE094F81231023B012B51
:10B8780043D8D4F814312449002B0CBF01230323E7
:10B8880041F80C3F20460122FFF710FE39E04B88B3
:10B89800012B29D0022B34D18B8813F0FF0F30D124
:10B8A80021691B0A013B4A68042B0FD8DFE803F023
:10B8B800030507090B00012306E0022304E0032324
:10B8C80002E0042300E0052363F306124A602046E1
:10B8D800FFF71EFE15E094F81231023B012B0CD83D
:10B8E8004B88012B0DD10023C4F81431D4F8E0356E
:10B8F80020469B6829469847E9E720462946FFF7EE
:10B908004DFE00207CBD00BF980D0020A00D00203A
:10B9180030B5C8B10023DDB20133C41814F8014CA6
:10B92800002CF8D16B1C5B0013800B7003234B7049
:10B93800022305E0CA545A1CD2B202338C54DBB23B
:10B9480010F8012B002AF5D130BD00BF70477047B1
:10B958007047704770477047704700000EB403B0D7
:10B9680070470A2810B5044602D10D20FFF7F9FFE9
:10B97800064A13681BB103F8014B136010BD044B52
:10B988001B680BB12046984710BD00BFA80D0020CA
:10B9980030CF002010B5044601E0FFF7E2FF14F8AD
:10B9A800010B0028F9D110BD2DE9F04F044685B0F0
:10B9B8000D464FF00A0A00E035462078002800F0CE
:10B9C800C480252801D0013467E06078302803D18D
:10B9D800A0780123033407E02D2802D00234002385
:10B9E80002E0A078022303344FF0000805E00AFBC8
:10B9F800080814F8010BA8F13008A0F13002D2B2FF
:10BA0800092AF4D96C2801D04C2803D114F8010B69
:10BA180043F00403002800F09880602886BFA0F156
:10BA28002002D2B202464F2A3DD006D8432A2DD052
:10BA3800442A09D0422A30D133E0552A04D0582A62
:10BA480029D0532A29D101E00A272DE02E1D2F687D
:10BA5800002500E001357A5D002AFBD104E02020B2
:10BA6800FFF77FFF4D4601E0980704D4454505F1EF
:10BA78000109F4D34D463846FFF78CFF03E0202038
:10BA8800FFF76FFF01354545F9D395E728782E1D57
:10BA9800FFF767FF90E7102706E0FFF762FF2E46E3
:10BAA8008AE7022700E008272E1D442A296804D1C6
:10BAB800002902DA494243F00803002200E02A463E
:10BAC800B1FBF7FE07FB1E11CDB2092D714607D950
:10BAD800782814BF4FF0070C4FF0270C6544EDB2DF
:10BAE80030350DF80250551CBEF1000F02D0102D54
:10BAF800E5D10F22190705D504A94D192D2105F8FF
:10BB0800101C951C13F0010F0CBF4FF0200B4FF0C9
:10BB1800300B9B072F4604D508E05846FFF721FF56
:10BB28004F46474507F10109F7D34F46013D1DF838
:10BB38000500FFF716FF002DF8D103E02020FFF7DE
:10BB480010FF01374745F9D336E705B0BDE8F08F58
:10BB580070B5064D0C462E68286001E0FFF701FF1E
:10BB680014F8010B0028F9D12E6070BD30CF0020E9
:10BB78000FB407B504A951F8040B0191FFF714FF9E
:10BB8800BDE80E4004B070470EB417B505A9084CBF
:10BB980051F8043B206018460191FFF705FF226821
:10BBA800002313702360BDE81E4003B0704700BF38
:10BBB800A80D00200EB433B505A9074C51F8043B75
:10BBC8002568206018460191FFF7EEFE2560BDE864
:10BBD8003C4003B0704700BF30CF002070B51E4610
:10BBE80004461C481546FFF7C3FF022E1FD0042E3B
:10BBF80025D0012E2AD105E0A15D1748FFF7B8FF2F
:10BC0800013600E00026AE42F6DB2020FFF7A9FE51
:10BC1800002609E0A05DA0F12003DBB25E2B88BFFF
:10BC28002E20FFF79EFE0136AE42F3DB0EE034F81D
:10BC3800021B0A48FFF79CFF013DF8D106E054F8C3
:10BC4800041B0748FFF794FF013DF8D10A20BDE81F
:10BC5800704086E6209B0508279B05082D9B050854
:10BC6800339B050808B501214FF4807001F07CFA78
:10BC78004FF480700021BDE8084001F075BA4368B0
:10BC88000A6823F0407323F4807313430A7943EA64
:10BC980002234360CA680B6930B51A4384688D680B
:10BCA800084B2A43234013434A7943EA42038360FB
:10BCB8000B7DC26A013B22F47002DBB242EA0353F5
:10BCC800C36230BDFDF7FFC00023036003714371F9
:10BCD8008360C3600361012303757047074A084BFB
:10BCE800516810B50B4090E8120021438468C06881
:10BCF800214301430B43536010BD00BF00230140A3
:10BD0800E030FCFF0023036043608360C36070473A
:10BD1800836811B143F0010301E023F0010383605C
:10BD28007047436823F4400323F400730B434360D4
:10BD38007047416282627047436823F01F030B43D8
:10BD480043607047044B5A6810B142F4000201E0A6
:10BD580022F400025A60704700230140044B5A68DD
:10BD680010B142F4800201E022F480025A60704768
:10BD780000230140092970B50CB20CD904EB440426
:10BD88001E3CC6680725A54026EA0505A34045EAE6
:10BD98000304C4600AE0066904EB44040725A540CF
:10BDA80026EA050513FA04F42C430461062A0CD884
:10BDB8000523013A5A43446B1F23934024EA0303A3
:10BDC800914043EA0102426370BD0C2A12B20CD8BA
:10BDD80002EB8202233A046B1F23934024EA0303F5
:10BDE800914043EA0102026370BD02EB8202413ACC
:10BDF800C46A1F23934024EA0303914043EA0102E3
:10BE0800C26270BD836843F0804383607047806876
:10BE1800C0F380507047836811B143F4806301E038
:10BE280023F4806383607047836811B143F0020391
:10BE380001E023F00203836070474368013923F46B
:10BE4800604343EA413343607047436811B143F4A8
:10BE5800006301E023F4006343607047C06C80B264
:10BE68007047014B1868704708230140836811B177
:10BE780043F4807301E023F4807383607047836820
:10BE880011B143F4007301E023F400738360704739
:10BE9800044B5A6810B142F4005201E022F40052F7
:10BEA8005A60704700230140092970B50CB20CD9BB
:10BEB80004EB44041E3CC6680725A54026EA050590
:10BEC800A34045EA0304C4600AE0066904EB44049D
:10BED8000725A54026EA050513FA04F42C43046156
:10BEE800836BC3F30154121B0232D2B202EB8202FB
:10BEF8001F24944023EA040391400B43836370BDDD
:10BF0800836B013923F4401343EA01538363704779
:10BF180082B0002301930190019BCB180193019BF0
:10BF28001A6002B07047836823F470230B43836060
:10BF38007047836823F440130B438360704783681A
:10BF480043F48003836070478068C0F38050704773
:10BF5800436811B143F4806301E023F480634360D4
:10BF68007047436811B143F4805301E023F48053D0
:10BF78004360704782B0002301930190019B2833EE
:10BF88005B180193019B186880B202B070470123C7
:10BF9800C9B213FA01F143680AB1194301E023EA6F
:10BFA800010141607047036819420CBF002001205D
:10BFB8007047C943016070474368006810EA112060
:10BFC80007D00122C9B212FA01F119420CBF0020B0
:10BFD800012070476FEA112101607047036823F060
:10BFE800010303600023036043608360C36003614F
:10BFF800212343612C4B98421CD02C4B984220D0D3
:10C008002B4B984225D02B4B98422AD02A4B98424A
:10C018002FD02A4B984233D0294B984237D0294BFE
:10C02800984204D14FF03D5243F8AC2C7047264B50
:10C03800984203D13D2243F8082C7047234B98427D
:10C0480004D14FF4746243F8202C7047204B984277
:10C0580004D14FF4741243F8382C70471D4B9842A2
:10C0680004D14FF0746243F8502C70471A4B984231
:10C0780003D11A4A43F8642C7047194B984203D1EC
:10C08800184A43F87C2C7047174B984203D1174A3B
:10C0980043F8942C7047164B984204BF4FF03D521A
:10C0A80043F8AC2C704700BF106002402860024083
:10C0B8004060024058600240706002408860024060
:10C0C800A0600240B8600240106402402864024048
:10C0D8004064024058640240706402403D00002001
:10C0E80088640240400F0020A064024000003D2008
:10C0F800B86402400268134B10B51340CC680A6854
:10C1080022434C6922438C692243CC6922430C6A3E
:10C1180022434C6A22438C6A22434C6B22438C6B29
:10C1280022431343036042690C6BCB6A22F0070277
:10C138002343134343610B6943604B6883608B68F7
:10C14800C36010BD3F801CF0002303604360836020
:10C15800C360036143618361C361036243628362B5
:10C16800C3620363436383637047036811B143F099
:10C17800010301E023F0010303607047036811B174
:10C1880043F4004301E023F400430360704703686D
:10C1980011B143F0200301E023F02003036070474E
:10C1A80041607047406880B27047036812B143F439
:10C1B800002301E023F40023036001617047036852
:10C1C80011B143F4802301E023F480230360704716
:10C1D8000AB101617047C16070470068C0F3C04090
:10C1E8007047006800F001007047406900F03800AF
:10C1F80070470A4A0A4B10B50A4CA04288BF13463A
:10C208008A004CBF5B681B6821F0F02121F0821185
:10C2180019420CBF0020012010BD00BF006402407D
:10C22800006002400F64024010B5084B084A094CF0
:10C23800A04288BF134611F0005F21F0F02121F0E1
:10C24800821114BFD960996010BD00BF0060024020
:10C25800006402400F6402400B0607D5436912B11F
:10C2680043F0800301E023F080034361802909D073
:10C2780001F01E01036812B119430160704723EAF7
:10C28800010101607047124B124A10B5124CA042CE
:10C298008CBF14461C4621F0F02323F0C3132BB1A6
:10C2A800026802F01E0202EAD12202E0426902F0AC
:10C2B800800288004CBF6368236821F0F02121F0D8
:10C2C8008210184002D0101C18BF012010BD00BFFA
:10C2D80000600240006402400F64024010B5084B41
:10C2E800084A094CA04288BF134611F0005F21F0AC
:10C2F800F02121F0821114BFD960996010BD00BFF0
:10C3080000600240006402400F640240044B0022B7
:10C318001A605A609A60DA60024A5A61704700BF30
:10C32800003C0140FFFF7F00837910B5002B29D026
:10C338001A4B01681C68CA4314401C605C682240A0
:10C348005A60027902F1804202F59E321468214354
:10C35800116002689C68D1430C409C60DC682140F5
:10C36800D9604179102906D1996811439960D96833
:10C378000A43DA6010BD01F1804303F59E33196862
:10C388000A4308E00379016803F1804303F59E330B
:10C398001A6822EA01021A6010BD00BF003C014081
:10C3A80000230C2203600371427183717047024BB2
:10C3B8001A6902431A617047003C0140034B5B69EC
:10C3C80018420CBF00200120704700BF003C01400C
:10C3D800014B5861704700BF003C0140054B1A688B
:10C3E8005B69034004D010420CBF00200120704755
:10C3F80018467047003C0140014B5861704700BF28
:10C40800003C01404FF0204318B943F2DB021A60A8
:10C4180003E043F2D20243F820204FF02042411CAF
:10C428006FF0704342F8213002F5827242F82030F2
:10C43800704770B584684568C368C16A0268254357
:10C448001D4303691D4343691D4383691D43C36934
:10C458001D43036A1D43436A1D43836A1D43036BDF
:10C468000D431D434FF02043082C43F8225005D1BB
:10C4780053F8224044F0400443F82240436B9E693D
:10C488001D6835435E6845EA06159E6845EA062537
:10C49800DE6845EA06451E695B6945EA0655541C8F
:10C4A80045EA03654FF02043B1F5804F43F8245027
:10C4B80010D1836B986919680143586841EA0011E3
:10C4C800986841EA002118695B6941EA005141EA2C
:10C4D800036101E06FF07041014B43F8221070BD19
:10C4E800040100A0022242604FF480524262416B74
:10C4F8004FF4005210B5826200230F22FF2403601C
:10C508008360C360036143618361C3610362C36283
:10C5180003630A604A608C60CA600A614A618B6181
:10C52800816B0A604A608C60CA600A614A618B61EB
:10C5380010BD4FF0204321B153F8202042F00102F2
:10C5480003E053F82010024A0A4043F820207047BD
:10C55800FEFF0F0010280CBF064B074B4FF04002A0
:10C568004FF0180119605A604FF0FC329A60DA6097
:10C57800704700BF600000A0800000A030B583684D
:10C5880044681C43C36844F008041C4303691C4303
:10C59800436944EA4324836944EA4334C369996894
:10C5A8005A68090441EA02211A68DB68114341EA22
:10C5B8000361036A9A685D68120442EA05221D68ED
:10C5C800DB682A4342EA03620368102B0CBF034B63
:10C5D800034B1C609960DA6030BD00BF600000A0AA
:10C5E800800000A010230360C269002343608360B9
:10C5F800C360036143618361FC23136053609360EC
:10C60800D360026A136053609360D360704741B18E
:10C6180010280CBF074B084B1A6842F004021A6036
:10C62800704710280CBF034A034A044B11680B409B
:10C6380013607047600000A0800000A0FBFF0F009F
:10C6480041B110280CBF084B084B1A6842F0400251
:10C658001A60704710280CBF034A044A044B11683B
:10C668000B401360704700BF600000A0800000A06E
:10C67800BFFF0F00102802D1024B58697047024BC8
:10C6880058697047600000A0800000A0054B182280
:10C698001A6000225A604FF0FC329A60DA601A6120
:10C6A800704700BFA00000A00268436842F0100273
:10C6B80042EA4322836842EA4332144B10B51A60B7
:10C6C800C26891685468090441EA04211468D26870
:10C6D800214341EA02629A60026991685468090438
:10C6E80041EA04211468D268214341EA0262DA600F
:10C6F800426991685068090441EA00211068D268CB
:10C70800014341EA02621A6110BD00BFA00000A007
:10C71800C2680023036043608360FC231360536096
:10C728009360D3600269136053609360D360426979
:10C73800136053609360D3607047054B18B11A6853
:10C7480042F0040202E01968024A0A401A6070477F
:10C75800A00000A0FBFF0F0062B1102801D10E4B12
:10C7680003E0B0F5807F03D10C4B5A68114311E008
:10C778000B4BFAE7102804D1074B5A6822EA01014B
:10C7880008E0B0F5807F0CBF044B054B5A686FEA90
:10C798000101114059607047600000A0800000A0AE
:10C7A800A00000A0102801D1064B04E0B0F5807F5E
:10C7B8000CBF054B054B5B680B420CBF00200120EA
:10C7C800704700BF600000A0800000A0A00000A08B
:10C7D800102804D1074B5A6822EA010108E0B0F595
:10C7E800807F0CBF044B054B5A686FEA010111406A
:10C7F80059607047600000A0800000A0A00000A061
:10C80800102801D1084B04E0B0F5807F0CBF074B1E
:10C81800074B5B6813EA010004D013EAD1010CBF8F
:10C8280000200120704700BF600000A0800000A029
:10C83800A00000A0102804D1084B5A6822EAD101B0
:10C8480009E0B0F5807F0CBF054B064B5A684FEAEC
:10C85800D10122EA01015960704700BF600000A0C1
:10C86800800000A0A00000A008B52C4B984205D17C
:10C878000120014600F048FC012048E0284B98427E
:10C8880005D10220012100F03FFC02203FE0254BAA
:10C89800984205D10420012100F036FC042036E03E
:10C8A800214B984205D10820012100F02DFC0820D9
:10C8B8002DE01E4B984205D11020012100F024FCE8
:10C8C800102024E01A4B984205D12020012100F0C5
:10C8D8001BFC20201BE0174B984205D1402001216A
:10C8E80000F012FC402012E0134B984205D1802042
:10C8F800012100F009FC802009E0104B98420BD17F
:10C908004FF48070012100F0FFFB4FF4807000218C
:10C91800BDE8084000F0F8BB08BD00BF00000240B9
:10C928000004024000080240000C024000100240CF
:10C938000014024000180240001C0240002002407F
:10C948002DE9F0470023D1F800801A464FF0010C7A
:10C9580003270CFA02F404EA0805A5422ED106685A
:10C9680017FA03F4E443264006600E79D0F80090E5
:10C9780006FA03FA013E4AEA0909012EC0F80090B6
:10C9880014D8866891F8059026408660866809FA6A
:10C9980003F949EA06068660466826EA0505456001
:10C9A8008D7946689540ADB235434560C5682C40E1
:10C9B800C460CC79C5689C402C43C4600132023302
:10C9C800102AC6D1BDE8F0874FF6FF730360002335
:10C9D800037143718371C371704782B04FF4803320
:10C9E8000193019B0B430193019BC361C161019BAF
:10C9F800C361C3690193C369019302B070470369B6
:10CA080019420CBF002001207047006980B27047AE
:10CA1800436919420CBF002001207047406980B269
:10CA2800704701837047418370470AB1018370479B
:10CA3800418370474161704743694B404361704788
:10CA480001F00703C908083130B59B0050F82150A0
:10CA58000F249C4025EA040440F8214050F8214066
:10CA680012FA03F31C4340F8214030BD08B5134BBC
:10CA7800984207D14FF40010012100F069FB4FF4F0
:10CA8800001014E00E4B984207D14FF480000121AA
:10CA980000F05EFB4FF4800009E00A4B98420BD18E
:10CAA8004FF40000012100F053FB4FF40000002177
:10CAB800BDE8084000F04CBB08BD00BF0054004072
:10CAC80000580040005C00407FB5044686886846F0
:10CAD8000D4600F06DFA02992C482B6826F03F06A7
:10CAE8003604B1FBF0F0360C80B20643A6802288EB
:10CAF80022F001021204120C2280254A93420AD81D
:10CB08005B00B1FBF3F301309BB280B22084032BAE
:10CB180098BF042321E0EE884BF6FF72964205D1B8
:10CB280003225343B1FBF3F39BB206E019225343AC
:10CB3800B1FBF3F39BB243F480431A054FF49672AA
:10CB480008BF43F0010350434FF47A7290FBF2F0B0
:10CB5800013080B243F400432084A3832388698989
:10CB6800AA889BB243F001032380238823F48163BE
:10CB780023F002031B040A431B0C13439BB22380BC
:10CB88002A89AB8913439BB223817FBD40420F00A2
:10CB9800A086010041F288330360002383804BF6AE
:10CBA800FF72038143814FF48043C28083817047C1
:10CBB800038819B19BB243F0010303E023F001039A
:10CBC8001B041B0C03807047038819B19BB243F404
:10CBD800807303E023F480731B041B0C03807047ED
:10CBE800038819B19BB243F4007303E023F4007384
:10CBF8001B041B0C0380704712B141F0010101E0D6
:10CC080001F0FE0101827047038819B19BB243F419
:10CC1800806303E023F480631B041B0C03807047CC
:10CC280083899BB201F0FE0123F0FE030B4383814D
:10CC38007047838919B19BB243F0010303E023F0E5
:10CC480001031B041B0C83817047038819B19BB235
:10CC580043F0400303E023F040031B041B0C038054
:10CC68007047038829B16FEA43436FEA53439BB285
:10CC780001E05B045B0C03807047038819B99BB221
:10CC880043F0800303E023F080031B041B0C0380A4
:10CC98007047B1F5804F838B04D023F480431B0485
:10CCA8001B0C02E09BB243F4804383837047B1F5C9
:10CCB800006F038803D19BB243F4006303E023F4BD
:10CCC80000631B041B0C03807047B1F5005F0388E9
:10CCD80003D19BB243F4005303E023F400531B0435
:10CCE8001B0C03807047038819B19BB243F01003F3
:10CCF80003E023F010031B041B0C03807047018220
:10CD08007047008AC0B27047038819B19BB243F4D8
:10CD1800805303E023F480531B041B0C03807047EB
:10CD2800B1F5006F038803D19BB243F4006303E0BD
:10CD380023F400631B041B0C03807047038819B19C
:10CD48009BB243F0200303E023F020031B041B0CD9
:10CD580003807047008BC0F307207047838819B1A0
:10CD68009BB243F4006303E023F400631B041B0C31
:10CD780083807047838819B19BB243F4805303E0E2
:10CD880023F480531B041B0C8380704782B000235C
:10CD980001930190019BCB180193019B188880B2E5
:10CDA80002B0704783889BB20AB1194301E023EAB5
:10CDB800010181807047838A008B9BB243EA00405F
:10CDC800084020F07F40431A584240EB0300704768
:10CDD800838A008B9BB243EA004020F07F40704773
:10CDE80082B00023009301930B0F01900093009BE6
:10CDF80021F07F4113B1019B143302E0019B090C20
:10CE080018330193019B1B6819420CBF00200120B5
:10CE180002B07047C94389B2818270478388808A8B
:10CE280080B208409BB206D001F0E06113EA1141DC
:10CE38000CBF002001207047C94389B28182704726
:10CE48000A4B1A6842F001021A6000229A601968B7
:10CE580021F0847121F480311960054959601968FD
:10CE680021F480211960DA60704700BF0038024061
:10CE780010300024024B00221A701870704700BF4F
:10CE880002380240034B1A6822F0F80242EAC00254
:10CE98001A60704700380240014B1860704700BFA5
:10CEA80000004742064B002201281A701A7002D06F
:10CEB800042804D101E01870704705221A707047E1
:10CEC80070380240014B1860704700BF800E47421F
:10CED800014341EA821200995B08013B42EA016181
:10CEE80041EA0341014B5960704700BF00380240D6
:10CEF800014B1860704700BF600047428001034B38
:10CF080040EA0171C3F88410704700BF003802403E
:10CF1800014B1860704700BF68004742014B18601A
:10CF2800704700BF4C004742034B9A6822F0EC62FE
:10CF380002430A439A60704700380240034B9A68DC
:10CF480022F0784202430A439A6070470038024050
:10CF5800034B9A6822F0030202439A60704700BFAD
:10CF680000380240024B986800F00C00704700BF80
:10CF780000380240034B9A6822F0F00202439A609C
:10CF8800704700BF00380240034B9A6822F4E05211
:10CF980002439A60704700BF00380240034B9A680A
:10CFA80022F4604242EAC0029A60704700380240A8
:10CFB8001E4B9A6802F00C02042A10B503D0082A06
:10CFC80003D01B4B18E01B4B16E059685A6811F444
:10CFD800800F596814BF174B154B02F03F02B3FB83
:10CFE800F2F3124A5268C2F30142C1F388110132C6
:10CFF8004B435200B3FBF2F30C4903608B680E4AB3
:10D008000468C3F30313D35C34FA03F343608C68F6
:10D01800C4F38224145D33FA04F484608968C1F38C
:10D028004231525CD340C36010BD00BF003802409B
:10D038000024F40000127A00D402002000F44073A7
:10D04800B3F5407F084B08D1996820F0704221F46D
:10D05800F81122F440720A439A601A6F000542EAF6
:10D0680010501867704700BF00380240014B186025
:10D07800704700BF3C0E4742014B1860704700BF25
:10D08800400E4742014B1860704700BF5C014742A1
:10D09800044B1A6B09B1104301E022EA000018633F
:10D0A800704700BF00380240044B5A6B09B1104367
:10D0B80001E022EA00005863704700BF00380240D0
:10D0C800044B9A6B09B1104301E022EA000098630F
:10D0D800704700BF00380240044B1A6C09B1104376
:10D0E80001E022EA00001864704700BF00380240DF
:10D0F800044B5A6C09B1104301E022EA000058645D
:10D10800704700BF00380240044B1A6909B1104348
:10D1180001E022EA00001861704700BF00380240B1
:10D12800044B5A6909B1104301E022EA0000586132
:10D13800704700BF00380240044B9A6909B1104398
:10D1480001E022EA00009861704700BF0038024001
:10D15800044B1A6A09B1104301E022EA0000186280
:10D16800704700BF00380240044B5A6A09B11043A7
:10D1780001E022EA00005862704700BF0038024010
:10D18800044B1A6D09B1104301E022EA000018654A
:10D19800704700BF00380240044B5A6D09B1104374
:10D1A80001E022EA00005865704700BF00380240DD
:10D1B800044B9A6D09B1104301E022EA000098651A
:10D1C800704700BF00380240044B1A6E09B1104383
:10D1D80001E022EA00001866704700BF00380240EC
:10D1E800044B5A6E09B1104301E022EA0000586668
:10D1F800704700BF00380240044B1A7809B1104349
:10D2080001E022EA00001870704700BF0D380240A4
:10D218004309012B074A01D1136803E0022B0CBF15
:10D22800136F536F00F01F0033FA00F000F0010095
:10D23800704700BF0038024007B500230193312032
:10D24800FFF7E6FF019B01330193019BB3F5A06F44
:10D2580001D00028F3D03120FFF7DAFF003018BFE3
:10D2680001200EBD024B5A6F42F080725A67704718
:10D2780000380240034BDB6818420CBF0020012035
:10D28800704700BF00380240014B1870704700BF5C
:10D298000E38024008B5154B98420BD101214FF4C6
:10D2A8008050FFF761FF4FF480500021BDE808402F
:10D2B800FFF75ABF0E4B984207D14FF48040012127
:10D2C800FFF746FF4FF4804009E00A4B98420BD124
:10D2D8004FF400400121FFF73BFF4FF400400021CD
:10D2E800BDE80840FFF734BF08BD00BF003001406B
:10D2F80000380040003C00400B88028810B54C887C
:10D3080023438C882343CC8823430C8923434C89AB
:10D3180023438C892343CC8902F44152234313438A
:10D328009BB20380838B23F400631B041B0C838351
:10D338000B8A038210BD838B23F47B6323F00F03D6
:10D348001B041B0C8383022303848B68F0B5858B35
:10D35800022BADB238D0294A8E889468002E14BFAB
:10D3680002260126240203D5946824F4000494605C
:10D37800D2F88440D2F884705268DFF884C002F092
:10D388003F02BCFBF2F2C4F388145443C7F30272A1
:10D39800B4FBF2F4CA88B2F5007F4FF00A0201D15B
:10D3A800240A02E07601B4FBF6F46243B2FBF3F31D
:10D3B80005330A229BB2B3FBF2F303F00102120217
:10D3C800C3F34F0392B200E000229C1EA4B2FE2CCD
:10D3D80028BF0022CC8828BF0223134323439BB2D3
:10D3E80003840B884A882B4343F4006313438A88D9
:10D3F80013438A8913439BB28383F0BD00380240EC
:10D4080000127A000023038043808380C380038155
:10D4180043818381C381072303827047002302224B
:10D42800038043808380C380826083817047038840
:10D4380019B19BB243F0400303E023F040031B04FF
:10D448001B0C03807047838B19B19BB243F4806334
:10D4580003E023F480631B041B0C83837047038859
:10D4680023F400631B041B0C038003889BB20B434B
:10D4780003807047B1F5804F038803D19BB243F412
:10D48800804303E023F480431B041B0C0380704794
:10D498004FF6FF639942038803D09BB243F480732D
:10D4A80003E023F480731B041B0C038070478388FC
:10D4B80019B19BB243F0040303E023F004031B04F7
:10D4C8001B0C83807047838819B19BB243F010030B
:10D4D80003E023F010031B041B0C83807047838B2D
:10D4E80023F47B6323F00F031B041B0C83830223A9
:10D4F80003840B88828BB3F5007F10B592B205D0F8
:10D50800002B0CBF4FF48073002301E04FF48073AD
:10D518004C8822438C88898942F4006222430A435A
:10D5280092B21343838310BD808980B27047818192
:10D538007047038819B19BB243F4005303E023F406
:10D5480000531B041B0C0380704703889BB243F4F1
:10D55800805303807047012902D0008B80B2704746
:10D56800808A80B27047008A80B2704783889BB2F5
:10D578000AB1194301E023EA0101818070470909D2
:10D5880001238B409BB21AB1828892B2134303E005
:10D59800828892B222EA0303838070470389194282
:10D5A8000CBF002001207047C94389B20181704730
:10D5B80010B584880089012301F00F0280B213FAA4
:10D5C80002F21040A4B205D009098B401C420CBFDE
:10D5D8000020012010BD01F00F0101238B40DB4327
:10D5E8009BB20381704700BF08B501214FF480400A
:10D5F800FFF7BAFD4FF480400021BDE80840FFF76F
:10D60800B3BD014B186070470038014001F00302B8
:10D6180089080A4B023130B5920053F821500F2483
:10D62800944025EA040443F8214053F8214010FAB5
:10D6380002F2144343F8214030BD00BF00380140D6
:10D64800014B1860704700BFDC002742014B18608F
:10D65800704700BF00042742024B186AC0F300203D
:10D66800704700BF0038014030B5048C24F0010435
:10D678002404240C0484058B048CADB2A4B225F0D8
:10D68800F305154324F00A0445EA031544F00104A0
:10D69800ADB20C430583048430BD30B5048C24F04E
:10D6A80010042404240C0484048B058C24F4407492
:10D6B800ADB22405240D25F0A00544EA022445F066
:10D6C800100544EA033445EA0115A4B2ADB2048357
:10D6D800058430BD08B5474B984205D10120014665
:10D6E800FFF742FD01203DE0B0F1804F05D1012058
:10D6F8000146FFF72DFD012076E03F4B984205D10A
:10D7080002200121FFF724FD02206DE03B4B9842E7
:10D7180005D104200121FFF71BFD042064E0384BEC
:10D72800984205D108200121FFF712FD08205BE08F
:10D73800344B984205D110200121FFF709FD102034
:10D7480052E0314B984205D120200121FFF700FD1E
:10D75800202049E02D4B984209D102200121FFF7F2
:10D7680003FD02200021BDE80840FFF7FDBC284B5F
:10D77800984207D14FF480300121FFF7F5FC4FF4B0
:10D788008030EFE7234B984207D14FF40030012156
:10D79800FFF7EAFC4FF40030E4E71F4B984207D14B
:10D7A8004FF480200121FFF7DFFC4FF48020D9E7F8
:10D7B8001A4B984205D140200121FFF7C9FC4020AF
:10D7C80012E0174B984205D180200121FFF7C0FCD9
:10D7D800802009E0134B98420BD14FF4807001214F
:10D7E800FFF7B6FC4FF480700021BDE80840FFF752
:10D7F800AFBC08BD00000140000400400008004024
:10D80800000C0040001000400014004000040140DB
:10D818000040014000440140004801400018004019
:10D82800001C0040002000401C4A038890429BB224
:10D8380012D002F5806290420ED0B0F1804F0BD02A
:10D84800A2F58032904207D002F58062904203D060
:10D8580002F58062904203D14A8823F07003134393
:10D868000F4A904208D002F58062904204D023F417
:10D8780040730A899BB2134303804B68C3620B88C9
:10D888000385064B984203D003F58063984201D183
:10D898008B7A038601238382704700BF0000014012
:10D8A800001000404FF0FF334360002303800381E2
:10D8B800438083727047018582827047038823F012
:10D8C80070031B041B0C0B430380704741627047B5
:10D8D800C1627047406A7047008D80B27047038804
:10D8E80019B19BB243F0020303E023F002031B04C7
:10D8F8001B0C03807047038819B19BB243F00403E3
:10D9080003E023F004031B041B0C03807047038807
:10D9180019B19BB243F0800303E023F080031B049A
:10D928001B0C03807047038823F008031B041B0C9F
:10D93800038003889BB20B4303807047038823F45A
:10D9480040731B041B0C038003889BB20B430380AA
:10D958007047038819B19BB243F0010303E023F039
:10D9680001031B041B0C03807047038C23F0010385
:10D978001B041B0C038470B5038C8488028B0D88F0
:10D988004E8822F073021204120C2A438D8923F068
:10D9980002031B0435431B0CADB22B430E4DA842AA
:10D9A800A4B203D005F58065A8420ED1CD894E8A70
:10D9B80023F008032B438D8823F004032B430D8A9F
:10D9C800354324F44074ADB22C43848002838A68C2
:10D9D8004263038470BD00BF00000140038C23F044
:10D9E80010031B041B0C0384038C828830B5048B42
:10D9F8000D8824F4E6442404240C23F0200344EA8C
:10DA080005241B048D891B0C43EA05134D8843EA42
:10DA18000513134DA84292B2A4B29BB203D005F5E8
:10DA28008065A84215D1CD8923F080039BB243EAD3
:10DA380005134FF6BF751D408B8845EA03130D8A01
:10DA480022F4406242EA85024D8A42EA85029BB28C
:10DA580092B282808A6804838263038430BD00BFE7
:10DA680000000140038C23F480731B041B0C038407
:10DA7800038C828830B5848B0D8824F073042404C9
:10DA8800240C23F400731B042C438D891B0C43EADC
:10DA980005234D8843EA0523124DA84292B29BB252
:10DAA80003D005F58065A84215D1CD8923F400631C
:10DAB8009BB243EA05234FF6FF351D408B8845EAA4
:10DAC80003230D8A22F4405242EA05124D8A42EAA3
:10DAD80005129BB292B282808A688483C2630384EF
:10DAE80030BD00BF00000140038C23F480531B04A9
:10DAF8001B0C0384038C30B58488828B0D8822F438
:10DB0800E6421204120C23F4005342EA05221B04D5
:10DB18008D891B0C43EA05334D8843EA05330B4DC9
:10DB2800A842A4B292B29BB203D005F58065A84280
:10DB380005D10D8A24F4804444EA8514A4B2848073
:10DB480082838A680264038430BD00BF00000140FC
:10DB5800002303804380838083608381C3810382A1
:10DB68004382704730B5058C0124ADB28C4025EA5C
:10DB7800040400F11803048409B1082907D14908ED
:10DB88004FF68F70CC582040C850C8580AE0043966
:10DB9800C1F34E0148F6FF70CC582040C85012021D
:10DBA800C85892B20243CA5030BD4163704781637E
:10DBB8007047C163704701647047038B23F070039B
:10DBC8001B041B0C0B4303837047038B23F4E043B4
:10DBD8001B041B0C43EA01239BB203837047838B0E
:10DBE80023F070031B041B0C0B4383837047838B48
:10DBF80023F4E0431B041B0C43EA01239BB28383F9
:10DC08007047038B23F008031B041B0C0B4303838F
:10DC18007047038B23F400631B041B0C43EA0123A6
:10DC28009BB203837047838B23F008031B041B0CF0
:10DC38000B4383837047838B23F400631B041B0C03
:10DC480043EA01239BB283837047038B23F00403C9
:10DC58001B041B0C0B4303837047038B23F4806363
:10DC68001B041B0C43EA01239BB203837047838B7D
:10DC780023F004031B041B0C0B4383837047838B23
:10DC880023F480631B041B0C43EA01239BB28383A8
:10DC98007047038B23F080031B041B0C0B43038387
:10DCA8007047038B09025B0441EA53439BB2038329
:10DCB8007047838B23F080031B041B0C0B43838367
:10DCC8007047838B09025B0441EA53439BB2838309
:10DCD8007047038C23F002031B041B0C0B430384C3
:10DCE8007047038C23F008031B041B0C0B430384AD
:10DCF8007047038C23F020031B041B0C43EA011319
:10DD08009BB203847047038C23F080031B041B0C15
:10DD180043EA01139BB203847047038C23F4007316
:10DD28001B041B0C43EA01239BB203847047038C3A
:10DD380023F400631B041B0C43EA01239BB20384F6
:10DD48007047038C23F400531B041B0C43EA013374
:10DD58009BB20384704710B5048C01238B40A4B296
:10DD680024EA03030384038C12FA01F10B439BB2E8
:10DD7800038410BD10B5048C04238B40A4B224EA9C
:10DD880003030384038C12FA01F10B439BB203844F
:10DD980010BD00230122038043808280C380038159
:10DDA8007047406B7047806B7047C06B7047006C62
:10DDB8007047038B23F00C031B041B0C0383038B9A
:10DDC8009BB20B4303837047038B23F440631B040C
:10DDD8001B0C0383038B9BB243EA01239BB203838F
:10DDE8007047F8B50C464988A288B4F800E0238942
:10DDF800054600290CBF02270027012A14BF012667
:10DE08000226BEF1000F10D1FFF72EFC2846E1884C
:10DE1800FFF7CFFF2846394632462389FFF73DFCF6
:10DE2800E1882846BDE8F840CEE7FFF736FC2846EB
:10DE3800E188FFF7C9FF2846394632462389FFF7AC
:10DE480013FCE1882846BDE8F840B2E7838B23F04D
:10DE58000C031B041B0C8383838B9BB20B438383B0
:10DE68007047838B23F440631B041B0C8383838BD1
:10DE78009BB243EA01239BB283837047F8B50D46F2
:10DE88000B88AA88498804463BB92B89FFF7ECFB25
:10DE9800E9882046BDE8F8408BE7042B07D12B8999
:10DEA800FFF7FBFBE9882046BDE8F8408CE7082B24
:10DEB800B5F808C0078C1DD127F480773F043F0CC4
:10DEC8000784868B038CB6B29BB226F0F30623F444
:10DED800206346EA0C1C43EA01211FFA8CFC89B234
:10DEE8004CEA020241F4807182830184E988BDE82A
:10DEF800F840ABE727F480573F043F0C0784868B34
:10DF0800038C26F4407623F4005336055B04360D63
:10DF18005B0C46EA022243EA013342EA0C329BB226
:10DF2800E98892B243F4805382830384BDE8F840C1
:10DF380097E74A880B8813438A881343CA88134390
:10DF48000A8913434A8913438A8913439BB2A0F869
:10DF5800443070470023038043808380C38003815B
:10DF6800438183817047B0F8443029B16FEA434355
:10DF78006FEA53439BB201E05B045B0CA0F84430AA
:10DF88007047838819B19BB243F0040303E023F080
:10DF980004031B041B0C83807047838819B19BB250
:10DFA80043F0010303E023F001031B041B0C8380EF
:10DFB800704783899BB20AB1194301E023EA010142
:10DFC8008181704781827047038A19420CBF002003
:10DFD80001207047C94389B201827047038A828948
:10DFE80011EA030092B203D011420CBF00200120B5
:10DFF8007047C94389B2018270470A43A0F8482094
:10E00800704783899BB20AB1194301E023EA0101F1
:10E0180081817047838819B19BB243F0080303E0FC
:10E0280023F008031B041B0C83807047038923F02B
:10E0380007031B041B0C03817047038923F070033B
:10E048001B041B0C0B43038103899BB243F007039A
:10E058000381704738B50D4611460122602D0446EC
:10E0680002D1FFF71AFB01E0FFF7FEFA238923F03C
:10E0780070031B041B0C1D43258123899BB243F0AD
:10E088000703238138BD038923F070031B041B0C8D
:10E098000B4303817047838823F070031B041B0C18
:10E0A800838083889BB20B4383807047038923F066
:10E0B80007031B041B0C038103899BB20B430381D9
:10E0C8007047038923F080031B041B0C0381038919
:10E0D8009BB20B430381704710B50489E4B20C432B
:10E0E800144344EA0324A4B2048110BD10B50446C5
:10E0F800FFF7F2FF23899BB243F48043238110BDCD
:10E1080010B50446FFF7E8FF238923F077031B04C3
:10E118001B0C43F07703238110BD70B50489068B6F
:10E12800058C26F44076ADB226F0030624F00704E9
:10E13800360425F022052404360C1543240C46F435
:10E14800807645EA0315214346F00106ADB2018108
:10E158000683058470BD838819B19BB243F08003A0
:10E1680003E023F080031B041B0C83807047A0F896
:10E178005010704708B5234B984205D11020012153
:10E18800FEF7F2FF102037E01F4B984207D14FF4FB
:10E1980000300121FEF7DCFF4FF4003009E01B4B93
:10E1A80098420BD14FF480200121FEF7D1FF4FF4A4
:10E1B80080200021BDE80840FEF7CABF144B9842F2
:10E1C80007D14FF400200121FEF7C2FF4FF40020D1
:10E1D800EFE7104B984207D14FF480100121FEF76A
:10E1E800B7FF4FF48010E4E70B4B984209D1202089
:10E1F8000121FEF7B9FF20200021BDE80840FEF705
:10E20800B3BF08BD00100140004400400048004072
:10E21800004C00400050004000140140038ACA88A6
:10E228009BB223F4405330B513430D4603828389D0
:10E238000989AA8823F4B0530A43698923F00C0397
:10E248001B040A431B0C92B213438381838AAA8955
:10E258009BB223F44073134385B083820446684617
:10E26800FEF7A6FE1A4B9C4203D003F580639C423E
:10E2780001D1039B00E0029BA28912B2002A4FF051
:10E2880019012A6801FB03F101DA520000E092004B
:10E298006423B1FBF2F1B1FBF3F21201100903FBA5
:10E2A8001011A08900B2002806DAC9003231B1FB8A
:10E2B800F3F303F0070305E009013231B1FBF3F38F
:10E2C80003F00F031A4392B2228105B030BD00BF9C
:10E2D800001001404FF4165303600C220023838082
:10E2E800C38003814281838170470B88028A10B5FD
:10E2F8004C8823438C88C988234392B20B4322F469
:10E3080070629BB21343038210BD002303804380D5
:10E318008380C3807047838919B19BB243F400534B
:10E3280003E023F400531B041B0C83817047038B09
:10E3380003F47F430383038B9BB20B430383704730
:10E34800838929B16FEA43436FEA53439BB201E0E3
:10E358005B045B0C83817047838A19B19BB243F4D9
:10E36800006303E023F400631B041B0C83827047E3
:10E37800C905C90D818070478088C005C00D7047E8
:10E38800038A23F00F031B041B0C0382038A9BB22E
:10E398000B4303827047838919B19BB243F0020390
:10E3A80003E023F002031B041B0C8381704783895D
:10E3B80023F400631B041B0C838183899BB20B43EA
:10E3C80083817047038A23F020031B041B0C0382FC
:10E3D800038A9BB20B4303827047038A19B19BB22D
:10E3E80043F4804303E023F480431B041B0C0382A3
:10E3F800704783899BB243F0010383817047838A06
:10E4080019B19BB243F0080303E023F008031B048F
:10E418001B0C83827047038BDBB20383038B9BB295
:10E4280043EA012303837047838A19B19BB243F0FF
:10E43800200303E023F020031B041B0C8382704796
:10E44800838A19B19BB243F0100303E023F0100351
:10E458001B041B0C83827047838A23F004031B046C
:10E468001B0C8382838A9BB20B4383827047838A07
:10E4780019B19BB243F0020303E023F002031B042B
:10E488001B0C83827047838A9BB20AB1194301E04F
:10E4980023EA010181827047C1F3421310B501F0EC
:10E4A8001F01012414FA01F1A34201D10C3004E048
:10E4B800022B01D1103000E0143003680AB119436F
:10E4C80001E023EA0101016010BD038819420CBF75
:10E4D800002001207047C94389B20180704701229A
:10E4E80010B501F01F03C1F342149A40012C01D169
:10E4F800838903E0022C0CBF038A838A9BB21340F2
:10E50800028892B243B1090A012313FA01F11142B8
:10E518000CBF0020012010BD184610BD090A0123B8
:10E528008B40DB439BB20380704700BF81F0004102
:10E5380002E000BF83F0004330B54FEA41044FEAE0
:10E54800430594EA050F08BF90EA020F1FBF54EA7B
:10E55800000C55EA020C7FEA645C7FEA655C00F017
:10E56800E2804FEA5454D4EB5555B8BF6D420CDDE8
:10E578002C4480EA020281EA030382EA000083EA6B
:10E58800010180EA020281EA0303362D88BF30BD0B
:10E5980011F0004F4FEA01314FF4801C4CEA113161
:10E5A80002D0404261EB410113F0004F4FEA0333C0
:10E5B8004CEA133302D0524263EB430394EA050F4B
:10E5C80000F0A780A4F10104D5F1200E0DDB02FABA
:10E5D8000EFC22FA05F2801841F1000103FA0EF24E
:10E5E800801843FA05F359410EE0A5F120050EF114
:10E5F800200E012A03FA0EFC28BF4CF0020C43FA45
:10E6080005F3C01851EBE37101F0004507D54FF051
:10E61800000EDCF1000C7EEB00006EEB0101B1F5A1
:10E62800801F1BD3B1F5001F0CD349085FEA3000E7
:10E638004FEA3C0C04F101044FEA445212F5800FF2
:10E6480080F09A80BCF1004F08BF5FEA500C50F18F
:10E65800000041EB045141EA050130BD5FEA4C0C72
:10E66800404141EB010111F4801FA4F10104E9D1FB
:10E6780091F0000F04BF01460020B1FA81F308BFF2
:10E688002033A3F10B03B3F120020CDA0C3208DDBE
:10E6980002F1140CC2F10C0201FA0CF021FA02F199
:10E6A8000CE002F11402D8BFC2F1200C01FA02F109
:10E6B80020FA0CFCDCBF41EA0C019040E41AA2BF2E
:10E6C80001EB0451294330BD6FEA04041F3C1CDAF6
:10E6D8000C340EDC04F11404C4F1200220FA04F016
:10E6E80001FA02F340EA030021FA04F345EA0301C0
:10E6F80030BDC4F10C04C4F1200220FA02F001FA82
:10E7080004F340EA0300294630BD21FA04F0294603
:10E7180030BD94F0000F83F4801306BF81F480119C
:10E728000134013D4EE77FEA645C18BF7FEA655C0F
:10E7380029D094EA050F08BF90EA020F05D054EAE1
:10E74800000C04BF1946104630BD91EA030F1EBFE6
:10E758000021002030BD5FEA545C05D140004941EA
:10E7680028BF41F0004130BD14F580043CBF01F5DD
:10E77800801130BD01F0004545F0FE4141F47001C3
:10E788004FF0000030BD7FEA645C1ABF194610469E
:10E798007FEA655C1CBF0B46024650EA013406BF9F
:10E7A80052EA033591EA030F41F4002130BD00BF5E
:10E7B80090F0000F04BF0021704730B54FF480641B
:10E7C80004F132044FF000054FF0000150E700BF9C
:10E7D80090F0000F04BF0021704730B54FF48064FB
:10E7E80004F1320410F0004548BF40424FF00001E8
:10E7F8003EE700BF42004FEAE2014FEA31014FEA2B
:10E8080002701FBF12F07F4393F07F4F81F0605179
:10E81800704792F0000F14BF93F07F4F704730B5E8
:10E828004FF4607401F0004521F0004120E700BF7B
:10E8380050EA010208BF704730B54FF000050AE002
:10E8480050EA010208BF704730B511F0004502D503
:10E85800404261EB41014FF4806404F132045FEA05
:10E86800915C3FF4DCAE4FF003025FEADC0C18BFAA
:10E8780003325FEADC0C18BF033202EBDC02C2F1A0
:10E88800200300FA03FC20FA02F001FA03FE40EA32
:10E898000E0021FA02F11444C1E600BF70B54FF032
:10E8A800FF0C4CF4E06C1CEA11541DBF1CEA135514
:10E8B80094EA0C0F95EA0C0F00F0DEF82C4481EA7C
:10E8C800030621EA4C5123EA4C5350EA013518BF9C
:10E8D80052EA033541F4801143F4801338D0A0FB89
:10E8E80002CE4FF00005E1FB02E506F00042E0FB36
:10E8F80003E54FF00006E1FB03569CF0000F18BF3C
:10E908004EF0010EA4F1FF04B6F5007F64F54074E3
:10E9180004D25FEA4E0E6D4146EB060642EAC62176
:10E9280041EA55514FEAC52040EA5E504FEACE2EE3
:10E93800B4F1FD0C88BFBCF5E06F1ED8BEF1004FE6
:10E9480008BF5FEA500E50F1000041EB045170BD62
:10E9580006F0004646EA010140EA020081EA0301A6
:10E96800B4EB5C04C2BFD4EB0C0541EA045170BDA2
:10E9780041F480114FF0000E013C00F3AB8014F11C
:10E98800360FDEBF002001F0004170BDC4F1000465
:10E99800203C35DA0C341BDC04F11404C4F12005E6
:10E9A80000FA05F320FA04F001FA05F240EA020041
:10E9B80001F0004221F0004110EBD37021FA04F677
:10E9C80042EB06015EEA430E08BF20EAD37070BD31
:10E9D800C4F10C04C4F1200500FA04F320FA05F090
:10E9E80001FA04F240EA020001F0004110EBD37092
:10E9F80041F100015EEA430E08BF20EAD37070BD02
:10EA0800C4F1200500FA05F24EEA020E20FA04F3DA
:10EA180001FA05F243EA020321FA04F001F0004189
:10EA280021FA04F220EA020000EBD3705EEA430EFA
:10EA380008BF20EAD37070BD94F0000F0FD101F029
:10EA48000046400041EB010111F4801F08BF013C62
:10EA5800F7D041EA060195F0000F18BF704703F0A0
:10EA68000046520043EB030313F4801F08BF013D27
:10EA7800F7D043EA0603704794EA0C0F0CEA1355E3
:10EA880018BF95EA0C0F0CD050EA410618BF52EA9D
:10EA98004306D1D181EA030101F000414FF00000A3
:10EAA80070BD50EA410606BF1046194652EA4306B1
:10EAB80019D094EA0C0F02D150EA013613D195EA25
:10EAC8000C0F05D152EA03361CBF104619460AD16D
:10EAD80081EA030101F0004141F0FE4141F4700177
:10EAE8004FF0000070BD41F0FE4141F4780170BD67
:10EAF80070B54FF0FF0C4CF4E06C1CEA11541DBFCC
:10EB08001CEA135594EA0C0F95EA0C0F00F0A7F8CD
:10EB1800A4EB050481EA030E52EA03354FEA0131FA
:10EB280000F088804FEA03334FF0805545EA13130D
:10EB380043EA12634FEA022245EA111545EA1065D5
:10EB48004FEA00260EF000419D4208BF964244F16C
:10EB5800FD0404F5407402D25B084FEA3202B61A8B
:10EB680065EB03055B084FEA32024FF480104FF45F
:10EB7800002CB6EB020E75EB030E22BFB61A7546D3
:10EB880040EA0C005B084FEA3202B6EB020E75EB66
:10EB9800030E22BFB61A754640EA5C005B084FEACE
:10EBA8003202B6EB020E75EB030E22BFB61A75469B
:10EBB80040EA9C005B084FEA3202B6EB020E75EBA6
:10EBC800030E22BFB61A754640EADC0055EA060E67
:10EBD80018D04FEA051545EA16754FEA06164FEAAA
:10EBE800C30343EA52734FEAC2025FEA1C1CC0D156
:10EBF80011F4801F0BD141EA00014FF000004FF0E3
:10EC0800004CB6E711F4801F04BF01430020B4F1A3
:10EC1800FD0C88BFBCF5E06F3FF6AFAEB5EB030C5B
:10EC280004BFB6EB020C5FEA500C50F1000041EB58
:10EC3800045170BD0EF0004E4EEA113114EB5C0425
:10EC4800C2BFD4EB0C0541EA045170BD41F48011F8
:10EC58004FF0000E013C90E645EA060E8DE60CEA00
:10EC6800135594EA0C0F08BF95EA0C0F3FF43BAF1D
:10EC780094EA0C0F0AD150EA01347FF434AF95EAD4
:10EC88000C0F7FF425AF104619462CE795EA0C0FB8
:10EC980006D152EA03353FF4FDAE1046194622E785
:10ECA80050EA410618BF52EA43067FF4C5AE50EA5F
:10ECB80041047FF40DAF52EA43057FF4EBAE12E74F
:10ECC8004FF0FF3C06E000BF4FF0010C02E000BF30
:10ECD8004FF0010C4DF804CD4FEA410C7FEA6C5C13
:10ECE8004FEA430C18BF7FEA6C5C1BD001B050EAB6
:10ECF800410C0CBF52EA430C91EA030F02BF90EAA1
:10ED0800020F0020704710F1000F91EA030F58BF5F
:10ED1800994208BF90422CBFD8176FEAE37040F0C1
:10ED2800010070474FEA410C7FEA6C5C02D150EA5F
:10ED3800013C07D14FEA430C7FEA6C5CD6D152EA1A
:10ED4800033CD3D05DF8040B704700BF84461046DF
:10ED580062468C461946634600E000BF01B5FFF7DE
:10ED6800B7FF002848BF10F1000F01BD4DF808EDAE
:10ED7800FFF7F4FF0CBF012000205DF808FB00BF7F
:10ED88004DF808EDFFF7EAFF34BF012000205DF8D9
:10ED980008FB00BF4DF808EDFFF7E0FF94BF012026
:10EDA80000205DF808FB00BF4DF808EDFFF7CEFF27
:10EDB80094BF012000205DF808FB00BF4DF808ED66
:10EDC800FFF7C4FF34BF012000205DF808FB00BF37
:10EDD8004FEA410212F5001215D211D56FF478737B
:10EDE800B3EB625212D94FEAC12343F0004343EA1E
:10EDF800505311F0004F23FA02F018BF40427047F9
:10EE08004FF00000704750EA013005D111F0004082
:10EE180008BF6FF0004070474FF00000704700BF18
:10EE28004A0011D212F5001211D20DD56FF4787381
:10EE3800B3EB62520ED44FEAC12343F0004343EAD6
:10EE4800505323FA02F070474FF00000704750EA21
:10EE5800013002D14FF0FF3070474FF0000070478B
:10EE68004FEA4102B2F1E04324BFB3F5001CDCF1E4
:10EE7800FE5C0DD901F0004C4FEAC0024CEA50701C
:10EE8800B2F1004F40EB830008BF20F0010070474B
:10EE980011F0804F21D113F13872BCBF01F000404E
:10EEA800704741F480114FEA5252C2F11802C2F180
:10EEB800200C10FA0CF320FA02F018BF40F0010001
:10EEC8004FEAC1234FEAD32303FA0CFC40EA0C00B3
:10EED80023FA02F34FEA4303CCE77FEA625307D1F0
:10EEE80050EA01331EBF4FF0FE4040F44000704727
:10EEF80001F0004040F0FE4040F40000704700BFC1
:10EF08004BB942B9002908BF002802D04FF0FF31A1
:10EF1800084600F037B882B0EC462DE9005000F002
:10EF28001BF8DDF804E002B00CBC7047F8B51446D5
:10EF380006460F461D4600F027F804FB01F300FBC8
:10EF48000535A4FB0023EB18069CB21A67EB0303F4
:10EF5800C4E90023F8BD00BFF8B5144606460F46BD
:10EF68001D4600F075F900FB05F5A0FB042304FB22
:10EF78000155EB18069CB21A67EB0303C4E900239A
:10EF8800F8BD00BF704700BF00292DE9F0071D46F6
:10EF9800C0F29E800024002DC0F2958007460D46E1
:10EFA80016469C46002B3ED18A4254D9B2FA82F3C7
:10EFB80043B1C3F1200620FA06F501FA03F19A409D
:10EFC80029439840160CB1FBF6F597B206FB1511CC
:10EFD8004FEA104C07FB05F34CEA01418B4209D973
:10EFE800891805F1FF3C80F015818B4240F21281AF
:10EFF800023D8918C3EB010CBCFBF6F306FB13C1F9
:10F0080080B207FB03F740EA0140874207D9591E3F
:10F01800821880F00581974240F20281023B43EA60
:10F028000542002303E08B420AD900231A46104602
:10F03800194614B1404261EB4101BDE8F007704741
:10F04800B3FA83F3002B40F087808C4501D38242CA
:10F05800ECD80122EBE712B90123B3FBF2F2B2FAC2
:10F0680082F6002E3AD1891A150C1FFA82FC012368
:10F07800B1FBF5F705FB17114FEA10480CFB07F633
:10F0880048EA01418E4207D9891807F1FF3802D2B0
:10F098008E4200F2DA804746891BB1FBF5F605FB84
:10F0A800161180B20CFB06FC40EA0140844507D9E2
:10F0B800711E821880F0B080944540F2AD80023E07
:10F0C80046EA0742B3E7E443524263EB430365E78A
:10F0D800404261EB41014FF0FF345CE7B240C6F1BA
:10F0E800200521FA05F320FA05F701FA06F9150CAF
:10F0F800B3FBF5F847EA09091FFA82FC05FB183744
:10F108004FEA19410CFB08F341EA0747B040BB42FC
:10F118000AD9BF1808F1FF3180F09580BB4240F250
:10F128009280A8F10208BF18FE1AB6FBF5F305FB9A
:10F1380013611FFA89F90CFB03F649EA01418E4273
:10F1480006D95F1E891878D28E4276D9023B891873
:10F15800891B43EA08438BE7C3F1200726FA07F81F
:10F168000CFA03F248EA020C21FA07F105FA03FA4D
:10F178004FEA1C4920FA07F5B1FBF9F845EA0A05F8
:10F1880009FB18172A0C1FFA8CFA0AFB08F142EA45
:10F198000747B94206FA03F609D917EB0C0708F135
:10F1A800FF324ED2B9424CD9A8F1020867447F1AFF
:10F1B800B7FBF9F209FB1271ADB20AFB02FA45EA94
:10F1C80001418A4507D9551E11EB0C0137D28A45F2
:10F1D80035D9023A614442EA08424FEA124C1FFA12
:10F1E80086F808FB0CF7360C95B208FB05F806FB09
:10F1F800057505EB184506FB0CFCAF4288BF0CF5FE
:10F20800803CCAEB01010CEB1546B14212D309D080
:10F2180000230CE76546EDE60E4646EA074206E798
:10F228000B46FCE61FFA88F800FA03F308EB0545DD
:10F23800AB42EDD2013A0023F9E63B4688E72A467D
:10F24800C9E79046B3E788466EE7023F891823E787
:10F258002DE9F00F144605460E46002B3FD18A4291
:10F268004AD9B2FA82F343B1C3F1200025FA00F279
:10F2780001FA03F69C4016439D40210CB6FBF1F2BF
:10F288002F0CA0B201FB126C00FB02F347EA0C46FC
:10F29800B34208D9571E361980F0FF80B34240F2B6
:10F2A800FC80023A3619F61AB6FBF1F301FB13613A
:10F2B800ADB200FB03F045EA0141884207D95E1E62
:10F2C800091980F0EC80884240F2E980023B43EA69
:10F2D8000242002310461946BDE8F00F70478B42E2
:10F2E80043D8B3FA83F4002C42D18B42234601D38E
:10F2F80082423BD80122EDE712B90123B3FBF2F4B5
:10F30800B4FA84F2002A40F08A80091B260CA7B2BE
:10F318000123B1FBF6F006FB10114FEA154C07FB71
:10F3280000F24CEA01418A4207D9091900F1FF3C71
:10F3380002D28A4200F2D3806046C2EB010CBCFBC9
:10F34800F6F206FB12C1ADB207FB02F745EA01452A
:10F35800AF4207D9511E2C1980F0A380A74240F272
:10F36800A080023A42EA0042B4E700231A46B1E715
:10F37800C4F1200722FA07F603FA04F3334321FA0B
:10F3880007FA4FEA134C01FA04FB20FA07F141EAA5
:10F398000B0BBAFBFCF70CFB17A61FFA83F84FEA16
:10F3A8001B4508FB07F945EA0645A94502FA04FA90
:10F3B80004D97A1EED18C0F088801746C9EB0505F8
:10F3C800B5FBFCF60CFB16521FFA8BFB08FB06F884
:10F3D8004BEA0241884503D9721EC91870D31646F4
:10F3E80046EA0742170C1FFA8AFC0CFB07F695B28F
:10F3F8004FEA1A430CFB05FC03FB056505EB1C45AE
:10F4080003FB07F3AE4288BF03F58033C8EB010165
:10F4180003EB1543994250D347D000235AE7944051
:10F42800C2F12008260C20FA08F721FA08F501FA9B
:10F4380002F9B5FBF6F847EA090906FB1855A7B221
:10F448004FEA194C4CEA054C07FB08F3634500FAF0
:10F4580002F509D91CEB040C08F1FF323DD26345D3
:10F468003BD9A8F10208A444C3EB0C02B2FBF6F3A3
:10F4780006FB13201FFA89F907FB03F249EA00414A
:10F488008A4206D9581E091925D28A4223D9023B35
:10F498000919891A43EA08433BE73A4603E7334622
:10F4A80015E70A4642EA004214E71FFA8CF100FA0F
:10F4B80004F001EB0545A842AFD2013A002309E761
:10F4C80088458CD9023EC9188AE7A9457FF675AFE9
:10F4D800023FED1872E70346DBE79046C4E70238BF
:10F4E80009192AE7002103E00A4B5B58435004310D
:10F4F80009480A4B42189A42F6D3094A02E0002307
:10F5080042F8043B074B9A42F9D3FAF7E5F900F0C1
:10F518000DF870473CA0050800000020A40B00204F
:10F52800A80B002038CF0020FEE70000984BF7B565
:10F538004FF4FA661E60974A974B984F1A60984A9C
:10F54800984B1A60984B42F210721A60974B6424D9
:10F558001C6001233B70964B4FF0FF321A60954BAD
:10F5680000251D70F8F79EFBF6F724FDF6F72EFD33
:10F57800F6F73CFDF7F716FB2046F7F793FFF7F78A
:10F5880037FB2046F7F78EFFF8F772FBF8F7C0F95C
:10F59800F7F796FF2046F7F785FFFAF7BFFA2046F8
:10F5A800F7F780FF4FF4FA50F7F7E8FE2046F7F731
:10F5B80079FFF7F74FFA2046F7F774FF2846F8F770
:10F5C80053F87D48F7F76EFFF4F7B0FD2046F7F7DC
:10F5D80069FF7A4B03F1100229468DE8240028467A
:10F5E8005A681B68F4F7A8FF3046F7F75BFF284610
:10F5F800F5F722FA4FF6FF70F5F734FA32200321B7
:10F608006F4A2B46F5F746FB96206E4A8C212B460F
:10F61800F5F740FB9620A0216B4A2B46F5F73AFBFD
:10F628006A4A2B469620B421F5F734FBFAF7E2F83C
:10F638005021DC20FAF7B1F83046F7F733FF644A77
:10F648002B46DC212846F5F725FB6248F7F72AFF09
:10F658002046F7F727FFF6F7C5FF2046F7F722FF02
:10F668009FED5D0AF8F718F82046F7F71BFFF7F744
:10F6780041FFF5F7D7FD2046F7F714FF14200146A0
:10F68800F6F720FD2846F6F773FD2046F7F70AFF40
:10F69800F6F7F2FE2046F7F705FFF7F77BFA204664
:10F6A800F7F700FFF6F7EEFF00B13D70F6F7F6FF4B
:10F6B80008B1FAF749F8494B00241C70F2F78AF9A7
:10F6C800F5F766FD08B9464802E0464B46481C7007
:10F6D800F2F797F9F6F7D0F9F8F7A7FFF8F7DAFF96
:10F6E800F8F72DFDF8F7E6FBFAF751F8FAF7A8F95D
:10F6F800FAF7A0F83D4B3E4E3E4D802814BF4FF41C
:10F7080080504FF4806018603B4BC010186037463B
:10F71800F6F7DAFF337833B1012B02D1F8F726F97F
:10F7280001E0F8F74BF900243C70F8F789FAF3F791
:10F738007FFFF9F745FF2A8812B2012A0FD12F4817
:10F748004FF40051FDF771F9F9F704F8F8F722FAC8
:10F758002A484FF400512246FDF767F92C80284BC0
:10F768001B7843B1FAF746F8F0209621FAF715F816
:10F778002448F7F78DFC244C2046FBF7BAFC0028F8
:10F78800C6D02378112BC3D1F9F742FFC0E700BFD9
:10F79800EC3B0020E0673500243C0020EC0D002005
:10F7A80080C3C9014442002018420020CC3B0020FD
:10F7B8001C3C0020A443002000127A00A078010815
:10F7C800A4980508BE980508CB980508D798050899
:10F7D800E0980508002D31010000FA44FC3B0020A8
:10F7E800D40E0020B43B0020C0100020183C00209C
:10F7F8001C420020BC0C00203042002000080240BF
:10F80800D80C002040420F00B53B002010B4314C0A
:10F818000180B1F5807F44608270C37052D00DD9E9
:10F82800B1F5806F39D017D9B1F5006F2ED0B1F589
:10F83800805F24D0FF2040B210BC704720293AD006
:10F8480014D9402930D08029F4D123494FF020120F
:10F85800C26081600020EEE7B1F5007FEAD11F4B5E
:10F868004FF00811C16083600020E4E71029E1D15E
:10F878001B494FF00122C26081600020DBE7194B71
:10F888004FF00111C16083600020D4E7164A4FF0A1
:10F898000213C36082600020CDE714494FF00412C0
:10F8A800C26081600020C6E7114B4FF04011C16073
:10F8B80083600020BFE70F4A4FF08013C360826067
:10F8C8000020B8E70C4A4FF01013C3608260002094
:10F8D800B1E700BFC497040802880508D287050865
:10F8E800C2890508C4870508C6870508CA870508A8
:10F8F80042880508C2880508E28705082DE9F00F47
:10F90800B2B02E9030932E9B00882E9C5B68309F5F
:10F91800A4682D90451E03EB4506BF082093289444
:10F928002C952F911F921E96319700F03A814FEA3D
:10F93800900A4FEACA0B00F003002F99299003F1AF
:10F94800080504EB0B00CDF884A0CDF8A8B01995F4
:10F958001A921B97189617912B90179A189E13882E
:10F968003380B2F802C0A6F802C09488B480D78861
:10F97800F78008361896219F199E0832179256F874
:10F98800041C56F8082C4FF0000A4FF0000B002F0B
:10F9980000F06982CDE904ABCDE906ABCDE902AB55
:10F9A800CDE900AB289CBC46029BDDF80C9025688D
:10F9B800C2FBC5394FF0000848EA030ACB46CDE937
:10F9C80002AB049BDDF814B0C1FBC53BCDF824B0F5
:10F9D800CDF82080DDE908ABC1EA02004AEA030A53
:10F9E800CDE904AB069BDDF81CB03268C0FBD53B03
:10F9F800CDF82CB0CDF82880DDE90AABC2EA0107C2
:10FA08004AEA030ACDE906AB9DE80108C7FBD50B16
:10FA1800CDF834B0CDF83080DDE90CAB4AEA000A05
:10FA280063680298CDE900AB0834DDF80CB0C1FB7F
:10FA3800C30BCDF83CB0CDF83880DDE90EAB4AEA0F
:10FA4800000ACDE902AB71680498DDF814B0C2FB76
:10FA5800C30BCDF844B0CDF84080DDE910AB4AEADD
:10FA6800000ACDE904AB0698DDF81CB0C7FBD30B40
:10FA7800CDF84CB0CDF84880DDE912ABC1EA0205FB
:10FA88004AEA000ACDE906AB9DE80108C5FBD30B9D
:10FA9800CDF854B0CDF85080DDE914AB08364AEA09
:10FAA800000ABCF1010CCDE900AB7FF47DAF2A9DC3
:10FAB80019982B9B2E18299F002F35D01868039F63
:10FAC800029BC2FBC03700241D971C94DDE91C452E
:10FAD80044EA0304CDE90245049B059DC1FBC035FA
:10FAE800002723952297DDE9224544EA0304CDE95E
:10FAF8000445C1EA0203079D069AC3FBD025259554
:10FB08002497DDE9244544EA02043368C3EA010185
:10FB1800CDE9064553465D46C1FBD0352795269766
:10FB2800DDE926AB4AEA030A069A029C0499039D7A
:10FB3800079FD30B059AE60BC90B46EA454043EAF3
:10FB4800474441EA424604F30F0500F30F0C199BA2
:10FB5800CCEA054706F30F001A9D1B9E2F604FEA5B
:10FB6800DA3A08334AEA4B4B0BF30F04C0EA044273
:10FB78006A600835711E19931A951B917FF4EDAED2
:10FB8800319A2F9E1E991F9BDDF880B0D000371840
:10FB98000D182F970BEB000A1F181E951F97CDF80D
:10FBA80080A0DDF8C0C01CF0030BCDF820B000F039
:10FBB80086802D9BDDF8BC80CDF808B05808DDF8AC
:10FBC80080A0DDF8A0B00690CDF81080049A1E9EA3
:10FBD80032F8025B069826F8025B0492BAF80270C3
:10FBE800BBF80230BAF80020BBF800401E9617FB9D
:10FBF80003F112FB04F6451E4FEAE17711EB060804
:10FC08002B4605F0010047EBE6790AF104020BF1F7
:10FC18000401002D3BD0A8B1B2F800C0BBF80470B5
:10FC2800548848881CFB07F518EB050749EBE5766F
:10FC380014FB00F917EB090846EBE97904320431A3
:10FC4800013B24D00F88B2F800C0568848888C88B9
:10FC580095881CFB07FC18EB0C0816FB00F7D088EE
:10FC6800CE8849EBEC7C15FB04F518EB07084CEB48
:10FC7800E77918EB050710FB06FC49EBE57417EB71
:10FC88000C0844EBEC7908320831023BDAD11F9AB0
:10FC980002994FEAD83545EA494404F30F0322F89C
:10FCA800023B4F1E0AF1020A1F9202978ED1DDF81D
:10FCB80080A0DDF820B00AEB4B0ACDF880A02C9E7E
:10FCC8002E98B50840683FD0209F47EA000212F0FE
:10FCD800030F00F1080307F1080214BF00210121F6
:10FCE8009F4298BF904294BF00260126314277D0A8
:10FCF80097E84200016001216C1EA942466004EAAF
:10FD0800010419D044B192E81200196002215C6024
:10FD180008320833A9420FD092E850001C605E6098
:10FD2800966802F1080BD2689E600231DA601033DF
:10FD3800A9420BF10802EFD1DDF880C0ED000CEB11
:10FD4800050B4019CDF880B02C9C14F0030343D068
:10FD58005A085400002A00F08E80209D40EA0507CA
:10FD680017F0030F209F14BF00250125011D3E1D1C
:10FD7800012B94BF002505F001058F4298BFB042C2
:10FD880094BF002101210D4275D039689200BF1837
:10FD9800A342016020971044C4EB03011CD0209BB0
:10FDA800013933F8024B0A4620F8024B01F00101F1
:10FDB80092B129B133F8021B013A20F8021B0BD08B
:10FDC8001C46014634F802CB21F802CB5D88A31CFF
:10FDD8004580881C023AF3D132B0BDE8F00F704775
:10FDE800B7F800C0A0F800C07C884480BE88868030
:10FDF800691EFE880C46BA4601F00101C680002C37
:10FE08009AD089B1B2F800B0A3F800B051885980EF
:10FE1800B2F804C0A3F804C0B2F806B00832A3F8D8
:10FE280006B00833013C87D016881E805188598057
:10FE3800B2F804B0A3F804B0B2F806C0A3F806C03C
:10FE480016891E8103F1080B5189ABF802109389BA
:10FE5800ABF80430D6891032023C0BF10803ABF83A
:10FE68000660E1D168E7289BCDE904ABCDE906AB94
:10FE7800CDE902AB1FE6194691E700BF2DE9F00F67
:10FE88009CB006780F900F9C40880F9DA4686D6801
:10FE98001990B3FBF6FA471E4FEA5A0804EB4709D4
:10FEA800AAEB480340460A940D951A97CDF86C8042
:10FEB8000C911492CDF82C901193002800F0B58184
:10FEC8001746199A199CCDF848809108CA001591CF
:10FED80004F00303A9181792169310971891760047
:10FEE80075084FEA450C002D00F03B840B9FDDF8A8
:10FEF800308047EA080010F0030F14BF00210121E9
:10FF080008F10404381D012E94BF002101F00101FD
:10FF1800804598BFA74294BF4FF000094FF00109F0
:10FF280011EA090F00F01D84BB46D8F80020012310
:10FF38006F1EAB42CBF8002007EA030721460246B2
:10FF480014D237B1246802230431021DAB42046085
:10FF58000CD20C46104654F8047B40F8047B4968E0
:10FF680002335160211D021DAB42F2D3DDF830800F
:10FF7800DDF82CB04FEA4C05664508EB05020BEBA3
:10FF88000503CCEB06001DD0013832F802CB014640
:10FF980023F802CB00F00100A1B128B132F8029B8E
:10FFA800013923F8029B0DD014461F4634F8029BF2
:10FFB80027F8029BB2F802A0A21CA3F802A0BB1C5F
:10FFC8000239F1D10C9ADDF83CC00B989CF80080FE
:10FFD800710053180A9E0C93159BCDF84C80451858
:10FFE80006EB48020B950E92002B00F0B18300241B
:08FFF8000025CDE90445CDE927
:020000040801F1
:10000000024507930D9913460A9AB3F804A0B2F873
:1000100006B0CDF804A0B3F806A00E881588CDF878
:1000200020B0CDF824A0DDE902AB15FB06F51AEBF4
:10003000050A4BEBE57BCDE902AB1F884888B2F897
:1000400002C0B3F80290B2F804808C88CDF8188012
:10005000DDE904AB16FB07F61AEB060A4BEBE67B71
:10006000DDE902671CFB00F5761910FB09F047EB90
:10007000E5771AEB000A4BEBE07BCDE902ABDDF84C
:1000800018B0DDF804C0B1F80680099D1BFB04F030
:1000900016EB000A47EBE07BDDE9026714FB0CF48A
:1000A000361947EBE477089C14FB08F00831083256
:1000B00008331AEB000418FB05F84BEBE0750798C2
:1000C00016EB080A47EBE87B0138CDE90245CDE99C
:1000D00004AB079099D1179E0E9C0A9B1899A719FB
:1000E0009A190E97169F002F73D00E9B31F8020BB2
:1000F00032F8024B33F8026BDDE90289DDE904AB2B
:1001000014FB00F47D1E10FB06F618EB040849EB07
:10011000E4791AEB060A4BEBE67B2F4605F001006B
:10012000CDE90289CDE904AB002D52D0002873D06F
:1001300031F8024B32F8020B33F8025B10FB04F685
:1001400014FB05F0DDE90245DDE90489A41945EB5E
:10015000E67518EB000849EBE079013FCDE902456F
:10016000CDE9048935D0C246CB46DDE902890D468A
:1001700014460497214628461A4630F8026B31F897
:10018000027B32F802CB6D8864885B8817FB06F728
:1001900018EB070816FB0CF649EBE7791AEB060794
:1001A00014FB05FA4BEBE67B15FB03FC8C1C931C44
:1001B0000499851C18EB0A0849EBEA7917EB0C0A3D
:1001C0004BEBEC7B8A1ECDE902890492D2D1CDE9BA
:1001D00004AB029D03990498DDF828A0059BEA0B67
:1001E000109D42EA4148129908F30F09A5F80090C2
:1001F000DDF84C90C70B0AEB8908281D4A1E47EA18
:100200004346CDF8288006F30F0410906C801292BC
:100210000AD00F9C267866E6DDE904AB0D4614464D
:100220000497DDE90289A5E7149F1B9B07EB830672
:100230001496119F002F00F0A681DDF864B0DDF860
:100240006480DDF834C04FEA9B09CDF81C904FEA7A
:10025000C90908F0030A0CEB090BCDF82090CDF882
:1002600010A0CDF824B0DDF83CC09CF80060750803
:100270004FEA450C002D00F07E820C990B980B9FE5
:1002800040EA010414F0030F14BF002201220C1DE8
:100290000430012E94BF002202F00102814298BF77
:1002A000A74294BF002301231A4200F06482BA4699
:1002B00001230F68691EAB42CAF80070024601EACA
:1002C0000307214614D237B127680223211D021DDE
:1002D000AB4207600CD20C46104654F8047B40F841
:1002E000047B496802335160211D021DAB42F2D3E9
:1002F000DDF83090DDF82C804FEA4C05664509EBBF
:10030000050208EB0503CCEB06001DD0013832F8DE
:1003100002BB014623F802BB00F00100A1B128B1E5
:1003200032F8025B013923F8025B0DD014461F46F8
:1003300034F802AB27F802ABB2F802C0A21CA3F853
:1003400002C0BB1C0239F1D1DDF82CA0DDF830B0C1
:10035000079876000AEB060C0BEB0608CDF82CC0CC
:10036000CDF83080002800F0F0810A9ADDF8348062
:100370005788B2F800A0DDF828909488B9F8069064
:10038000B8F8062084460D9841880588B8F804001E
:1003900017FB01F61AFB05F3B3461BEB03014FEA0B
:1003A000E67714FB00F047EBE3750F180A9B19FB87
:1003B00002F145EBE0750CF1FF3617EB010AB1468F
:1003C00006F0010008F1080203F1080345EBE17BA8
:1003D000002E00F0858048B3DDF834C01E88BCF8DC
:1003E00008405888518897889D88B2F80680B3F8ED
:1003F00006C016FB04F41AEB040A10FB01F14BEBE8
:10040000E4761AEB010415FB07FB46EBE17014EBF5
:100410000B011CFB08F640EBEB740832083311EBC0
:10042000060A44EBE67BB9F1010959D0CDE902ABEC
:10043000CB46B3F80080B3F808901688CDF8389012
:1004400018FB06F6DDE902895D8854889888918852
:10045000B2F806C0DF88B2F808A015FB04F418EB68
:10046000060810FB01F149EBE67918EB040817FBCD
:100470000CF749EBE47918EB010849EBE17918EB4B
:10048000070849EBE779CDE90289DDF838905D8905
:10049000548998899189B2F80EC0DE8919FB0AF750
:1004A000DDE9028915FB04F418EB070810FB01F1E4
:1004B00049EBE77918EB040849EBE47916FB0CF6F5
:1004C00018EB010449EBE17510321033A01945EB2C
:1004D000E671BBF1020BCDE90201AAD182468B463F
:1004E0000DF1200898E816006318049D9DB332F8BA
:1004F00002CB33F8026B16FB0CF4013D1AEB040A35
:10050000294605F001004BEBE47B25B358B132F8E6
:10051000028B33F8020B10FB08F71AEB070A4BEBC0
:10052000E77B691E17D01446184634F8025B30F892
:10053000027B52885B8817FB05F81AEB08064BEB29
:10054000E87713FB02FBA21C831C16EB0B0A47EB9C
:10055000EB7B0239E7D10F9DDDF8508095F800C0A4
:100560000A9A119E4FEADA3343EA4B4404F30F0030
:1005700028F8020B02EB4C07711E0A97CDF8508049
:1005800011917FF470AE1A9E0F9CB508A06842D0FE
:100590000A9F47EA000616F0030F07F1080200F170
:1005A000080314BF002101219F4298BF904294BFCD
:1005B0004FF0000A4FF0010A11EA0A0F7FD097E8C6
:1005C0004200016001216C1EA942466004EA010458
:1005D00019D044B192E81200196002215C6008321F
:1005E0000833A9420FD092E850001C605E60966804
:1005F00002F10804D2689E600231DA601033A94229
:1006000004F10802EFD1DDF828A0ED000AEB05099E
:100610004019CDF82890DDF868A01AF003034AD0FD
:100620005A085400002A00F0A480DDF828B040EAFF
:100630000B0515F0030F14BF002501250BF104066F
:10064000011D012B94BF002505F001058B4598BFC6
:10065000B04294BF4FF0000C4FF0010C15EA0C0FA4
:1006600000F08780DBF8001092009344A342016001
:10067000CDF828B01044C4EB03011CD00A9B01390B
:1006800033F8024B0A4620F8024B01F0010192B107
:1006900029B133F8021B013A20F8021B0BD01C468B
:1006A000014634F802CB21F802CB5D88A31C4580BB
:1006B000881C023AF3D11CB0BDE8F00F7047B7F8C0
:1006C0000090A0F800907C884480BE888680691ED7
:1006D000FE880C46B84601F00101C680002C92D07D
:1006E00091B111881980B2F802C0A3F802C0B2F823
:1006F00004A0A3F804A0B2F806900832A3F806906C
:100700000833013C3FF47FAF11881980B2F802C072
:10071000A3F802C0B2F80490A3F80490B2F806A0BF
:10072000A3F806A016891E8103F1080C5189ACF8C4
:1007300002109389ACF80430D6891032023C0CF1D7
:100740000803ACF80660DFD15DE70D9A0A9B4FF015
:10075000000A4FF0000BC8E600260027CDE9046729
:100760000A9A0D99CDE90267BCE430460B9B0C9ABE
:100770000EE4194682E730460B9B0C9AC6E500BF93
:1007800000B553EC102B42F2FB1223F00043C3F6EA
:10079000E972934285B026DD4FF6FF72C7F6EF721D
:1007A00093420BDD51EC100B02460B46FDF7C6FEE3
:1007B00002460B4643EC102B05B000BD684600F026
:1007C000BFFB00F0030001289DED000B9DED021B17
:1007D0001AD0022810D0F8B900F0D2FE53EC102B3A
:1007E00010461946E4E79FED101B00F0C9FE53ECDC
:1007F000102B10461946DBE700F0C2FE53EC102B1D
:10080000104603F10041D3E701F0F6FB53EC102B47
:10081000104603F10041CBE7012001F0EDFB53EC62
:10082000102B10461946C3E700000000000000002E
:100830002DE9F04759EC108BC9F30A56A6F57E74E2
:10084000073C132C4D46CA46474626DC002C4FDB9E
:100850004FF6FF76C0F20F0646FA04F606EA0905DF
:1008600055EA080517D044A3D3E9002351EC100B37
:10087000FDF766FE00220023FEF7A4FA00284AD006
:10088000B9F1000F6EDB2AEA060A4FF00008534662
:10089000424643EC102BBDE8F087332C0CDDB4F559
:1008A000806FF8D151EC100B3A460B46FDF748FE2D
:1008B00041EC100BBDE8F087A6F58265033D4FF0D3
:1008C000FF3323FA05F515EA080FE4D02AA3D3E98C
:1008D000002351EC100BFDF733FE00220023FEF73E
:1008E00071FAC0B1B9F1000F1CDB28EA050813E06A
:1008F00021A3D3E9002351EC100BFDF721FE0022C8
:100900000023FEF75FFA38B1B9F1000F1BDB4FF09F
:100910000008C24600E0CA465346424643EC102B4C
:10092000BDE8F087142C09D0C6F5866303334FF079
:10093000010808FA03F818EB0708D6D30AF1010AF0
:1009400028EA0508E8E729F0004848EA07084FF0D8
:10095000000AD045CBF6F07A08BFCA4618BF4FF060
:100960000008D9E74FF4801343FA04F409EB040AB2
:1009700089E700BFAFF300809C7500883CE4377EB8
:1009800000B553EC102B42F2FB1223F00043C3F6E8
:10099000E972934285B027DD4FF6FF72C7F6EF721A
:1009A00093420BDD51EC100B02460B46FDF7C6FDE2
:1009B00002460B4643EC102B05B000BD684600F024
:1009C000BFFA00F0030001289DED000B9DED021B16
:1009D0001DD0022812D008BB012001F00DFB53EC02
:1009E000102B10461946E3E700209FED111B01F084
:1009F00003FB53EC102B10461946D9E7012001F0F8
:100A0000FBFA53EC102B104603F10041D0E700F045
:100A1000B7FD53EC102B10461946C9E700F0B0FDA6
:100A200053EC102B104603F10041C1E7AFF30080F7
:100A3000000000000000000000F0E6B8D0B52DED89
:100A4000048BB0EE408AF0EE608A3C4C8AB000F035
:100A5000DBF994F90030B0EE409AF0EE609A013381
:100A600035D0B0EE480AF0EE680A01F04FFD0028DC
:100A70002DD051EC180B00220023FEF78FF930B374
:100A80002F4B24780193002308938DED028B8DED7D
:100A9000048B002C23D000270026CFF6F07751ECF2
:100AA000180B00220023CDE90667FEF763F9002842
:100AB00025D002239C42009336D0684601F05EFDAB
:100AC000002831D0089B002B27D19DED069BB0EE6E
:100AD000490AF0EE690A0AB0BDEC048BD0BD4FF6AE
:100AE000FF774FF06046CCF2EF7751EC180B002205
:100AF0000023CDE90667FEF73DF90028D9D101238F
:100B0000022C009315D0684601F038FD88B10D48DD
:100B100001F036FD8DED060BD4E701F0EFFF089BE9
:100B20009DED069B0360D2E701F0E8FF22230360FE
:100B3000C8E701F0E3FF21230360E8E7E4020020B7
:100B40003C9B0508A09D050810B52DED048BB0EE6B
:100B5000408AF0EE608A294C8AB000F02DFC94F9AE
:100B60000030B0EE409AF0EE609A01332BD0B0EE38
:100B7000480AF0EE680A01F0C9FC20B351EC180BEA
:100B800000220023FEF700F9E8B11D4B2478019301
:100B900001230093002308938DED048B8DED028BD0
:100BA000CCB10020002102460B46FDF7A5FF022C28
:100BB000CDE9060115D101F0A1FF21230360089BB7
:100BC000ABB99DED069BB0EE490AF0EE690A0AB09A
:100BD000BDEC048B10BD0022002343EC172B8DEDE0
:100BE000067B684601F0CAFC0028E8D1E3E701F083
:100BF00085FF089B9DED069B0360E4E7E40200206F
:100C0000449B050800000000F8B5B0EE407AF0EE15
:100C1000607A53EC112B544210461D46002125F0FA
:100C20000047044353EC102B47EAD474C7F6F07125
:100C30008C4216463DD85442344323F0004242EAE7
:100C4000D4748C4235D805F1404101F5801101433F
:100C50004FD0AC1704F00204164344EAD37435D0E5
:100C6000384341D00021C7F6F0718F424FD00021A8
:100C7000C7F6F0718A4237D0D21B12153C2A42DCEB
:100C8000002D7DDB53EC112B51EC170BFDF734FFDE
:100C900041EC100B01F030FC01F06AFA51EC100B42
:100CA000012C68D0022C57D0002C48D141EC170BF6
:100CB00007E051EC170B53EC112BFDF741FC41EC15
:100CC000170BB0EE470AF0EE670AF8BD032CC7D841
:100CD00001A151F824F000BFC30C0108C30C0108A6
:100CE000010D0108FB0C0108002B25DB9FED307B7B
:100CF000E7E7BDE8F84001F03BBA9FED2F7BE0E766
:100D00009FED2F7BDDE72AA1D1E90001C8E7BA42B8
:100D10003CD0032CABD801A151F824F0330D0108CD
:100D20002D0D0108010D0108FB0C01089FED267B2C
:100D3000C7E79FED277BC4E79FED277BC1E730A383
:100D4000D3E90023FDF7FAFB1DA3D3E90023FDF748
:100D5000F5FB41EC170BB4E729A3D3E90023FDF71A
:100D6000EDFB02460B4616A1D1E90001FDF7E6FBBB
:100D700041EC170BA5E701F1004141EC170BA0E78F
:100D80003C32BFF67FAF0020002189E7032CABD8AF
:100D9000DFE804F00B0805029FED117B91E79FED62
:100DA000127B8EE79FED127B8BE79FED137B88E72D
:100DB000182D4454FB21F93F182D4454FB2109C040
:100DC000182D4454FB210940000000000000008061
:100DD0000000000000000000182D4454FB21F9BF62
:100DE000D221337F7CD902C0D221337F7CD902400B
:100DF000182D4454FB21E9BF182D4454FB21E93F31
:100E0000075C143326A6A13C2DE9F84F55EC104B96
:100E1000B5F5801F2F4622DA25F00043234368D022
:100E2000002D2046294670DB00230022C4F25033F7
:100E3000FDF738FD4FF6FF730F46C7F6EF739F427D
:100E400004460D466FF0350210DD20462946224645
:100E50002B46FDF775FB41EC100BBDE8F88F4FF604
:100E6000FF73C7F6EF7300229F42EEDC3B15A3F53C
:100E70007E73073B9A18D60F901927F07F47C6F567
:100E80007E76FDF7A9FC073627F4700747EA06557A
:100E900045EC104B8046894601F00AFC4046494625
:100EA00021A3D3E9002355EC104BFDF7FBFC20A355
:100EB000D3E9002382468B4640464946FDF7F2FCC3
:100EC0001DA3D3E9002306460F4620462946FDF719
:100ED000E9FC02460B4630463946FDF731FB024637
:100EE0000B4650465946FDF72BFB41EC100BBDE875
:100EF000F88F00210020CCF2503100220023FDF7B2
:100F0000FBFD41EC100BBDE8F88F22462B46FDF7A8
:100F100015FB00220023FDF7EFFD41EC100BBDE8AF
:100F2000F88F00BFAFF3008000609F501344D33FA1
:100F3000362BF111F3FE593D0EE526157BCBDB3F39
:100F40002DE9F04F53EC102B42F2FB1223F000443A
:100F5000C3F6E97294428FB01E46074640F3AA805A
:100F60004DF67B13C4F202039C422ADC002E51ECA6
:100F7000100BDDA3D3E9002340F3CA81FDF7DEFAAD
:100F800042F2FB13C3F6F9739C428046894600F097
:100F9000AA80D7A3D3E90023FDF7D0FA0D46044673
:100FA0002B462246C7E9004540464946FDF7C6FAAA
:100FB000CFA3D3E90023FDF7C1FA0125C7E9020158
:100FC00081E042F2FB13C4F239139C4240F3AA8041
:100FD0004FF6FF73C7F6EF739C4278DC4FEA245A52
:100FE000AAF5826AAAF1060A51EC100BA4EB0A5387
:100FF00019461D460446FDF7EFFEFDF7EDFB804662
:10100000894642464B4620462946CDE90889FDF7E8
:1010100095FA00230022C4F27013FDF743FC0D463D
:101020000446FDF7D9FEFDF7D7FB804689462046EA
:10103000294642464B46CDE90A89FDF77FFA00234F
:101040000022C4F27013FDF72DFC002204460D4669
:101050000023CDE90C45FDF78DFE002800F07B81D3
:101060004046494600220023FDF784FE03240AADD2
:10107000013C40B175E9020100220023FDF77AFE30
:10108000013C0028F6D12346022400949E4C08A877
:1010900039465246019400F0ABFB002E054612DAA9
:1010A0007A68FB6802F1004203F100437A60FB605A
:1010B000454208E00022002343EC172B87ED000B8C
:1010C00080ED027B002528460FB0BDE8F08F51EC83
:1010D000100B02460B46FDF731FA0025C7E9020165
:1010E000C7E90001EFE77AA3D3E90023FDF726FA69
:1010F00079A3D3E9002380468946FDF71FFA0D4600
:1011000004462B462246C7E9004540464946FDF7BE
:1011100015FA71A3D3E90023FDF710FA0125C7E9F9
:101120000201D0E701F0E8F959EC108B6CA3D3E988
:10113000002340464946FDF7B5FB00230022C3F6D5
:10114000E073FDF7FDF9FDF747FE0546FDF744FBAB
:1011500065A3D3E90023CDE90201FDF7A3FB024615
:101160000B4640464946FDF7E9F961A3D3E9002360
:1011700082468B46DDE90201FDF794FB1F2DCDE988
:101180000401504659462BDC6A1E604B53F822304E
:10119000A34225D0DDE90423FDF7D0F902460B4632
:1011A000C7E90023814688464A4643465046594689
:1011B000FDF7C4F9DDE90423FDF7C0F9002E02466E
:1011C0000B46C7E90223BFF67EAF08F1004301F1E9
:1011D0000041C7F800907B60B860F9606D4272E72B
:1011E000DDE90423FDF7AAF988462415C8F30A535C
:1011F000E31A102B8146C7E90001D5DD34A3D3E9FA
:101200000023DDE90201FDF74DFB80468946424699
:101210004B4650465946FDF791F9CDE90601DDE907
:10122000062350465946FDF789F942464B46FDF7DD
:1012300085F929A3D3E9002380468946DDE9020127
:10124000FDF730FB42464B46FDF778F9CDE9040146
:10125000DDE90423DDE90601FDF770F98846C8F3EE
:101260000A53E41A312C8146C7E9000140F3958006
:1012700021A3D3E90023DDE90201FDF713FB80463A
:10128000894642464B46DDE90601FDF757F982469D
:101290008B4652465B46DDE90601FDF74FF94246B3
:1012A0004B46FDF74BF916A3D3E900238046894648
:1012B000DDE90201FDF7F6FA42464B46FDF73EF93D
:1012C000CDE904015046594664E700BFAFF3008002
:1012D0000000601A61B4D03D7370032E8A19A33BDD
:1012E00083C8C96D305FE43F00004054FB21F93FE3
:1012F0003163621A61B4D03D0000002E8A19A33B0D
:10130000C14920259A837B39CC9B05084C9B050855
:10131000FDF716F942F2FB13C3F6F9739C428046BF
:1013200089461AD01EA3D3E90023FDF709F90D461B
:1013300004462B462246C7E9004540464946FDF78C
:10134000FDF817A3D3E90023FDF7FAF84FF0FF35B6
:10135000C7E90201B7E6032495E613A3D3E9002306
:10136000FDF7EEF812A3D3E9002380468946FDF786
:10137000E7F80D4604462B462246C7E9004540469D
:101380004946FDF7DBF80AA3D3E90023FDF7D8F8B7
:101390004FF0FF35C7E9020195E6DDE906AB03E74B
:1013A0003163621A61B4D03D0000601A61B4D03D6F
:1013B0007370032E8A19A33B2DE9F84353EC102BCD
:1013C00000242546C7F6F074C7F6F0751C40AC4201
:1013D0002DED028BB0EE408AF0EE608A1946104681
:1013E00000F0AB80002B7FDD1A1500F08980A2F59C
:1013F0007E7721F07F4323F47003073FD20743F445
:10140000801366D5C20F4FF0000C02EB43037F1030
:101410004200654616204FF400116C18D60F9C420E
:101420004FEA420202DC65181B1B8C444908013854
:1014300006EB4303F1D1202680464FF0004107E040
:1014400043D0D40F49085200013E04EB43031BD0A4
:10145000AB4208EB0104F3DD04F00049B9F1004FA1
:1014600004EB01082BD0A9469442C5EB0303C4EB5F
:10147000020288BF013B4018D40F49085200013EC8
:101480004D4604EB4303E3D11A4327D146084FEA04
:101490006C0101F17E511CF0010F01F5C00118BF74
:1014A00046F0004601EB0753324643EC182BB0EEF2
:1014B000480AF0EE680ABDEC028BBDE8F883B8F18B
:1014C000000FD0DB05F10109CEE79442C4D91D46D7
:1014D000B7E7C20F02EB4303400093E7431C39D048
:1014E00000F001031818D1E723F000441443DED0C4
:1014F000002B36D11A46C10A153A40050029FAD008
:1015000011F4801329D149000133CC02FBD5C3F17A
:101510000105C3F1200420FA04F452192143984034
:10152000A2F57E7721F07F4323F47003073FD207B3
:1015300043F480133FF566AFCBE751EC100BFDF79A
:10154000B1F902460B4651EC180BFCF7F9FF41ECE0
:10155000180BACE70CF1010C99E7202401250023BE
:10156000D9E751EC100B0B46FCF7E8FF02460B469F
:10157000FDF7C2FA41EC180B99E700BF000000002C
:101580002DE9F04F5BEC10AB2DED028BB0EE418AF4
:10159000F0EE618A2BF00044B4F1795F85B071DA26
:1015A00050465946FDF718FC002800F0FD805246D1
:1015B0005B4650465946FDF775F981A3D3E90023F0
:1015C00006460F46FDF76EF97FA3D3E90023FCF72B
:1015D000B7FF32463B46FDF765F97DA3D3E900230B
:1015E000FCF7ACFF32463B46FDF75CF97AA3D3E942
:1015F0000023FCF7A5FF32463B46FDF753F978A3DD
:10160000D3E90023FCF79AFF32463B46FDF74AF93F
:1016100075A3D3E90023FCF793FF32463B46FDF761
:1016200041F98046894600230022C3F6E073304624
:101630003946FDF737F94246CDE900014B463046C1
:101640003946FDF72FF953EC182B04460D4650464A
:101650005946FDF727F902460B4620462946FCF776
:101660006DFF02460B46DDE90001FCF767FF0B4604
:1016700000210246C3F6F0710020FCF75FFF41EC49
:10168000100B83E052465B4650465946FDF70AF977
:101690004BA3D3E9002306460F46FDF703F94AA3FF
:1016A000D3E90023FCF74CFF32463B46FDF7FAF83E
:1016B00047A3D3E90023FCF741FF32463B46FDF741
:1016C000F1F845A3D3E90023FCF73AFF32463B4645
:1016D000FDF7E8F842A3D3E90023FCF72FFF3246D9
:1016E0003B46FDF7DFF840A3D3E90023FCF728FFD2
:1016F0003B463246FDF7D6F843F23233C3F6D37396
:101700009C42804689468EDD0023C3F6E9739C42E5
:1017100041DC0021A4F5001300220020C3F6F07183
:1017200014461D46FCF70AFFCDE902010023002202
:10173000C3F6E07330463946FDF7B4F822462B462F
:10174000FCF7FCFE4246CDE900014B4630463946E7
:10175000FDF7A8F853EC182B04460D4650465946A1
:10176000FDF7A0F802460B4620462946FCF7E6FEA8
:1017700002460B46DDE90001FCF7E0FE02460B469F
:10178000DDE90201FCF7DAFE41EC100B05B0BDEC1F
:10179000028BBDE8F08F9FED067B00258DED027B6F
:1017A0000024C3F6D275C1E79FED030BEEE700BF3F
:1017B000000000000000E73F000000000000F03FD4
:1017C000D43888BEE9FAA8BDC4B1B4BD9EEE213EAE
:1017D000AD529C804F7E923E9015CB19A001FA3EEF
:1017E0007751C1166CC1563F4C5555555555A53FBF
:1017F0002DE9F04F4AF6AB25ADF51B7DD41EC2F6A0
:10180000AA2585FB0465E417A49F114E0690C4EB3E
:10181000A50424EAE47456F827600A941F46E343BB
:1018200003EB43037C1E02EBC30314EB060809968B
:1018300002940891079321D40A9EA599351B08F1BB
:1018400001080CAE4FEA8808002401EB85090BE083
:10185000D49C050859F80400FCF7BEFF0434013598
:101860004445E6E9020109D0002DF3DA04340020F2
:10187000002101354445E6E90201F5D1099C002C1F
:101880002CDB099C5EAE06EBC4060DF5B87ABB46B0
:101890000096029D002DC0F254820EA9069D01EB18
:1018A000CB064FF000084FF00009002476E9022330
:1018B000F5E80201FCF7F6FF02460B4640464946B2
:1018C000FCF73EFE0134BC4280468946EED1EAE98F
:1018D0000289009DAA450BF1010BDAD1099E731E06
:1018E0009B0086AC9AAD04EB8604ED180B93009632
:1018F0000C940D95009C009EE4009AAD2B19002ECF
:10190000049453E93C892EDD04995EAC059485AEC0
:10191000651800230022C3F6706340464946FCF771
:10192000C1FFFDF759FAFCF757FF00230022C4F26C
:10193000701382468B46FCF7B5FF02460B464046C5
:101940004946FCF7FBFDFDF747FA044646F8044F0D
:1019500075E9020152465B46FCF7F2FD059CA54283
:1019600080468946D5D149EC108B079800F010FECF
:1019700055EC104B00224FF07F5320462946FCF7D0
:1019800091FF41EC100BFEF753FF002351EC100BBD
:101990000022C4F22003FCF785FF02460B462046D6
:1019A0002946FCF7CBFD0D460446FDF715FA064621
:1019B000FCF712FF02460B4620462946FCF7BEFD07
:1019C000079D002D8046894640F3C180009C9AAD5A
:1019D000621E05EB8202079C52F8503CC4F11800CD
:1019E00043FA00F101FA00F01B1AC4F1170076184F
:1019F00042F8503C43FA00F5002D30DD009C0136E2
:101A0000002C40F3B18186AA02EB840000244FF63B
:101A1000FF7352F8041BC0F2FF035B1A14B9C1F143
:101A2000807311B142F8043C01248242EFD107993E
:101A3000002911DD012900F06D8102290CD1009AE5
:101A40009AA9531E01EB830353F8502C22F07F42D6
:101A500022F4400243F8502C022D00F082804046D0
:101A6000494600220023FDF785F9002800F09C80FC
:101A7000009C601E099C84420EDC009C86A901EB40
:101A800084030C9C002253F8041DA34242EA010285
:101A9000F9D1002A40F070820D9C54F8503C002B84
:101AA00040F068820B9D86AE7219012352F8041D26
:101AB00001330029FAD0009CE31804F1010A9A4589
:101AC000059341DC0A9E029D04EB060BA59C05EBE9
:101AD0000A0304EB8B0B049C013B0EAD5EAE05EBE1
:101AE000C3053619009504965BF8040FFCF774FEE5
:101AF000009D029EE5E90201002E00954FF00008CE
:101B00004FF0000917DB0AEB07060EA9069D01EB53
:101B1000C606002476E90223F5E80201FCF7C2FEBE
:101B200002460B4640464946FCF70AFD0134BC42DA
:101B300080468946EED1049C059DE4E902890AF1BC
:101B4000010AAA450494CFDD059E0096D2E640F036
:101B5000EF80009D9AA901EB850353F8545CED15C5
:101B60004AE7002142464B460020C3F6F071FCF7DD
:101B7000E5FC80468946002C3FF471AF07989FED45
:101B80008E0B00F005FD404653EC102B4946FCF748
:101B9000D5FC804689464046494600220023FDF791
:101BA000E9F800287FF464AF05960495002840F01A
:101BB000FC81079C49EC108B604200F0E9FC57EC7B
:101BC000106B0023304639460022C4F27013FDF733
:101BD000EFF8002800F0F78100230022C3F67063BD
:101BE00030463946FCF75EFEFDF7F6F8FCF7F4FDEB
:101BF00000230022C4F2701380468946FCF752FE8F
